:100000000C9420080C943F080C943F080C947D0B32
:100010000C94B30B0C943F080C943F080C943F08CD
:100020000C943F080C943F080C943F080C943F0834
:100030000C943F080C943F080C943F080C94540F08
:100040000C943F080C943F080C943F080C943F0814
:100050000C94B65E0C94C2550C943F080C943F0867
:100060000C943F080C9498560C943F080C948C56B2
:100070000C943F080C943F080C943F080C943F08E4
:100080000C94796A0C943F080C943F080C943F0838
:100090000C94D6560C943F080C94CA560C943F0806
:1000A0000C943F080C943F080C943F080C943F08B4
:1000B0000C943F080C943F080C943F080C943F08A4
:1000C0000C943F080C943F080C943F080C943F0894
:1000D0000C943F080C943F080C943F080C943F0884
:1000E0000C943F080C946F5E0C94795E0C94655EE2
:1000F0000C941F5E0C94AA5E0C949B5E0C948F5E15
:100100000C94835E0C943F080C943F080C943F08B9
:100110000C943F080C943F080C943F080C943F0843
:10012000084AD73B3BCE016E84BCBFFDC12F3D6C5E
:1001300074319ABD56833DDA3D00C77F11BED9E4C4
:10014000BB4C3E916BAAAABE000000803F076342F1
:1001500036B79BD8A71A39685618AEBAAB558C1D5E
:100160003CB7CC5763BD6DEDFD753EF6177231BFE0
:10017000000000803F08000000BE922449123EAB00
:10018000AAAA2ABECDCCCC4C3E00000080BEABAAB1
:10019000AAAA3E00000000BF000000803F0000004F
:1001A0000000084178D3BB4387D1133D190E3CC3EF
:1001B000BD4282AD2B3E68EC8276BED98FE1A93E6E
:1001C0004C80EFFFBE01C4FF7F3F000000000050E5
:1001D0003A20256C642050612020252D372E326670
:1001E000206D0A002563002563004932433A200050
:1001F00025630074746C3D252D64200074746C3D7F
:10020000252D6420004E65772074746C3D252D6487
:100210002000256300256C642050612020252D37A7
:100220002E3266206D00256C64204320002563007B
:10023000545F52483D252D342E3166200052483DF2
:10024000252D342E316620002563002563002563AB
:100250000025630043757272656E74207265706F5D
:10026000727420696E74657276616C3D252D642010
:100270007365630A004E6577207265706F72742033
:10028000696E74657276616C3D252D6420736563BB
:100290000A002563007265706F72745F616C6C3D5B
:1002A000007265706F72743D002563002563002540
:1002B0006300256300204F534343414C3D25642098
:1002C0000020467573653A2065653D2530327820FB
:1002D00068663D25303278206C663D2530327820C6
:1002E0006C623D25303278004D43553D2530366CEB
:1002F0007800256300252D31306C7520252D313097
:100300006C7520252D31306C7520252D31306C75A4
:10031000200A007478206C656E20202020207268EE
:10032000206D697373202020207268207374616CC3
:10033000652020207268206D6973630A00256300C0
:100340004F4B0A00256300256300256300256300E9
:1003500025630064656275675F616C6C3D00646570
:100360006275673D0064656275673D0025730A002C
:1003700025372E33662025372E33660025352E325D
:100380006620004572726F72203020566F6C7400C8
:100390004E6F7420737570706F727465640A0045D7
:1003A00072726F72203020566F6C74004572726FDB
:1003B00072203020566F6C740025730A0073656ECE
:1003C000743D252D75206475703D252D7520696758
:1003D0006E6F7265643D252D752074746C5F7A654F
:1003E000726F3D252D750A0074787077723D256413
:1003F0000A006368616E3D25640A005465737420C9
:10040000362025730A005465737420352025730A3D
:10041000005465737420342025730A005465737486
:1004200020332025730A005465737420322025730D
:100430000A005465737420312025730A0025730A5D
:100440000025730A00646565700A00666F72636553
:100450005F69646C650A006E6F6E650A0070777282
:10046000733D005854414C5F5452494D3D25640042
:1004700025730A00696E74725F7365635F70313D46
:10048000252D372E33660A00696E74725F70313D18
:10049000252D6C640A00696E74725F7365635F700A
:1004A000303D252D372E33660A00696E74725F70F9
:1004B000303D252D6C640A00765F6D63753D252DFA
:1004C000352E32660A00707077723D25730A00641B
:1004D000656275673D0025730A006175746F0A00D7
:1004E0006C6F675F6D6F64653D007573625F7077F9
:1004F000723D25730A007265706F72745F6D61736F
:100500006B3D007265706F72745F696E74657276B0
:10051000616C3D252D640A0072656C61793D25731F
:100520000A0074746C3D252D640A0052494D455FE4
:10053000616464723D252D642E252D640A006E656C
:10054000696768626F725F7461626C655F73697A14
:10055000653D25640A00747870773D25640A006360
:1005600068616E3D25640A006932633D0069643D3F
:10057000007478743D25730A0053797374656D2097
:1005800053756D6D6172790A00706100700061646D
:1005900034006164330061643200616431006133AE
:1005A00000613200613100765F696E00726800752B
:1005B0007074696D650070315F7400703100703067
:1005C0005F7400703000765F6D637500745F6D63FB
:1005D0007500743100740069640065363400747805
:1005E00074006175746F006E6F6E650072656C618A
:1005F000795F6C65647900636F6D7061737300611E
:100600006363656C007072657300705F7077720071
:100610006165730070315F6C6564790070305F6C88
:10062000656472006576656E74006C6564006F7752
:1006300000706B740074785F6C6564790072785F29
:100640006C656472006F706572006E6F6E65002578
:1006500030327800765F6164343D252D382E366661
:10066000002000765F6164333D252D382E3666000C
:100670002000765F6164323D252D382E36660020DD
:1006800000765F6164313D252D382E3666002000EE
:10069000765F6C696768743D252D382E36660020BC
:1006A00000765F61323D252D372E336600200076BF
:1006B0005F61313D252D372E3366002000765F695E
:1006C0006E3D252D352E326600204E657665722DE5
:1006D0007573656420737461636B203E202564200C
:1006E00062797465730A00757074696D653D252DB6
:1006F000642D646179732D253032643A253032647B
:100700003A253032642D686F7572730A0074657310
:1007100074205B6F66667C317C327C337C347C3544
:100720005D20202020202020202D2074657374203F
:100730006D6F6465730A0D00776474205B6F6E7C67
:100740006F66667C746573745D20202020202020F5
:10075000202020202D207761746368646F670A0D64
:10076000007570677220202020202020202020206B
:10077000202020202020202020202020202D20721A
:1007800065626F6F742076696120626F6F746C6F41
:10079000616465720A0D00626F6F74202020202052
:1007A0002020202020202020202020202020202049
:1007B0002020202D207265626F6F740A0D00707703
:1007C0007273205B646565707C666F7263655F69D8
:1007D000646C657C6E6F6E655D202D206D63752089
:1007E000736C656570206D6F64650A0D00726573CA
:1007F0007420656570726F6D2020202020202020DD
:100800002020202020202020202D20726573746F4E
:10081000726520656570726F6D0A0D007070777279
:10082000205B6F6E7C6F66665D202020202020207C
:1008300020202020202020202D2070726F677261E0
:100840006D6D61626C65207077720A0D007478744A
:10085000205B737472696E675D2020202020202049
:100860002020202020202020202D2053657420725D
:1008700065706F7274207465787420737472696E19
:10088000670A0D0074787077205B31352D305D205C
:100890002020202020202020202020202020202058
:1008A0002D205458205077722E2048696768657350
:1008B00074203020283364426D290A0D0074746C52
:1008C000205B302D31355D2020202020202020206D
:1008D0002020202020202020202D2074696D652DCF
:1008E000746F2D6C69766520666F72207061636B22
:1008F0006574730A0D0073732020202020202020AF
:1009000020202020202020202020202020202020E7
:1009100020202D2073797374656D2073756D6D6162
:1009200072790A0D007273202020202020202020C0
:1009300020202020202020202020202020202020B7
:10094000202D20726164696F2073746174730A0DC5
:10095000007269205B696E745D20202020202020B9
:10096000202020202020202020202020202D207228
:1009700065706F727420696E74657276616C0A0DB1
:10098000007265205B6D61736B7C6175746F5D20B7
:10099000202020202020202020202020202D206DFD
:1009A0006F7465207265706F7274207365747469FA
:1009B0006E670A0D006F7720202020202020202045
:1009C0002020202020202020202020202020202027
:1009D000202D206F6E652D776972652073656E73AB
:1009E0006F72730A0D006C6F67205B6175746F7CAA
:1009F0006F6E7C6F66665D202020202020202020E6
:100A000020202D206D6F7465732064617461206FE8
:100A10006E205553420A0D006E65205B666C75733F
:100A2000685D202020202020202020202020202041
:100A3000202020202D206E65696768626F72207407
:100A400061626C650A0D00657272202020202020F2
:100A50002020202020202020202020202020202096
:100A60002020202D206572726F7220696E666F0AD9
:100A70000D006D63752020202020202020202020C4
:100A800020202020202020202020202020202D2059
:100A90006D637520696E666F0A0D006964205B7274
:100AA000657365745D2020202020202020202020D8
:100AB000202020202020202D2069642068616E6481
:100AC0006C696E670A0D0068756D2020202020205B
:100AD0002020202020202020202020202020202016
:100AE0002020202D2068756D6964697479207365F4
:100AF0006E736F720A0D0072656C6179205B6F6EA8
:100B00007C6F66667C73746174735D202020202086
:100B10002020202D2072656C6179206E6574776FBE
:100B2000726B207265706F7274730A0D00646520B9
:100B30005B6D61736B5D2020202020202020202011
:100B40002020202020202020202D20646562756731
:100B50000A0D006368616E205B31312D32365D20F5
:100B60002020202020202020202020202020202D78
:100B7000206368616E2031312D32362028322E34C8
:100B800030352D32343830204D687A290A0D006313
:100B9000616C69205B5B765F696E7C61317C613280
:100BA0005D20766F6C747C72657365747C6E6F6E9D
:100BB000655D202D2063616C6962726174650A0D48
:100BC000006164632020202020202020202020207D
:100BD000202020202020202020202020202D2073B5
:100BE000686F7720765F696E2C2061312C2061322E
:100BF00020766F6C74616765730A0D007520202084
:100C000020202020202020202020202020202020E4
:100C100020202020202020202D20757074696D65F3
:100C20000A0D0076202020202020202020202020B7
:100C30002020202020202020202020202020202DA7
:100C40002076657273696F6E0A0D0068202020207F
:100C50002020202020202020202020202020202094
:100C6000202020202020202D2068656C700A0D0097
:100C7000256300756E6B6E6F776E20636D640A007E
:100C8000484D43353838330025730025730020253F
:100C900073002025362E326620002530327800740D
:100CA000656D705F65787465726E3D252D362E32E8
:100CB0006600202573002025362E3266204F6E2DCB
:100CC000426F61726400253032780074656D705F28
:100CD000626F6172643D252D362E3266000A004532
:100CE0002025642E256420636C6F636B20256C7552
:100CF0002063707520256C75206C706D20256C75D7
:100D00002069727120256C7520676C656420256CE4
:100D10007520796C656420256C7520726C65642083
:100D2000256C7520747820256C75206C697374654A
:100D30006E20256C752073656E736F727320256C41
:100D4000752073657269616C20256C750A005320EB
:100D500025642E256420636C6F636B20256C7520E1
:100D6000747820256C7520727820256C752072743B
:100D70007820256C752072727820256C752072653C
:100D8000786D697420256C752061636B74782025FB
:100D90006C75206E6F61636B747820256C752061B3
:100DA000636B727820256C752074696D65646F754E
:100DB0007420256C752062616461636B72782025F4
:100DC0006C7520746F6F6C6F6E6720256C75207466
:100DD0006F6F73686F727420256C75206261647325
:100DE000796E636820256C7520626164637263208C
:100DF000256C7520636F6E74656E74696F6E6472B6
:100E00006F7020256C752073656E64696E676472FF
:100E10006F7020256C75206C6C747820256C7520A3
:100E20006C6C727820256C750A00257325730A0096
:100E30004F6E6C696E650A000A002C20636865635A
:100E40006B207261746520257520487A0025732017
:100E500025732C206368616E6E656C20257520708B
:100E60006F776572202575000A0025783A004D419C
:100E7000432061646472657373200052616E646F15
:100E80006D20455549363420616464726573732062
:100E900067656E6572617465640A000A2A2A2A2AE7
:100EA0002A2A2A426F6F74696E672025732A2A2ABC
:100EB0002A2A2A2A0A00020000FFFE0000014154EB
:100EC0004D45474131323872666131006C6F636164
:100ED0006C686F737400454550524F4D2069732004
:100EE000636F72727570742C2072657772697469A1
:100EF0006E6720776974682064656661756C7473C9
:100F00002E0A006E616E00696E660000407A10F372
:100F10005A00A0724E18090010A5D4E80000E87627
:100F200048170000E40B54020000CA9A3B0000007E
:100F3000E1F505000080969800000040420F000097
:100F400000A08601000000102700000000E8030058
:100F50000000006400000000000A00000000000122
:100F600000000000002C76D888DC674F0823DFC122
:100F7000DFAE59E1B1B796E5E3E453C63AE65199DD
:100F80007696E8E6C28426EB898C9B62ED407C6F06
:100F9000FCEFBC9C9F40F2BAA56FA5F490055A2ABD
:100FA000F75C936B6CF9676DC11BFCE0E40D47FEC9
:100FB000F520E6B500D0ED902E03009435770500BE
:100FC00080841E080000204E0A000000C80C333345
:100FD00033330F986E12831141EF8D2114893BE654
:100FE0005516CFFEE6DB18D1844B381BF77C1D90DD
:100FF0001DA4BBE424203284725E228100C9F12446
:10100000ECA1E53D27494E46494E4954594E414EC3
:10101000CDCCCC3D0AD7233C17B7D13877CC2B3277
:101020009595E6241FB14F0A000020410000C842F8
:1010300000401C4620BCBE4CCA1B0E5AAEC59D7457
:1010400011241FBECFEFD1E4DEBFCDBF18E0A0E07A
:10105000B2E0E4EAFEE001E00BBF02C007900D92AF
:10106000A232B107D9F71FE2A2E2B8E001C01D9297
:10107000AE37B107E1F70E947C540C9450870C9472
:10108000000029E0FC0120935700C895802D0895A9
:1010900000D08DE594E0EDB7FEB7928381830E9486
:1010A000418480910A0690910B060F900F9093FF58
:1010B00004C000D087E594E009C092FF04C000D0CE
:1010C0008BE494E003C000D085E494E0EDB7FEB774
:1010D000928381830E9441840F900F900895E09144
:1010E000A319F0E0EF71F070E850F64E8083809124
:1010F000A3198F5F8093A3198091B826886080938D
:10110000B82642E356E0CA0161E10E94D44480E07F
:1011100090E00895EF92FF92CF93DF93E82EE701DE
:101120007E01F92EE701809122089091230886FF25
:101130002DC08DB79EB70C970FB6F8949EBF0FBE0B
:101140008DBFEDB7FEB7319680E092E0ADB7BEB788
:1011500012969C938E9311978A81828313828B813E
:10116000848315828C81868317828D818087118686
:101170008E81828713860E942F842DB73EB7245F0D
:101180003F4F0FB6F8943EBF0FBE2DBF87E498E0E7
:10119000BE010E9419468BE996E0BE010E9485457A
:1011A000DF91CF91FF90EF9008954F925F926F92F1
:1011B0007F928F929F92AF92BF92CF92DF92EF92E7
:1011C000FF920F931F93DF93CF93CDB7DEB7609756
:1011D0000FB6F894DEBF0FBECDBF3B010E94A15AEF
:1011E000E82FF0E0EE0FFF1FE359F64E808191816A
:1011F000019691838083809122089091230881FD3C
:10120000749880910A0690910B064424439496FFAB
:1012100044240E949C4B7C01DC018C91982F929578
:101220009F709130B1F490E08F709070009751F4FE
:1012300080918119909182190196909382198093DF
:101240008119DFC18DEB96E2B3010E94A1420097A4
:1012500051F080917F199091801901969093801997
:1012600080937F19CEC187E498E00E94CB454FC0A0
:10127000C8010296B3010E94A142009709F444C03C
:10128000C8010F9660E074E64AE858E098010E94B1
:101290009048F7019181D80114968C911497981772
:1012A00031F51A968C911A978F5F1A968C938091CC
:1012B0007D1990917E19019690937E1980937D19E6
:1012C00084E00E94D04CF801208530E028173907CF
:1012D00028F584E00E94D04CD80118968C9318977A
:1012E000F70180818F7019968C9319978AC1D80164
:1012F0001A961C9284E00E94D04CF8018087D70196
:101300008C918F7081873BC0C8010E949146082F45
:10131000192F0115110509F0ABCF7BC144242FC053
:10132000C8010296B3010E949842F7018181815061
:10133000D80114968C9380E091E0A0E0B0E0F80131
:1013400083879487A587B687128684E00E94D04C55
:10135000D80118968C931897F70180818F70199691
:101360008C9387E498E0B8010E945246C8010F961A
:1013700060E074E64AE858E098010E949048D7017E
:1013800011968C911197F80184838C918F708783CB
:1013900084E00E94D04CD80115968C9383E00E9483
:1013A000D04C582EF8018683D70111968C90119756
:1013B0008481881A9924AA24BB24B6E0880C991C3D
:1013C000AA1CBB1CBA95D1F7638574858585968563
:1013D00020EC30E040E050E00E94337F672F782F10
:1013E000892F9927860E971EA81EB91EF80183869D
:1013F0009486A586B686809122089091230881FD67
:1014000008C080910A0680FD04C081FFFAC01D9BC0
:10141000F8C08DB79EB744970FB6F8949EBF0FBE25
:101420008DBFCDB6DEB60894C11CD11C8FE292E010
:10143000ADB7BEB712969C938E931197C7010296D3
:10144000F60193838283D3018C9184831582119654
:101450008C9186831782F7018181D60118968C932F
:10146000189719961C921997808190E08F70907050
:101470001B969C938E931A97F80185811C968C93EA
:101480001C971D961C921D971E965C921E971F9688
:101490001C92BB27AB2D9A2D892DF601918B808B49
:1014A000C501B40124E630E040E050E00E94337F03
:1014B000672F782F892F99270E94797FD60153961D
:1014C0007C936E9352970E942F842091EC05EDB788
:1014D000FEB774960FB6F894FEBF0FBEEDBF222381
:1014E000A9F000D000D0EDB7FEB7319687EE91E0BD
:1014F000ADB7BEB712969C938E9311972283138239
:101500000E9441840F900F900F900F9080910A06D7
:1015100090910B0696FF2FC0442069F1F7012081BE
:10152000822F90E08F70907082309105DCF0822FD6
:101530008F708150207F822B808383E398E00E940C
:10154000384380917B1990917C19019690937C1976
:1015500080937B19809122089091230896FF0BC0FD
:10156000739809C080918119909182190196909386
:101570008219809381198091411E86FF42C00E948A
:101580008251C70105960E9441518DB79EB70C97B5
:101590000FB6F8949EBF0FBE8DBFEDB7FEB7319664
:1015A0006E010894C11CD11CADB7BEB71296DC9277
:1015B000CE92119780E190E09383828383E792E05B
:1015C00095838483D80115968C911597868317820D
:1015D00016968C9180871186D70111968C918287FF
:1015E00013860E949884EDB7FEB73C960FB6F89428
:1015F000FEBF0FBEEDBF82E00E945E51C6010E9499
:101600004151809122089091230881FF0DC0749A66
:101610000BC08BE996E00E945F45082F192F01153A
:10162000110509F07DCEEDCF60960FB6F894DEBFC0
:101630000FBECDBFCF91DF911F910F91FF90EF9023
:10164000DF90CF90BF90AF909F908F907F906F90E2
:101650005F904F900895CF93DF93EB01009791F047
:1016600000D000D08BE89CE0EDB7FEB79283818379
:1016700086E892E0948383830E9441840F900F90C8
:101680000F900F9000D000D088E89CE0EDB7FEB737
:1016900092838183D483C3830E9441840F900F90EF
:1016A0000F900F90DF91CF91089587EE93E0811511
:1016B000910511F00197F1F708958823B9F0529838
:1016C0005A981DBA80916900806280936900EA9AF5
:1016D00053985B98EB9A80916900806880936900C9
:1016E000809168008160809368000895109269007D
:1016F0005A9AEA985B9AEB9808951F920F920FB648
:101700000F9211248F939F93AF93BF9380916800A2
:1017100080FF20C08091982690919926A0919A26CA
:10172000B0919B260196A11DB11D809398269093A0
:101730009926A0939A26B0939B2680912208909197
:10174000230887FF07C0749882E090E09093DF053C
:101750008093DE05BF91AF919F918F910F900FBE47
:101760000F901F9018951F920F920FB60F92112491
:101770008F939F93AF93BF938091680080FF20C0A9
:1017800080919C2690919D26A0919E26B0919F26A7
:101790000196A11DB11D80939C2690939D26A09338
:1017A0009E26B0939F26809122089091230890FF57
:1017B00007C0739882E090E09093DF058093DE0588
:1017C000BF91AF919F918F910F900FBE0F901F907F
:1017D000189580937C0080917B00877F80937B00AD
:1017E00080917C00806C80937C0085E080937A00FF
:1017F00080917A00806880937A0080917B0087FFD7
:10180000FCCF80917B0085FFFCCF80917A008064C3
:1018100080937A0080917A0086FDFCCF1092790047
:101820001092780084E090E060E070E020917A000F
:10183000206420937A0020917A0026FDFCCF20912D
:10184000780030917900620F731F019779F7109239
:101850007C0080917A008F7780937A0076956795E7
:101860007695679580E090E00E94B67C089580E0D0
:101870000E94E90B2091E0053091E1054091E205DD
:101880005091E3050E94947D21EE3AE744E95EE33E
:101890000E94847B089580E18093510180935101DF
:1018A0009091510195FF03C08F5F8F31B9F76BE4C1
:1018B000869FB0011124882777FD8095982F0E947C
:1018C000B87C20E030E64FE954E40E94847B20E0BD
:1018D00030E04AE754E40E944E7C0895809104066B
:1018E00085FF4BC080917B00886080937B0089ECF2
:1018F00080937C0085E080937A0080917A008068F4
:1019000080937A0080917B0087FFFCCF80917B00E1
:1019100085FFFCCF80917A00806480937A0080916B
:101920007A0086FDFCCF80917A00806480937A00F3
:1019300080917A0086FDFCCF6091780070917900EB
:1019400080E090E00E94B67C27ED33EA40E95FE357
:101950000E94947D26E636E648E853E40E94837BA5
:101960006093701970937119809372199093731921
:1019700080917A008F7780937A0008956F927F929A
:101980008F929F92AF92BF92CF92DF92EF92FF928F
:101990000F931F93DF93CF93CDB7DEB72A970FB680
:1019A000F894DEBF0FBECDBF3C0110922A088FEF26
:1019B000898344EBC42E49E1D42E00E010E032E0EC
:1019C000E32EF12CEC0EFD1E4E010894811C911C9F
:1019D0002AE0A22EB12CAC0EBD1E3FC0083011056E
:1019E00009F441C0C401B7012A870E948E4E898143
:1019F0002A858F3F11F08E3F19F480932A0834C056
:101A00006114710479F4C7010E94A84E8093B52631
:101A1000F701ADEAB6E281918D93EA15FB05D9F79E
:101A200021E022C0C7010E94A84EF6018083D701A1
:101A3000F80193E0EE0FFF1F9A95E1F7E00FF11F19
:101A4000E455F64E8D918193AA15BB05D9F70F5F2A
:101A50001F4F89E090E0C80ED91E202F898188236E
:101A600009F0BCCF01C028E0822F2A960FB6F89467
:101A7000DEBF0FBECDBFCF91DF911F910F91FF90C1
:101A8000EF90DF90CF90BF90AF909F908F907F901E
:101A90006F90089500D08DED9CE0EDB7FEB7928376
:101AA00081830E9441840F900F9008952F923F925E
:101AB0004F925F926F927F928F929F92AF92BF925E
:101AC000CF92DF92EF92FF920F931F93DF93CF930A
:101AD00000D000D0CDB7DEB78C014B01009741F4A8
:101AE00089E290E06BE270E04AE250E027E00AC051
:101AF0008130910549F489E290E06BE270E04AE2BE
:101B000050E026E00E946A4DC8010E94BE0CF80118
:101B1000E85DF74F80830115110581F0B4EBCB2E02
:101B2000B9E1DB2E00E010E03F01AAE94A2EACE06B
:101B30005A2EF2E92F2EFCE03F2E44C18DEA96E2A8
:101B40000E94DA4F9C01B901882777FD8095982F74
:101B50000E94B87CC82EE92E81149104A1F000D017
:101B600000D000D00DB71EB70F5F1F4F8BEC9CE06D
:101B7000ADB7BEB712969C938E931197562F472FF1
:101B80003C2D2E2D97C0EDEAAE2EE6E2BE2E06ECE1
:101B90001CE0D5018D915D0100D000D0EDB7FEB7FE
:101BA0003196ADB7BEB712961C930E9311978283F0
:101BB00013826B837C830E9441840F900F900F905F
:101BC0000F906B817C81B5EBAB16B6E2BB0609F7D3
:101BD00000D000D000D00DB71EB70F5F1F4F86EBAF
:101BE0009CE0EDB7FEB7928381838C2D9E2D20E083
:101BF00030E048EC52E40E944E7CD80112966D937E
:101C00007D938D939C9315970E944184EDB7FEB709
:101C100036960FB6F894FEBF0FBEEDBF8091B52685
:101C2000882319F088E892E002C081E992E000D0B0
:101C300000D022EB3CE0ADB7BEB712963C932E939A
:101C4000119714969C938E9313970E9441840F9042
:101C50000F900F900F9048C0780153E0EE0CFF1CDE
:101C60005A95E1F7E00EF11EECEAF9E1EE0EFF1EE7
:101C7000C7010E94DA4F9C01B901882777FD809542
:101C8000982F0E94B87C5C018114910481F100D0EE
:101C900000D000D00DB71EB70F5F1F4F8FE99CE03B
:101CA000ADB7BEB712969C938E931197562F472FC0
:101CB0003A2D2B2D652F742F832F922F20E030E0AB
:101CC00048EC52E40E944E7CF80162837383848363
:101CD00095830E9441842DB73EB72A5F3F4F0FB6D0
:101CE000F8943EBF0FBE2DBF0E944A0D72C020E087
:101CF00030E0D7018D917D0100D000D0EDB7FEB767
:101D00003196ADB7BEB712965C924E921197828310
:101D1000138229833A836B837C830E9441842981C7
:101D20003A812F5F3F4F0F900F900F900F906B8174
:101D30007C8128303105E9F600D000D000D0EDB626
:101D4000FEB60894E11CF11CEDB7FEB73282218289
:101D50008A2D9B2D20E030E048EC52E40E944E7C1E
:101D6000D70112966D937D938D939C9315970E9446
:101D70004184EDB7FEB736960FB6F894FEBF0FBE9E
:101D8000EDBFD6018C91882319F088E892E002C05B
:101D900081E992E000D000D02EE83CE0EDB7FEB73C
:101DA00032832183948383830E9441840F900F9018
:101DB0000F900F900E944A0D0F5F1F4F89E090E037
:101DC000C80ED91ED3018C9190E0081719070CF4A6
:101DD00043CF0F900F900F900F90CF91DF911F91F5
:101DE0000F91FF90EF90DF90CF90BF90AF909F90BA
:101DF0008F907F906F905F904F903F902F900895BD
:101E0000DF93CF9300D0CDB7DEB78091AE26898324
:101E10008091B4268A83CE0101960E94B3420F902E
:101E20000F90CF91DF910895CF93DF93EC018091D4
:101E3000AD268F3FB1F58091AE268F3F91F5809111
:101E4000AF268F3F71F58091B0268F3F51F580917D
:101E5000B1268F3F31F58091B2268F3F11F58091E9
:101E6000B3268F3FF1F48091B4268F3FD1F489E2FD
:101E700090E06BE270E04AE250E027E00E946A4D99
:101E800080E090E00E94BE0CC85DD74F88838DEA49
:101E900096E269E170E049E050E00E948A850E9484
:101EA000000FDF91CF9108951F920F920FB60F92FE
:101EB0000BB60F9211241F932F933F934F935F9371
:101EC0006F937F938F939F93AF93BF93EF93FF9302
:101ED0008091B82682608093B82680910A0686FD9C
:101EE0002B9A80910A0687FD2B9A8091DE059091AE
:101EF000DF051816190614F4749A739A8091220853
:101F00009091230885FF02C0749873988091A3066E
:101F10009091A40601979093A4068093A30600973E
:101F200009F07EC0809156089091570801969093D1
:101F300057088093560820914322309144224091C3
:101F40004522509146222F5F3F4F4F4F5F4F2093C6
:101F5000432230934422409345225093462220E16D
:101F600030E03093A4062093A30620910A0620FDBA
:101F700002C01D9B05C0109226081092250806C0BD
:101F800021E030E030932608209325086091080670
:101F9000709109066115710599F001960E94527FB2
:101FA000009771F47798809122089091230892FF0E
:101FB00007C0749884E090E09093DF058093DE057D
:101FC00060910806709109066115710579F080919C
:101FD0005608909157080E94527F009739F48EE47A
:101FE00096E062E140E050E00E94D44480910A060D
:101FF00086FD2B9880910A0690910B0691FF10C0E8
:102000000E94A15A8A3119F0182F1F5F01C01BE0EE
:102010000E94E558812F90E00E94B95A0E9483598E
:102020008DEB96E060E040E050E00E94D444FF91E8
:10203000EF91BF91AF919F918F917F916F915F9140
:102040004F913F912F911F910F900BBE0F900FBE9C
:102050000F901F9018958091A31990915722891B7A
:1020600008950E942B10882379F0E0915722F0E028
:10207000EF71F070E850F64E208130E080915722E9
:102080008F5F8093572202C02FEF3FEFC901089561
:10209000CF93DF93EC0110924A081092490888818F
:1020A0009981009731F023E08631920709F0B9C099
:1020B00009C00E942B10882341F486E193E09983A4
:1020C0008883B3C0613109F0B0C0F89478940E945D
:1020D000311090E090934E0880934D088D3009F4B4
:1020E0007CC08F3F31F38231910569F18F379105C3
:1020F00021F08830910509F053C0809151089091EA
:102100005208181619060CF060C06091782F709173
:10211000792F88E090E00E9403846091782F70917D
:10212000792F80E290E00E9403846091782F709173
:10213000792F88E090E00E9403848091510890916B
:10214000520801973EC06091782F7091792F8DE0F1
:1021500090E00E9403841092500810924F0814C01F
:10216000885A9D4DFC0180816091782F7091792F64
:1021700090E00E94038480914F089091500801964E
:102180009093500880934F0880914F089091500889
:102190002091510830915208821793070CF315C013
:1021A0006091782F7091792F0E940384809151085B
:1021B0009091520820914D08FC01E85AFD4D208372
:1021C0000196909352088093510880915108909104
:1021D00052088F33910509F06CCF109257228091ED
:1021E00057228093A3198091510890915208FC01C5
:1021F000E85AFD4D108290934A0880934908109246
:102200005208109251088091B6269091B7260097F7
:1022100009F44FCF60914B0840E050E00E94D44455
:1022200048CF1982188283E001C081E0DF91CF910D
:102230000895789480912508909126080097C9F018
:1022400080910A0690910B0693FD13C092FF03C084
:1022500083B7817F03C083B7817F866083BFF89493
:1022600083B7816083BF7894889583B78E7F83BF5F
:1022700078940895CF93DF93EC018881998100973A
:1022800021F02CE08D3A920799F40E94D3570E94D6
:10229000191180915C1090915D1065E840E050E06C
:1022A0000E94D4448DEA9CE09983888381E003C036
:1022B0001982188283E0DF91CF910895CF93DF9345
:1022C000EB01009781F000D000D08BE89CE0EDB7E7
:1022D000FEB792838183548343830E9441840F908D
:1022E0000F900F900F9000D000D088E89CE0EDB7E1
:1022F000FEB792838183D483C3830E9441840F906D
:102300000F900F900F90DF91CF910895EF92FF9271
:102310000F931F93CF93DF930E94D35780EB0E94BC
:102320005A508823A1F40E94C0508091411E909180
:10233000421E81609093421E8093411E80E090E097
:1023400062E972E00E942B0B01E010E002C000E0A5
:1023500010E0EEB0FF2484E0E822FF24729A0E948D
:10236000D3578EE40E945A50882399F40E94C0509B
:102370008091411E9091421E82609093421E8093F4
:10238000411EE8012196C8016AE972E00E942B0B08
:102390008E01E114F10409F472980E94D3578EEE75
:1023A0000E945A50882399F40E94C0508091411E87
:1023B0009091421E84609093421E8093411EE801DA
:1023C0002196C80162EA72E00E942B0B8E0186EA18
:1023D0000E945A50882399F40E94C0508091411E57
:1023E0009091421E88609093421E8093411EE801A6
:1023F0002196C80169EA72E00E942B0B8E010E94AF
:10240000D3578CE30E945A508823F1F40E94C050A5
:102410008091411E9091421E80619093421E809354
:10242000411EE8012196C80161EB72E00E942B0B6E
:1024300000D080E89CE0EDB7FEB7928381830E94D4
:1024400041840F900F908E010E94D35782ED0E941D
:102450005A50882399F40E94C0508091411E909157
:10246000421E80629093421E8093411EE801219695
:10247000C80169EB72E00E942B0B8E010E94D357BA
:1024800080ED0E945A50882399F40E94C050809198
:10249000411E9091421E80689093421E8093411E7F
:1024A000E8012196C80162EC72E00E942B0B8E01BC
:1024B000C7E0D0E00E94D3578CE70E945A5088238F
:1024C00089F40E94C0508091411E9091421E806408
:1024D0009093421E8093411EC8016AEC72E00E94F4
:1024E0002B0B02C0219731F70E94C0500E944A0D69
:1024F000DF91CF911F910F91FF90EF900895DF939F
:10250000CF9300D0CDB7DEB74A8369830E9496503F
:102510006981862F0E94C8504A81842F0E94C8502A
:102520000E94C0500F900F90CF91DF910895AF920D
:10253000BF92DF92EF92FF920F931F93DF93CF939F
:1025400000D00F92CDB7DEB7082FD22E4A835B831F
:1025500069830E9496506981862F0E94C850802FFF
:1025600081600E94BD504A815B81042F152FAA24EF
:10257000BB24ED2CFF240894E108F1080FC0AE1431
:10258000BF0419F40E94E35002C00E94D950F80120
:1025900080830894A11CB11C0F5F1F4FAD1478F30A
:1025A0000E94C0500F900F900F90CF91DF911F911C
:1025B0000F91FF90EF90DF90BF90AF900895AF9292
:1025C000BF92CF92DF92EF92FF920F931F93DF9310
:1025D000CF93CDB7DEB760970FB6F894DEBF0FBECE
:1025E000CDBFB82EA42E662309F455C0AE014F5FAF
:1025F0005F4F80E1DA011D928A95E9F780EB68E987
:1026000028E00E949712BB2059F000D083ED92E0A1
:10261000EDB7FEB7928381830E942F840F900F90B5
:102620008E010F5F1F4F38E0E32EF12CEC0EFD1EE4
:102630002AEDC22E22E0D22ED8018D918D0100D03C
:1026400000D0EDB7FEB73196ADB7BEB71296DC92AB
:10265000CE921197828313820E942F840F900F9045
:102660000F900F900E151F0539F700D000D0EDB771
:10267000FEB731968FED92E0ADB7BEB712969C9340
:102680008E9311978885828313820E942F840F90E6
:102690000F900F900F90AA2009F457C0AE014F5F22
:1026A0005F4F80E1FA0111928A95E9F780EB60E8CB
:1026B00028E00E949712BB2069F000D085EE92E0DE
:1026C000ADB7BEB712969C938E9311970E942F843C
:1026D0000F900F908E010F5F1F4F90E1E92EF12CAC
:1026E000EC0EFD1E8AEDC82E82E0D82EF8018191F5
:1026F0008F0100D000D0EDB7FEB73196ADB7BEB7B1
:102700001296DC92CE921197828313820E942F84BC
:102710000F900F900F900F900E151F0539F700D0F6
:1027200000D0EDB7FEB731968FED92E0ADB7BEB7F2
:1027300012969C938E9311978885828313820E94B0
:102740002F840F900F900F900F9060960FB6F89413
:10275000DEBF0FBECDBFCF91DF911F910F91FF90D4
:10276000EF90DF90CF90BF90AF9008950F931F939D
:10277000DF93CF9300D0CDB7DEB71A8219828EEEE9
:102780006AEA8E010F5F1F4FA80122E00E94971294
:10279000398120E08A8190E0822B932B9093191A43
:1027A0008093181A8EEE6CEAA80122E00E9497121C
:1027B000398120E08A8190E0822B932B90931B1A21
:1027C00080931A1A8EEE6EEAA80122E00E949712F8
:1027D000398120E08A8190E0822B932B90931D1AFF
:1027E00080931C1A8EEE60EBA80122E00E949712E3
:1027F000398120E08A8190E0822B932B90932B1AD1
:1028000080932A1A8EEE62EBA80122E00E949712B2
:10281000398120E08A8190E0822B932B90932D1AAE
:1028200080932C1A8EEE64EBA80122E00E9497128E
:10283000398120E08A8190E0822B932B90932F1A8C
:1028400080932E1A8EEE66EBA80122E00E9497126A
:10285000398120E08A8190E0822B932B90931F1A7C
:1028600080931E1A8EEE68EBA80122E00E94971258
:10287000398120E08A8190E0822B932B9093211A5A
:102880008093201A8EEE6AEBA80122E00E94971234
:10289000398120E08A8190E0822B932B9093251A36
:1028A0008093241A8EEE6CEBA80122E00E9497120E
:1028B000398120E08A8190E0822B932B9093271A14
:1028C0008093261A8EEE6EEBA80122E00E949712EA
:1028D000398120E08A8190E0822B932B9093291AF2
:1028E0008093281A0F900F90CF91DF911F910F9135
:1028F00008952F923F924F925F926F927F928F92A4
:102900009F92AF92BF92CF92DF92EF92FF920F937E
:102910001F93DF93CF93CDB7DEB76C970FB6F894C4
:10292000DEBF0FBECDBFA82E4A8B2B8FFE01319686
:1029300083E0DF011D928A95E9F780913C1A882394
:1029400039F46C8F0E94B61381E080933C1A6C8D31
:10295000662309F475C08EEE64EF4EE20E947F128A
:1029600069E07AE180E090E00E9447508EEE66EFE9
:10297000AE014F5F5F4F22E00E949712698170E0C5
:1029800080E090E0982F872F762F66272A8130E00D
:1029900040E050E0622B732B842B952B20912E1A54
:1029A00030912F1A40E050E0621B730B840B950BA3
:1029B00020912C1A30912D1A40E050E00E94337F74
:1029C0007B018C013FE015950795F794E7943A95C4
:1029D000D1F76091261A7091271A882777FD809584
:1029E000982F2BE0660F771F881F991F2A95D1F724
:1029F0002091281A3091291A442737FD4095542FE9
:102A00002E0D3F1D401F511F0E949B7F2E0D3F1D0D
:102A10003093231A2093221A285F3F4F14E03595F4
:102A200027951A95E1F779010027F7FC0095102FFB
:102A3000E092301AF092311A0093321A1093331A3E
:102A4000BA2DB295BB0FBB0FB07CBC5CB9872A2DE9
:102A500030E03E8B2D8B63E070E00A2C02C0660FE5
:102A6000771F0A94E2F7882777FD8095982F25E352
:102A700035E040E050E00E94337FDC01CB0102965C
:102A8000A11DB11D8A879B87AC87BD8720E533ECEC
:102A900040E050E004C05595479537952795AA9496
:102AA000D2F72E873F87488B598B18861C821D8250
:102AB0001E821F8248E050E08D899E89481B590B79
:102AC0005C8B4B8B69C18EEE64EF49850E947F124F
:102AD0006A857B858C859D850E9447508EEE66EFCA
:102AE000AE014F5F5F4F23E00E9497128091221A40
:102AF0009091231A805A9F401C01442437FC409433
:102B0000542CC201B101A20191010E94337F6F8B4D
:102B1000788F898F9A8F20911C1A30911D1A442723
:102B200037FD4095542FC201B1010E94337F7B01D4
:102B30008C01BDE015950795F794E794BA95D1F708
:102B400022E030E040E050E0E20EF31E041F151FCB
:102B50006F89788D898D9A8DACE09595879577955D
:102B60006795AA95D1F720911E1A30911F1A442714
:102B700037FD4095542F0E94337FBC01992777FD84
:102B80009095892FE60EF71E081F191FE2E0159594
:102B90000795F794E794EA95D1F780E090E8A0E0F4
:102BA000B0E0E80EF91E0A1F1B1F20912A1A30916F
:102BB0002B1A40E050E0C801B7010E94337F3B016F
:102BC0004C017FE096948794779467947A95D1F737
:102BD000A980BB24CC24DD246501BB24AA248A81DE
:102BE00090E0A0E0B0E0BA2FA92F982F8827A82A5C
:102BF000B92ACA2ADB2A8B8190E0A0E0B0E0A82A9B
:102C0000B92ACA2ADB2A0B8804C0D594C794B79482
:102C1000A7940A94D2F720911A1A30911B1A4427CC
:102C200037FD4095542FC201B1010E94337F7B01D3
:102C30008C014BE015950795F794E7944A95D1F7E9
:102C40008091181A9091191AAA2797FDA095BA2F6A
:102C500032E0880F991FAA1FBB1F3A95D1F7E80EE3
:102C6000F91E0A1F1B1F2091201A3091211A442798
:102C700037FD4095542F6F89788D898D9A8D0E94EC
:102C8000337F27E195958795779567952A95D1F7B5
:102C9000E60EF71E081F191F0D8804C0EE0CFF1C5E
:102CA000001F111F0A94D2F722E030E040E050E00C
:102CB000E20EF31E041F151F82E015950795F79489
:102CC000E7948A95D1F7AE18BF08C00AD10AC601A9
:102CD000B5012E853F85488959890E94337F97FD2C
:102CE0000BC0660F771F881F991FA40193010E94D4
:102CF000797F79018A010AC0A40193010E94797F3A
:102D000079018A01EE0CFF1C001F111F552717FDCA
:102D10005A95412F302F2F2DCA01B9010E94337FC0
:102D20002EED3BE040E050E00E94337F5B016C0100
:102D3000C801B70123E433EE4FEF5FEF0E94337F0A
:102D4000BC01992777FD9095892F6153714F8F4F63
:102D50009F4F5601DD24B7FCD094CD2C6A0D7B1D0E
:102D60008C1D9D1D44E095958795779567954A95AF
:102D7000D1F76E0D7F1D801F911F2C813D814E81EB
:102D80005F81260F371F481F591F2C833D834E83B9
:102D90005F8338853F5F388748855A89451708F42F
:102DA00092CE552391F0252F30E040E050E06C8129
:102DB0007D818E819F810E94797F2093341A309388
:102DC000351A4093361A5093371A8B8D8823C9F1E0
:102DD0006091341A7091351A8091361A9091371A91
:102DE000611571058105910561F10E94B87C20E8AB
:102DF00036EE45EC57E40E944E7C21E03EED42E485
:102E00005EE30E94F77D562F472F382F292F60E071
:102E100070E080E89FE3DA01F9012B2F3A2F4F2F62
:102E20005E2F0E94837B2BE43AE34DEB57E30E9435
:102E30004E7C6093381A7093391A80933A1A9093A3
:102E40003B1A6C960FB6F894DEBF0FBECDBFCF9184
:102E5000DF911F910F91FF90EF90DF90CF90BF9087
:102E6000AF909F908F907F906F905F904F903F902A
:102E70002F900895DF93CF9300D000D000D0CDB72E
:102E8000DEB7FE01319686E0DF011D928A95E9F7F3
:102E900080917A19882399F486EA61E340E00E94E0
:102EA0007F1286EA6CE24AE00E947F1281E0809302
:102EB0007A196CE77EE380E090E00E94475086EA52
:102EC0006DE248E00E947F126CE77EE380E090E0D4
:102ED0000E94475086EA62E3AE014F5F5F4F26E0F3
:102EE0000E94971286EA6DE247E00E947F129A8163
:102EF00080E0498150E0482B592B5093751940933D
:102F000074199C8180E02B8130E0282B392B309381
:102F10007719209376197E8160E08D8190E0862B71
:102F2000972B90937919809378196DB77EB7685075
:102F300070400FB6F8947EBF0FBE6DBFEDB7FEB701
:102F4000319669EE72E0ADB7BEB712967C936E9380
:102F500011975383428335832483978386830E940A
:102F60002F846DB77EB7685F7F4F0FB6F8947EBF32
:102F70000FBE6DBF26960FB6F894DEBF0FBECDBF55
:102F8000CF91DF9108958F929F92AF92BF92CF928F
:102F9000DF92EF92FF920F931F93DF93CF9300D0B6
:102FA00000D000D0CDB7DEB78E010F5F1F4F86E097
:102FB000F80111928A95E9F78CE362E041E00E9402
:102FC0007F128CE360E048E50E947F1262E174E3C7
:102FD00080E090E00E9447508CE363E0A80126E087
:102FE0000E9497128CE362E043E00E947F12998175
:102FF00080E00A8110E0082B192B109351190093DF
:1030000050199B8180E0EC80FF24E82AF92AF09295
:103010005319E09252199D8180E0CE80DD24C82AA8
:10302000D92AD0925519C0925419B701882777FD33
:103030008095982F0E94B87C4B015C01B8018827CD
:1030400077FD8095982F0E94B87C9B01AC01C5014B
:10305000B4010E94F77B2DB73EB72C5030400FB61D
:10306000F8943EBF0FBE2DBFADB6BEB60894A11CEE
:10307000B11C27EF32E0EDB7FEB732832183F501B3
:1030800013830283F582E482D782C68220EE3EE279
:1030900045E652E40E94947D20E030E044E353E4AE
:1030A0000E94847BF50160877187828793870E94E5
:1030B0002F842DB73EB7245F3F4F0FB6F8943EBF25
:1030C0000FBE2DBF26960FB6F894DEBF0FBECDBF44
:1030D000CF91DF911F910F91FF90EF90DF90CF90F4
:1030E000BF90AF909F908F900895CF93DF93EC01A6
:1030F00088819981009731F02CE08639920709F098
:1031000071C00BC08BE298E060E870E00E948A47D3
:1031100086E99CE09983888369C08BE298E00E94ED
:10312000B547009709F462C0809122089091230866
:1031300093FF3FC08091411E82FF3BC083E061E06E
:1031400048E021E00E9479148DB79EB70A970FB628
:10315000F8949EBF0FBE8DBFEDB7FEB731968FECD2
:1031600091E0ADB7BEB712969C938E931197809164
:10317000341A9091351AA091361AB091371A828379
:103180009383A483B5838091381A9091391AA091C2
:103190003A1AB0913B1A86839783A087B1870E9421
:1031A00041848DB79EB70A960FB6F8949EBF0FBEA6
:1031B0008DBF809122089091230894FF06C08091D2
:1031C000411E83FF02C00E943A178091220890910D
:1031D000230895FF97CF8091411E84FF93CF0E94D3
:1031E000C31790CF1982188283E001C081E0DF917C
:1031F000CF910895EF92FF920F931F93CF93DF9398
:10320000729A80910A0683FD06C0C0E5D0E00E9454
:10321000550B2197E1F78EE40E945A508823B1F0B4
:103220008091472290914822A0914922B0914A2250
:103230000196A11DB11D8093472290934822A0932F
:103240004922B0934A2221E030E087C0C0E5D0E0B7
:103250000E94550B2197E1F78FE40E945A500E947B
:10326000D950982F92959695969593709130A9F490
:1032700020914B2230914C2240914D2250914E2270
:103280002F5F3F4F4F4F5F4F20934B2230934C2285
:1032900040934D2250934E2216C09230A0F02091C0
:1032A0004F223091502240915122509152222F5F53
:1032B0003F4F4F4F5F4F20934F2230935022409308
:1032C0005122509352226FE3E62EE8220E94D950F9
:1032D000F82E0E94D950082F0E94E350182F0E9408
:1032E000C05080910A0683FF72987E2D60E06F0DBA
:1032F000711D80E090E00E94B67C20E134E048EC53
:103300005BE30E94947D60933D1A70933E1A809314
:103310003F1A9093401A702F60E0610F711D7695EF
:1033200067957695679580E090E00E94B67C24EAE8
:103330003CEF44E25CE30E94947D20E030E040E218
:1033400052E40E94837B6093B9267093BA268093DF
:10335000BB269093BC2620E030E0C901DF91CF91DD
:103360001F910F91FF90EF9008957298729A8EE4DA
:103370000E945A5080EA0E94C85080E00E94C850C3
:1033800080E00E94C8508FE40E945A500E94D95099
:1033900082958695869583708130A9F420914B2281
:1033A00030914C2240914D2250914E222F5F3F4F41
:1033B0004F4F5F4F20934B2230934C2240934D222E
:1033C00050934E2216C08230A0F020914F223091AF
:1033D000502240915122509152222F5F3F4F4F4F28
:1033E0005F4F20934F2230935022409351225093AD
:1033F000522200D000D0EDB7FEB731962CE033E07A
:10340000ADB7BEB712963C932E9311978283138269
:103410000E942F840F900F900F900F908EE40E94C7
:103420005A5080E80E94C85080E00E94C85080E056
:103430000E94C8500E94C05080E090E0089500D0E3
:1034400083E79CE0ADB7BEB712969C938E9311971D
:103450000E9441842091EC050F900F902223A9F047
:1034600000D000D0EDB7FEB7319680E79CE0ADB755
:10347000BEB712969C938E931197228313820E945B
:1034800041840F900F900F900F90089500D08BE41F
:103490009CE0EDB7FEB7928381830E94418483E272
:1034A0009CE0EDB7FEB7928381830E9441848CEF4C
:1034B0009BE0EDB7FEB7928381830E94418481EC4B
:1034C0009BE0EDB7FEB7928381830E9441848FE831
:1034D0009BE0EDB7FEB7928381830E94418483E530
:1034E0009BE0EDB7FEB7928381830E9441848DE219
:1034F0009BE0EDB7FEB7928381830E94418487EF02
:103500009AE0EDB7FEB7928381830E94418487ECF5
:103510009AE0EDB7FEB7928381830E9441848BE9E4
:103520009AE0EDB7FEB7928381830E94418482E7DF
:103530009AE0EDB7FEB7928381830E94418487E4CD
:103540009AE0EDB7FEB7928381830E94418488E1BF
:103550009AE0EDB7FEB7928381830E94418486EEA4
:1035600099E0EDB7FEB7928381830E94418485EB99
:1035700099E0EDB7FEB7928381830E94418481E890
:1035800099E0EDB7FEB7928381830E94418481E583
:1035900099E0EDB7FEB7928381830E94418485E272
:1035A00099E0EDB7FEB7928381830E94418486EF54
:1035B00098E0EDB7FEB7928381830E9441848DEB42
:1035C00098E0EDB7FEB7928381830E94418484E83E
:1035D00098E0EDB7FEB7928381830E9441848DE429
:1035E00098E0EDB7FEB7928381830E9441848CE11D
:1035F00098E0EDB7FEB7928381830E9441848DEEFF
:1036000097E0EDB7FEB7928381830E9441848EEBF1
:1036100097E0EDB7FEB7928381830E94418487E9EA
:1036200097E0EDB7FEB7928381830E94418481E6E3
:1036300097E0EDB7FEB7928381830E94418488E3CF
:1036400097E0EDB7FEB7928381830E9441848DE0BD
:1036500097E0EDB7FEB7928381830E9441840F907B
:103660000F9008958CE193E00E94618408952F9259
:103670003F924F925F926F927F928F929F92AF9202
:10368000BF92CF92DF92EF92FF920F931F93CF934F
:10369000DF93609143227091442280914522909162
:1036A0004622A0904322B0904422C0904522D09060
:1036B0004622609043227090442280904522909050
:1036C0004622209043223090442240904522509040
:1036D00046222DB73EB72A5030400FB6F8943EBF71
:1036E0000FBE2DBFCDB7DEB7219627EE36E0EDB782
:1036F000FEB732832183A0E8EA2EA1E5FA2EA1E0ED
:103700000A2F112DA80197010E94797F3B832A83FC
:10371000C601B501A80197010E94797FF0E1EF2E63
:10372000FEE0FF2E012D112DA80197010E94797F47
:10373000332727FD30953D832C83C401B301A801B5
:1037400097010E94797FECE3EE2EF12C012D112DD3
:10375000A80197010E94797F332727FD30953F8389
:103760002E83C201B101A80197010E94797F7727BA
:1037700067FD7095798768870E9441842DB73EB7B1
:10378000265F3F4F0FB6F8943EBF0FBE2DBFDF91AF
:10379000CF911F910F91FF90EF90DF90CF90BF904E
:1037A000AF909F908F907F906F905F904F903F90E1
:1037B0002F900895EEE7FFE28081918122E4823428
:1037C0009207B9F000D000D089EC96E0ADB7BEB753
:1037D00012969C938E931197EE57FF421496FC938A
:1037E000EE9313970E9441840F900F900F900F90CB
:1037F00008953A96B1E4E53FFB07F0F208950F9380
:103800001F93CF93DF93EC018C9A0E94370C00D06A
:1038100000D000D02DEB36E0EDB7FEB73283218328
:1038200063837483858396830E9441848DB79EB79A
:1038300006960FB6F8949EBF0FBE8DBF209719F065
:103840000E944A0D0BC000D08BEB96E0EDB7FEB79F
:10385000928381830E9441840F900F9081E00E94A7
:10386000E90B00D000D000D00DB71EB70F5F1F4F7F
:103870002FEA36E0EDB7FEB7328321832091E405CD
:103880003091E5054091E6055091E7050E94947D51
:10389000F80162837383848395830E9441848DB78A
:1038A0009EB706960FB6F8949EBF0FBE8DBF2097A9
:1038B00019F00E944A0D0BC000D08DEA96E0EDB7DA
:1038C000FEB7928381830E9441840F900F9082E023
:1038D0000E94E90B00D000D000D00DB71EB70F5FDB
:1038E0001F4F21EA36E0EDB7FEB7328321832091E6
:1038F000E8053091E9054091EA055091EB050E94F9
:10390000947DF80162837383848395830E9441844C
:103910008DB79EB706960FB6F8949EBF0FBE8DBFAB
:10392000209719F00E944A0D0BC000D08FE996E055
:10393000EDB7FEB7928381830E9441840F900F9070
:1039400083E00E94E90B00D000D000D020E936E0EF
:10395000EDB7FEB7328321836383748385839683B7
:103960000E9441848C988DB79EB706960FB6F89446
:103970009EBF0FBE8DBF209719F00E944A0D0BC04D
:1039800000D08EE896E0EDB7FEB7928381830E9467
:1039900041840F900F908091411E87FFA4C080ED5D
:1039A00061E042E121E00E94305200D000D000D01E
:1039B00021E836E0EDB7FEB7328321836383748359
:1039C000858396830E9441848DB79EB706960FB675
:1039D000F8949EBF0FBE8DBF209719F00E944A0D2C
:1039E0000BC000D08FE796E0EDB7FEB792838183DE
:1039F0000E9441840F900F9080ED62E042E121E04F
:103A00000E94305200D000D000D022E736E0EDB75F
:103A1000FEB73283218363837483858396830E94F8
:103A200041848DB79EB706960FB6F8949EBF0FBE21
:103A30008DBF209719F00E944A0D0BC000D080E77F
:103A400096E0EDB7FEB7928381830E9441840F9088
:103A50000F9080ED63E042E121E00E94305200D0FF
:103A600000D000D023E636E0EDB7FEB732832183E5
:103A700063837483858396830E9441848DB79EB748
:103A800006960FB6F8949EBF0FBE8DBF209719F013
:103A90000E944A0D0BC000D081E696E0EDB7FEB75C
:103AA000928381830E9441840F900F9080ED64E0A7
:103AB00042E121E00E94305200D000D000D024E545
:103AC00036E0EDB7FEB73283218363837483858349
:103AD00096830E9441848DB79EB706960FB6F894E0
:103AE0009EBF0FBE8DBF209711F40E944A0DDF913B
:103AF000CF911F910F9108950F931F93CF93DF9351
:103B0000882389F08DEA96E26FEF70E049E050E09B
:103B10000E94AA838DEA96E269E170E049E050E0F4
:103B20000E948A851CC0CDEAD6E20FE416E0899196
:103B300000D000D0EDB7FEB73196ADB7BEB7129644
:103B40001C930E931197828313820E9441840F90DD
:103B50000F900F900F90B6E2C53BDB0741F70E9434
:103B60004A0DDF91CF911F910F910895EF92FF922F
:103B70000F931F936091F2057091F30580E090E040
:103B80000E949C8367E373E00E94B183009709F071
:103B9000B6C08DE490E2A1E0B0E08093040690937B
:103BA0000506A0930606B093070684E096E06EE053
:103BB00070E044E050E00E948A858CE390E09093AE
:103BC00009068093080688E096E062E170E042E032
:103BD00050E00E948A858AE090E490930B068093DF
:103BE0000A068AE096E064E170E042E050E00E945C
:103BF0008A85109223081092220882E298E060E001
:103C000070E042E050E00E948A850F2EF2E2EF2E33
:103C1000FFEFFF2EFCEC0F2FFBE31F2FF02DE092A8
:103C2000E405F092E5050093E6051093E70584EEC0
:103C300095E066E070E044E050E00E948A85E09202
:103C4000E805F092E9050093EA051093EB0588EE8C
:103C500095E06AE070E044E050E00E948A8587EDDC
:103C600094E3AFEEBCE38093E0059093E105A0936D
:103C7000E205B093E30580EE95E062E070E044E099
:103C800050E00E948A851092270880E090E00E9410
:103C90002C5C87E298E066E170E041E050E00E9431
:103CA0008A858AE180930C068AE190E00E94A45AFA
:103CB0008CE096E067E170E041E050E00E948A8588
:103CC0008FE080930D068DE096E068E170E041E0C2
:103CD00050E00E948A8586E699E12AE0FC01119273
:103CE0002A95E9F762E270E04AE050E00E948A8596
:103CF00081E00E947C1D80E090E00E94140F1F91E3
:103D00000F91FF90EF900895EF92FF920F931F9302
:103D1000CF93DF937B018C01CB0181709070009772
:103D200049F080E090E06EE373E00E942B0B81E0AD
:103D300090E002C080E090E0E1FE07C0EC01219637
:103D400063E473E00E942B0BCE01E2FE07C0EC019E
:103D500021966BE473E00E942B0BCE01E3FE07C0BB
:103D6000EC01219663E573E00E942B0BCE01E4FE8B
:103D700007C0EC01219667E573E00E942B0BCE0192
:103D8000E5FE07C0EC0121966AE573E00E942B0B6B
:103D9000CE01E6FE07C0EC0121966EE573E00E94BD
:103DA0002B0BCE01E7FE07C0EC01219664E673E021
:103DB0000E942B0BCE01F0FE07C0EC0121966CE6B1
:103DC00073E00E942B0BCE01F1FE07C0EC0121969F
:103DD00064E773E00E942B0BCE01F2FE07C0EC01FA
:103DE000219668E773E00E942B0BCE01F3FE07C01B
:103DF000EC0121966EE773E00E942B0BCE01F4FEDE
:103E000007C0EC01219663E873E00E942B0BCE0102
:103E1000F5FE07C0EC01219669E873E00E942B0BC8
:103E2000CE01F6FE05C061E973E00E942B0B10C0C5
:103E3000E114F1040105110559F400D08AE496E07B
:103E4000EDB7FEB7928381830E9441840F900F905B
:103E5000DF91CF911F910F91FF90EF900895EF9216
:103E6000FF920F931F93CF93DF938C01C0E0D0E0BC
:103E700081C0C80165E476E00E948883009709F458
:103E8000C160C8016DE376E00E948883009709F461
:103E9000C260C80165E376E00E948883009709F458
:103EA000C460C80161E376E00E948883009709F44A
:103EB000C860C8016EE276E00E948883009709F42A
:103EC000C061C8016AE276E00E948883009709F425
:103ED000C062C80164E276E00E948883009709F41A
:103EE000C064C8016CE176E00E948883009709F401
:103EF000C068C80164E176E00E948883009709F4F5
:103F0000D160C80160E176E00E948883009709F4DF
:103F1000D260C8016AE076E00E948883009709F4C5
:103F2000D460C80165E076E00E948883009709F4B8
:103F3000D860C8016FEF75E00E948883009709F48C
:103F4000D061C80167EF75E00E948883009709F48B
:103F5000D062C8016CEE75E00E948883009709F476
:103F6000D0646091F2057091F30580E090E00E94CA
:103F70009C838C010115110509F07BCFCE01DF91E7
:103F8000CF911F910F91FF90EF900895EF92FF92C4
:103F90000F931F93CF93DF937B018C01CB01817033
:103FA0009070009749F080E090E06CE973E00E9427
:103FB0002B0B81E090E002C080E090E0E2FE07C0C1
:103FC000EC01219660EA73E00E942B0BCE01E1FE2A
:103FD00007C0EC01219664EA73E00E942B0BCE012E
:103FE000E3FE07C0EC01219667EA73E00E942B0B09
:103FF000CE01E4FE07C0EC01219669EA73E00E945D
:104000002B0BCE01E5FE07C0EC0121966CEA73E0B4
:104010000E942B0BCE01E6FE07C0EC01219662EB5D
:1040200073E00E942B0BCE01E7FE07C0EC01219646
:1040300068EB73E00E942B0BCE01F0FE07C0EC0191
:1040400021966BEB73E00E942B0BCE01F1FE07C0B3
:10405000EC01219660EC73E00E942B0BCE01F2FE86
:1040600007C0EC01219663EC73E00E942B0BCE019C
:10407000F3FE07C0EC01219668EC73E00E942B0B65
:10408000CE01F4FE07C0EC0121966FEC73E00E94B4
:104090002B0BCE01F5FE07C0EC01219662ED73E01B
:1040A0000E942B0BCE01F6FE07C0EC01219667EDB6
:1040B00073E00E942B0BCE01F7FE07C0EC012196A6
:1040C0006AED73E00E942B0BCE0100FF07C0EC01EC
:1040D00021966DED73E00E942B0BCE0101FF07C00E
:1040E000EC01219660EE73E00E942B0BCE0102FFE3
:1040F00007C0EC01219664EE73E00E942B0BCE0109
:1041000003FF07C0EC01219668EE73E00E942B0BC1
:10411000CE0104FF07C0EC0121966CEE73E00E9413
:104120002B0BCE0105FF07C0EC01219660EF73E079
:104130000E942B0BCE0106FF05C062EF73E00E94C8
:104140002B0B10C0E114F1040105110559F400D046
:1041500087EE95E0EDB7FEB7928381830E9441849C
:104160000F900F90DF91CF911F910F91FF90EF90E3
:104170000895EF92FF920F931F93CF93DF93EC017B
:1041800062EE75E00E948883009721F0EE24FF2400
:10419000870180C18091411E82FF08C09DE4E92E05
:1041A00090E2F92E91E2092F112D07C0BDE4EB2E0C
:1041B000B0E2FB2EB1E00B2F112D81FF6EC180E02C
:1041C00090E1A0E0B0E0E82AF92A0A2B1B2B65C198
:1041D000CE016EED75E00E948883009741F481E086
:1041E00090E0A0E0B0E0E82AF92A0A2B1B2BCE01D0
:1041F0006AED75E00E948883009741F484E090E0C6
:10420000A0E0B0E0E82AF92A0A2B1B2BCE0167EDCB
:1042100075E00E948883009741F482E090E0A0E07E
:10422000B0E0E82AF92A0A2B1B2BCE0165ED75E0D8
:104230000E948883009741F488E090E0A0E0B0E01D
:10424000E82AF92A0A2B1B2BCE0162ED75E00E94A9
:104250008883009741F480E190E0A0E0B0E0E82A94
:10426000F92A0A2B1B2BCE016CEC75E00E94888387
:10427000009741F480E290E0A0E0B0E0E82AF92A5B
:104280000A2B1B2BCE0166EC75E00E9488830097F9
:1042900041F480E490E0A0E0B0E0E82AF92A0A2B9B
:1042A0001B2BCE0163EC75E00E948883009741F4DC
:1042B00080E890E0A0E0B0E0E82AF92A0A2B1B2B66
:1042C000CE016EEB75E00E948883009741F480E098
:1042D00091E0A0E0B0E0E82AF92A0A2B1B2BCE01DE
:1042E0006BEB75E00E948883009741F480E890E0D2
:1042F000A0E0B0E0E82AF92A0A2B1B2BCE0166EBDE
:1043000075E00E948883009741F480E091E0A0E08E
:10431000B0E0E82AF92A0A2B1B2BCE016FEA75E0E0
:104320000E948883009741F480E098E0A0E0B0E02C
:10433000E82AF92A0A2B1B2BCE016CEA75E00E94B1
:104340008883009741F480E090E1A0E0B0E0E82AA3
:10435000F92A0A2B1B2BCE0167EA75E00E9488839D
:10436000009741F480E090E2A0E0B0E0E82AF92A6A
:104370000A2B1B2BCE0164EA75E00E94888300970C
:1043800041F480E090E4A0E0B0E0E82AF92A0A2BAA
:104390001B2BCE0161EA75E00E948883009741F4EF
:1043A00080E090E8A0E0B0E0E82AF92A0A2B1B2B75
:1043B000CE016EE975E00E948883009741F480E0A9
:1043C00090E0A1E0B0E0E82AF92A0A2B1B2BCE01ED
:1043D0006AE975E00E948883009741F480E090E0EC
:1043E000A2E0B0E0E82AF92A0A2B1B2BCE0166E9ED
:1043F00075E00E948883009741F480E090E0A4E09B
:10440000B0E0E82AF92A0A2B1B2BCE0162E975E0FD
:104410000E948883009741F480E090E0A8E0B0E03B
:10442000E82AF92A0A2B1B2BCE016EE875E00E94C0
:104430008883009741F480E090E0A0E1B0E0E82AB2
:10444000F92A0A2B1B2BCE016CE875E00E948883A9
:10445000009741F480E090E0A0E2B0E0E82AF92A79
:104460000A2B1B2BCE0169E875E00E948883009718
:1044700041F480E090E0A0E4B0E0E82AF92A0A2BB9
:104480001B2B6091F2057091F30580E090E00E9493
:104490009C83EC01209709F09BCEB701C801DF9106
:1044A000CF911F910F91FF90EF90089500D089E771
:1044B00095E0ADB7BEB712969C938E9311970E946C
:1044C00041840F900F900E94321B00D000D081E7F2
:1044D00095E0EDB7FEB79283818386E699E19483F8
:1044E00083830E9441840F900F908DE695E0ADB7D5
:1044F000BEB712969C938E9311970E9441840F90A1
:104500000F9080E00E947C1D00D088E695E0EDB71A
:10451000FEB7928381830E9441840F900F900E9486
:1045200086118091411E80FF05C081E061E041E07D
:104530000E94DF120E94371B00D000D0EDB7FEB7FB
:1045400031968FE595E0ADB7BEB712969C938E93EA
:10455000119780910C06828313820E944184EDB7EB
:10456000FEB7319686E595E0ADB7BEB712969C933F
:104570008E93119780912708828313820E94418431
:104580008EE395E0EDB7FEB79283818380E490E0FF
:10459000948383830E94418400D0EDB7FEB73196A7
:1045A0008BE295E0ADB7BEB712969C938E931197B0
:1045B0008091BD26828313828091BE2684831582DA
:1045C0000E9441840F900F90EDB7FEB7319682E2C2
:1045D00095E0ADB7BEB712969C938E9311978091DC
:1045E0000D06828313820E94418480910A06909175
:1045F0000B060F900F900F900F9096FF03C085EF62
:1046000093E002C088EF93E000D000D028E135E0CD
:10461000EDB7FEB732832183948383830E94418464
:1046200083E095E0ADB7BEB712969C938E93119739
:10463000809108069091090614969C938E93139787
:104640000E9441840F900F9086EF94E0EDB7FEB783
:10465000928381830E9441840F900F9060910406A1
:104660007091050680910606909107060E94C61F6C
:104670000E944A0D1D9B03C085EF93E002C088EFA6
:1046800093E000D000D02AEE34E0ADB7BEB712966A
:104690003C932E93119714969C938E9313970E949C
:1046A00041840F900F9080EE94E0EDB7FEB79283B7
:1046B00081830E94418480910A060F900F9081FFB0
:1046C0000EC000D08AED94E0ADB7BEB712969C93B1
:1046D0008E9311970E9441840F900F9017C080FF16
:1046E00003C085EF93E002C088EF93E000D000D0D4
:1046F00026ED34E0EDB7FEB73283218394838383C4
:104700000E9441840F900F900F900F9000D08FEC7B
:1047100094E0ADB7BEB712969C938E9311970E940A
:10472000418460912208709123080F900F9080E0DF
:1047300090E00E94841E0E944A0D779903C085EF85
:1047400093E002C088EF93E000D000D026EC34E084
:10475000EDB7FEB732832183948383830E94418423
:104760000F900F900F900F900E9448080E946E0CBF
:104770000E944B0C00D000D000D028EB34E0ADB745
:10478000BEB712963C932E931197EDB7FEB7638395
:104790007483858396830E9441848DB79EB7069665
:1047A0000FB6F8949EBF0FBE8DBF81E090E00E94CF
:1047B000FF1B8091982690919926A0919A26B091FE
:1047C0009B2600D000D000D02AEA34E0EDB7FEB737
:1047D0003283218383839483A583B6830E9441849B
:1047E00086E994E0ADB7BEB712969C938E9311976D
:1047F0008091A5269091A626A091A726B091A826E3
:10480000EDB7FEB783839483A583B6830E9441846A
:1048100080919C2690919D26A0919E26B0919F26E6
:1048200028E834E0EDB7FEB7328321838383948395
:10483000A583B6830E94418484E794E0ADB7BEB7F8
:1048400012969C938E9311978091A9269091AA26F7
:10485000A091AB26B091AC26EDB7FEB783839483CD
:10486000A583B6830E9441848DB79EB706960FB686
:10487000F8949EBF0FBE8DBF80E090E061E070E0D5
:104880000E94560D81E090E061E070E00E94560DBC
:1048900008952F923F924F925F926F927F928F92E4
:1048A0009F92AF92BF92CF92DF92EF92FF920F93BF
:1048B0001F93DF93CF9300D0CDB7DEB79A83898360
:1048C000DC018D919C911197009711F00C942F367B
:1048D0006091F2057091F30588E592E20E949C8355
:1048E00088E592E260E470E00E94C983009759F481
:1048F0006091782F7091792F8AE090E00E94038474
:1049000081E00C9435368130910549F4209058228D
:10491000332444245524662477244301BFC18230C4
:10492000910599F43091582220915922932F80E0DB
:10493000820F911D1C01892F880F880B482E582E3D
:10494000682E782E882E982EA9C18330910509F003
:104950009CC020915822A090592280905A2230E089
:1049600040E050E060E070E080E090E000E10E9414
:104970002077F22E132FE42ED52EC62EB72E282EFA
:10498000992E2A2D30E040E050E060E070E080E0B9
:1049900090E008E00E9420772F0DB1E02F1508F07D
:1049A000B0E0310FE1E0311708F0E0E0B30FF1E0E3
:1049B000B31708F0F0E0EF2B4E0D31E04E1508F084
:1049C00030E0E40FF1E0E41708F0F0E03F2B5D0D7C
:1049D00041E05D1508F040E0A32FA50F31E0A517D9
:1049E00008F030E0432B6C0D31E06C1508F030E03E
:1049F000F42FF60F41E0F61708F040E0342B7B0D62
:104A000041E07B1508F040E0532F570F31E0571776
:104A100008F030E0432B820D31E0821508F030E0E1
:104A2000480F61E0481708F060E0362B990D930FAE
:104A3000022F080D11E0021708F010E01B0F81E0B3
:104A40001B1708F080E0B82FBE0F71E0BE1708F00A
:104A500070E07A0F61E07A1708F060E06F0F31E0E4
:104A60006F1708F030E0350F21E0351708F020E02F
:104A7000240F81E0241708F080E018014B2E572EF8
:104A8000662E732E822E982EFEC0843091050CF473
:104A9000FCC020915822A090592270905A228090F8
:104AA0005B2230E040E050E060E070E080E090E0C9
:104AB00008E10E942077F22E132FE42ED52EC62E69
:104AC000B72E282E992E2A2D30E040E050E060E0ED
:104AD00070E080E090E000E10E9420772F0DF1E08F
:104AE0002F1508F0F0E0310FE1E0311708F0E0E0B9
:104AF000F30FA1E0F31708F0A0E0EA2B4E0D31E030
:104B00004E1508F030E0E40FA1E0E41708F0A0E053
:104B10003A2B5D0D41E05D1508F040E0B32FB50F75
:104B200031E0B51708F030E0432B6C0D31E06C1527
:104B300008F030E0A42FA60F41E0A61708F040E0EF
:104B4000342B7B0D41E07B1508F040E0532F570FCD
:104B500031E0571708F030E0432B820D31E0821529
:104B600008F030E0480F61E0481708F060E0362BAD
:104B7000990E930E122F180D81E0121708F080E0A5
:104B8000282E2F0E81E02F1608F080E0F82EFE0E62
:104B900081E0FE1608F080E0E82EEB0E81E0EB16D7
:104BA00008F080E0D82EDA0E81E0DA1608F080E016
:104BB000C82EC50E81E0C51608F080E0B82EB40EF0
:104BC00081E0B41608F080E0980E272D30E040E038
:104BD00050E060E070E080E090E008E00E94207724
:104BE000210FE1E0211708F0E0E0320DF1E032158D
:104BF00008F0F0E0E30FA1E0E31708F0A0E0FA2BE3
:104C00004F0D31E04F1508F030E0F40FA1E0F4173C
:104C100008F0A0E03A2B5E0D41E05E1508F040E0A0
:104C2000A32FA50F31E0A51708F030E0432B6D0D41
:104C300031E06D1508F030E0542F560F41E0561763
:104C400008F040E0342B7C0D41E07C1508F040E09A
:104C5000632F670F31E0671708F030E0432B8B0DAF
:104C600031E08B1508F030E0480F71E0481708F08C
:104C700070E0372B990D222E3E2E4F2E5A2E652E88
:104C8000762E842E932E990E09C0BAE02B2E332453
:104C90004424552466247724882499240E944A0DAC
:104CA000B22DB73691F4E32DEF3679F4F42DFC36BE
:104CB00061F4552051F4662041F4772031F48820C6
:104CC00021F4992011F40C945C319101A201B301FB
:104CD000C401A7E6AA2EFFE6BF2EECE6CE2EDD2409
:104CE000EE24FF2400E010E00E949177823008F06B
:104CF000A4C2822D893689F4932D923771F4442011
:104D000061F4552051F4662041F4772031F4882075
:104D100021F4992011F40C94F5339101A201B3010F
:104D2000C40109E6A02E12E7B12ECC24DD24EE2426
:104D3000FF2400E010E00E949177823008F023C148
:104D4000A22DA53681F4B32DB43669F4442059F46C
:104D5000552049F4662039F4772029F4882019F485
:104D6000992009F437C79101A201B301C401B5E646
:104D7000AB2EA4E6BA2ECC24DD24EE24FF2400E0E2
:104D800010E00E949177823008F07DC0E22DE53777
:104D900081F4332071F4442061F4552051F46620ED
:104DA00041F4772031F4882021F4992011F40C94F7
:104DB0001B2F9101A201B301C401F5E7AF2EBB2463
:104DC000CC24DD24EE24FF2400E010E00E94917743
:104DD000823010F5F22DF83611F00C942D36332078
:104DE00011F00C942D36442011F00C942D365520E2
:104DF00011F00C942D36662011F00C942D3677208E
:104E000011F00C942D36882011F00C942D36992039
:104E100011F00C942D3633C7822D863781F4332060
:104E200071F4442061F4552051F4662041F4772058
:104E300031F4882021F4992011F40C942A2F922D1A
:104E4000943611F00C942D36A32DA13611F00C944C
:104E50002D36442011F00C942D36552011F00C9471
:104E60002D36662011F00C942D36772011F00C941D
:104E70002D36882011F00C942D36992011F00C94C9
:104E80002D360C946634B22DB73789F4E32DEF3606
:104E900071F4442061F4552051F4662041F47720E8
:104EA00031F4882021F4992011F40C949632910168
:104EB000A201B301C401E7E7AE2E0FE6B02ECC2469
:104EC000DD24EE24FF2400E010E00E949177823080
:104ED000B8F5F22DF43681F4832D893669F4442037
:104EE00059F4552049F4662039F4772029F48820B4
:104EF00019F4992009F47FC7922D953611F00C947E
:104F00002D36A32DAE3611F00C942D36442011F021
:104F10000C942D36552011F00C942D36662011F08E
:104F20000C942D36772011F00C942D36882011F03A
:104F30000C942D36992011F00C942D360C94C0321F
:104F4000B22DB33389F4E32DE13771F4442061F4D9
:104F5000552051F4662041F4772031F4882021F463
:104F6000992011F40C946634F22DF53611F00C945E
:104F70002D36832D823711F00C942D36442011F0FC
:104F80000C942D361EC2922D923689F4A32DA5368F
:104F900071F4B42DB43659F4552049F4662039F42F
:104FA000772029F4882019F4992009F413C6910177
:104FB000A201B301C40112E6A12EB5E6BB2EA4E600
:104FC000CA2EDD24EE24FF2400E010E00E94917739
:104FD000823008F098C0E22DE13389F4F32DF436E5
:104FE00071F4842D813659F4552049F4662039F442
:104FF000772029F4882019F4992009F4FFC391013E
:10500000A201B301C401F1E3AF2EE4E6BE2E01E636
:10501000C02EDD24EE24FF2400E010E00E949177F2
:105020008230C0F5922D933789F4A32DA23771F405
:10503000442061F4552051F4662041F4772031F486
:10504000882021F4992011F40C944834B22DB33700
:1050500011F00C942D36E32DE33711F00C942D361E
:10506000442011F00C942D36552011F00C942D365F
:10507000662011F00C942D36772011F00C942D360B
:10508000882011F00C942D36992011F00C942D36B7
:105090000C945734F22DF33691F4832D843679F441
:1050A000942D913661F4552051F4662041F4772017
:1050B00031F4882021F4992011F40C946634A22D47
:1050C000A83711F00C942D36B32DB43611F00C9492
:1050D0002D36E42DE13611F00C942D36552011F0CB
:1050E0000C942D36662011F00C942D36772011F09B
:1050F0000C942D36882011F00C942D36992011F047
:105100000C942D3677C3F22DFD3691F4832D85371F
:1051100079F4942D983661F4552051F4662041F4C9
:10512000772031F4882021F4992011F40C947734FD
:105130009101A201B301C4011DE6A12EB5E7BB2E6A
:10514000A8E6CA2EDD24EE24FF2400E010E00E9431
:1051500091778230C8F5A22DA23791F4B32DB237E2
:1051600079F4E42DE53661F4552051F4662041F4DC
:10517000772031F4882021F4992011F40C94B9316E
:10518000F22DF33611F00C942D36832D8D3611F05F
:105190000C942D36942D983611F00C942D36552004
:1051A00011F00C942D36662011F00C942D367720DA
:1051B00011F00C942D36882011F00C942D36992086
:1051C00011F00C942D363EC3A22DA33689F4B32DD5
:1051D000B23371F4E42DE93659F4552049F46620D0
:1051E00039F4772029F4882019F4992009F426C38A
:1051F000F22DF43611F00C942D36832D833611F0F8
:105200000C942D36942D9C3611F00C942D3655208F
:1052100011F00C942D36662011F00C942D36772069
:1052200011F00C942D36882011F00C942D36992015
:1052300011F00C942D360C945931A22DA63391F413
:10524000B32DB93679F4E42DE53761F4F52DF53653
:1052500049F4662039F4772029F4882019F499203C
:1052600009F411C59101A201B301C401F6E3AF2E07
:10527000E9E6BE2E05E7C02E15E6D12EEE24FF246A
:1052800000E010E00E949177823008F04CC1822D3E
:105290008C3691F4932D943779F4A42DA43761F4CE
:1052A000552051F4662041F4772031F4882021F410
:1052B000992011F40C945E359101A201B301C4014F
:1052C000BCE6AB2EA4E7BA2EF4E7CF2EDD24EE2405
:1052D000FF2400E010E00E949177823008F087C040
:1052E000B22DB03391F4E32DE13379F4F42DF1379D
:1052F00061F4552051F4662041F4772031F4882080
:1053000021F4992011F40C94B9319101A201B30157
:10531000C401E0E3AE2E01E3B02E11E7C12EDD247F
:10532000EE24FF2400E010E00E949177823028F5FF
:10533000822D853711F00C942D36932D933611F074
:105340000C942D36A42DAD3611F00C942D3655202D
:1053500011F00C942D36662011F00C942D36772028
:1053600011F00C942D36882011F00C942D369920D4
:1053700011F00C942D360C941C32B22DB13391F4F3
:10538000E32DE13379F4F42DF13761F4552051F434
:10539000662041F4772031F4882021F4992011F41B
:1053A0000C941C32822D803711F00C942D36932DE5
:1053B000953611F00C942D36A42DA23711F00C94D3
:1053C0002D36552011F00C942D36662011F00C94DA
:1053D0002D36772011F00C942D36882011F00C9486
:1053E0002D36992011F00C942D360C949433B22D57
:1053F000B43791F4E32DEF3679F4F42DFF3661F4F0
:10540000852D823649F4662039F4772029F48820E6
:1054100019F4992009F47EC59101A201B301C401D8
:10542000B4E7AB2EAFE6BA2EFFE6CF2EE2E6DE2ED5
:10543000EE24FF2400E010E00E9491778230C8F54E
:10544000922D943789F4A32DA83771F4B42DB43775
:1054500059F4552049F4662039F4772029F488203E
:1054600019F4992009F459C5E22DE43711F00C9490
:105470002D36F32DF43611F00C942D36842D87370C
:1054800011F00C942D36552011F00C942D36662019
:1054900011F00C942D36772011F00C942D368820C5
:1054A00011F00C942D36992011F00C942D360C949B
:1054B000BE35922D993691F4A32DAC3679F4B42DE6
:1054C000B13661F4E52DE33649F4662039F47720EE
:1054D00029F4882019F4992009F4E0C1F22DFE3650
:1054E00011F00C942D36832D813611F00C942D364D
:1054F000942D983611F00C942D36A52DA33611F06D
:105500000C942D36662011F00C942D36772011F076
:105510000C942D36882011F00C942D36992011F022
:105520000C942D36CCC4B22DB13691F4E32DEC366B
:1055300079F4F42DF53661F4852D823749F466202F
:1055400039F4772029F4882019F4992009F4B1C39B
:105550009101A201B301C40101E6A02E1CE6B12E07
:10556000B5E6CB2EA2E7DA2EEE24FF2400E010E011
:105570000E949177823008F09FC0922D923791F46B
:10558000A32DA73779F4B42DB03761F4E52DE037BA
:1055900049F4662039F4772029F4882019F49920F9
:1055A00009F454C19101A201B301C401F2E7AF2E85
:1055B000E7E7BE2E00E7C02E10E7D12EEE24FF2431
:1055C00000E010E00E9491778230D0F5F22DF037A4
:1055D00091F4832D8C3679F4942D953661F4A52DB4
:1055E000A83649F4662039F4772029F4882019F484
:1055F000992009F444C3B22DB13611F00C942D3624
:10560000E32DED3611F00C942D36F42DF53711F015
:105610000C942D36852D883611F00C942D3666208D
:1056200011F00C942D36772011F00C942D36882033
:1056300011F00C942D36992011F00C942D368FC753
:10564000922D933799F4A32DA53681F4B42DB2375A
:1056500069F4E52DE03751F4662041F4772031F408
:10566000882021F4992011F40C94C534F22DF337DD
:1056700011F00C942D36832D823711F00C942D36B9
:10568000942D973711F00C942D36A52DA03711F0DD
:105690000C942D36662011F00C942D36772011F0E5
:1056A0000C942D36882011F00C942D36992011F091
:1056B0000C942D360C946033B22DB73791F4E32D52
:1056C000E03779F4F42DF83761F4852D843749F407
:1056D000662039F4772029F4882019F4992009F4F8
:1056E000C8C39101A201B301C401B7E7AB2EA0E783
:1056F000BA2EF8E7CF2EE4E7DE2EEE24FF2400E0FA
:1057000010E00E9491778230D0F5922D943791F479
:10571000A32DA33779F4B42DB53661F4E52DE23726
:1057200049F4662039F4772029F4882019F4992067
:1057300009F4C3C7F22DF43711F00C942D36832DE4
:10574000833711F00C942D36942D953611F00C946E
:105750002D36A52DA43711F00C942D36662011F0AE
:105760000C942D36772011F00C942D36882011F0F2
:105770000C942D36992011F00C942D36F5C3B22DD2
:10578000B23791F4E32DE73679F4F42DF03761F474
:10579000852D853749F4662039F4772029F488204F
:1057A00019F4992009F454C5922D9C3611F00C94EB
:1057B0002D36A32DA13611F00C942D36B42DB4370F
:1057C00011F00C942D36E52DE83711F00C942D36A0
:1057D000662011F00C942D36772011F00C942D36A4
:1057E000882011F00C942D36992011F00C942D3650
:1057F0000C9424350E943A170C942F3680ED61E00A
:105800004CE021E00E94305280ED61E04EE021E06A
:105810000E94305280ED61E040E121E00E94305270
:1058200080ED61E042E121E00E94305280ED61E0D4
:1058300040E122E00E9430520C942F360E948611E3
:105840000C942F360E94C3170C942F366091F205EA
:105850007091F30580E090E00E949C838C0165EFDD
:1058600073E00E94B183009719F477980C942F3657
:10587000C80168EF73E00E94B183009719F4779A2A
:105880000C942F36779903C085EF93E002C088EF20
:1058900093E000D000D02CE633E060C56091F205C3
:1058A0007091F30580E090E00E949C838C0167ED8D
:1058B00073E00E94B183009709F052C06091F20535
:1058C0007091F30580E090E00E949C838C0100972A
:1058D00011F40C942F366CEF73E00E94B1830097A3
:1058E00029F482E29FEFACECBBE30BC0C80162E09D
:1058F00074E00E94B183009789F482E29FEFACECE0
:10590000BAE38093E4059093E505A093E605B09390
:10591000E70584EE95E066E070E0DCC0C8010E9417
:1059200086827B018C0120E030E0A9010E944A7C44
:10593000882391F081E00E94E90B9B01AC01C80132
:10594000B7010E944E7C6093E4057093E505809357
:10595000E6059093E705DDCF00D08CEA93E08CC09C
:10596000C8016AED73E00E94B183009709F052C04C
:105970006091F2057091F30580E090E00E949C83B5
:105980008C01009711F40C942F366CEF73E00E9499
:10599000B183009729F482E29FEFACECBBE30BC02C
:1059A000C80162E074E00E94B183009769F482E26A
:1059B0009FEFACECBAE38093E8059093E905A093E0
:1059C000EA05B093EB051DC0C8010E9486827B01E9
:1059D0008C0120E030E0A9010E944A7C8823B1F0CC
:1059E00082E00E94E90B9B01AC01C801B7010E9453
:1059F0004E7C6093E8057093E9058093EA059093E7
:105A0000EB0588EE95E06AE070E064C000D08FE9B5
:105A100093E067C0C80162ED73E00E94B183009714
:105A200009F06BC06091F2057091F30580E090E0A1
:105A30000E949C838C01009711F40C942F366CEF1C
:105A400073E00E94B183009769F487ED94E3AFEEB1
:105A5000BCE38093E0059093E105A093E205B09349
:105A6000E30534C0C80162E074E00E94B18300978E
:105A700041F400D080E993E0EDB7FEB792838183D3
:105A800036C0C8010E9486821B012C0120E030E054
:105A9000A9010E944A7C882309F180E00E94E90B59
:105AA0007B018C01C201B10121EE3AE744E95EE3DA
:105AB0000E94837BA80197010E944E7C6093E005C1
:105AC0007093E1058093E2059093E30580EE95E005
:105AD00062E070E044E050E00C94013600D083E8CE
:105AE00093E0ADB7BEB712969C938E9311970E9428
:105AF00041840F900F900C942F360E94370C00D0E9
:105B000000D000D02CE733E0EDB7FEB7328321831D
:105B1000ADB7BEB713966D937D938D939C931697F7
:105B20000E944184EDB7FEB736960FB6F894FEBFDB
:105B30000FBEEDBF81E00E94E90B2091E40530919A
:105B4000E5054091E6055091E7050E94947D7B01B3
:105B50008C0182E00E94E90B9B01AC018DB79EB7DE
:105B60000A970FB6F8949EBF0FBE8DBFCDB6DEB6B6
:105B70000894C11CD11C80E793E0ADB7BEB7129664
:105B80009C938E9311978E2D9F2DA02FB12FF601F0
:105B900082839383A483B583CA01B9012091E80568
:105BA0003091E9054091EA055091EB050E94947D02
:105BB000D60116966D937D938D939C9319970E94B1
:105BC0004184EDB7FEB73A960FB6F894FEBF0FBE0C
:105BD000EDBF51C06091F2057091F30580E090E057
:105BE0000E949C830097F9F00E942F1F20912208A9
:105BF000309123088217930759F1909323088093DB
:105C0000220882E298E060E070E042E050E00E940A
:105C10008A8500D085E693E0ADB7BEB712969C9317
:105C20008E93119707C000D08EE593E0EDB7FEB7D5
:105C3000928381830E94418460912208709123089D
:105C40000F900F9080E090E00E94841E0E944A0D09
:105C500000D083E593E0ADB7BEB712969C938E93C8
:105C600011970E9441840F900F906FEF7FEF80E0BB
:105C700090E00E94841E0E944A0D0C942F360E94D0
:105C8000461A0C942F3680915C22843329F480E0EC
:105C900061E040E00E94DF122091EC05222309F42C
:105CA000DEC700D000D0EDB7FEB7319680E593E0B7
:105CB00099C080915C22893709F088C06091F20513
:105CC0007091F30580E090E00E949C838C0165EF69
:105CD00073E00E94B183009731F480910A0690919D
:105CE0000B0690640CC0C80168EF73E00E94B1839A
:105CF000009791F480910A0690910B069F7B9093F8
:105D00000B0680930A068AE096E064E170E042E0C8
:105D100050E00E948A855AC0C80167E074E00E9482
:105D2000B1830097A1F5EDB7FEB73A970FB6F89497
:105D3000FEBF0FBEEDBF31968DEB93E0ADB7BEB7A2
:105D400012969C938E93119780917B1990917C1958
:105D50009383828380917D1990917E1995838483AA
:105D600080917F1990918019978386838091811902
:105D700090918219918780870E944184EDB7FEB788
:105D80003A960FB6F894FEBF0FBEEDBF1FC08091CC
:105D90000A0690910B0696FF03C085EF93E002C0C0
:105DA00088EF93E000D000D029EB33E0ADB7BEB769
:105DB00012963C932E93119714969C938E9313975F
:105DC0000E9441840F900F900F900F902091EC054E
:105DD000222309F444C700D000D0EDB7FEB73196B6
:105DE0008DE493E0ADB7BEB712969C938E93119756
:105DF000228313822BC76091F2057091F30580E036
:105E000090E00E949C836CEF73E00E94B183009746
:105E100011F481E001C080E00E947C1D2091EC051E
:105E2000222309F41CC700D000D0EDB7FEB731968D
:105E30008AE493E0D7CF0E94371B2091EC05222300
:105E400009F40DC700D000D0EDB7FEB7319687E456
:105E500093E0C8CF0E94321B2091EC05222309F465
:105E6000FEC600D000D0EDB7FEB7319684E493E0D3
:105E7000B9CF6091F2057091F30580E090E00E9447
:105E80009C830E948A82803150F48093270890E09E
:105E90000E942C5C87E298E066E170E027C000D0A9
:105EA00000D0EDB7FEB7319688EE93E0ADB7BEB740
:105EB00012969C938E9311978091270829C0609128
:105EC000F2057091F30580E090E00E949C830E94AF
:105ED0008A82982F9B50903160F480930C0690E05A
:105EE0000E94A45A8CE096E067E170E041E050E047
:105EF00088C600D000D0EDB7FEB7319682EF93E0B0
:105F0000ADB7BEB712969C938E93119780910C06F5
:105F100082836FCF0C940000A2C66091F20570914D
:105F2000F30580E090E00E949C83BC01009769F03B
:105F300086E699E14AE050E00E94BA8386E699E15C
:105F400062E270E04AE050E05CC600D000D08DE034
:105F500094E0EDB7FEB79283818386E699E194835E
:105F600083830E942F8474C66091F2057091F305BB
:105F700080E090E00E949C838C0165E174E00E94C7
:105F8000B183009739F4219A80910A0690910B060B
:105F900080612DC6C80167E174E00E94B18300975B
:105FA00039F4229A80910A0690910B0680621FC6EE
:105FB000C80169E174E00E94B183009739F4239A23
:105FC00080910A0690910B06806411C6C8016BE1AE
:105FD00074E00E94B183009739F4239A80910A06F5
:105FE00090910B06806803C6C8016DE174E00E94C1
:105FF000B1830097C9F480910A0690910B069160D5
:1060000090930B0680930A068AE096E064E170E0C4
:1060100042E050E00E948A858EE496E062E140E032
:1060200050E00E94D4441BC6C8016FE174E00E9496
:10603000B183009771F4E3E8F9E11192119289E1DB
:10604000E33AF807D1F780910A0690910B06926027
:10605000CEC5C80168EF73E00E94B1839C018091B6
:106060000A0690910B0621153105A9F48F709C7FCB
:1060700090930B0680930A062B9A8AE096E064E1DF
:1060800070E042E050E00E948A858091A42690E072
:106090000E94B95AE4C584FF03C085EF93E002C0B3
:1060A00088EF93E000D000D022E334E0ADB7BEB774
:1060B00012963C932E93119714969C938E9313975C
:1060C0000E94418480910A060F900F900F900F90CC
:1060D00085FF03C085EF93E002C088EF93E000D016
:1060E00000D027E234E0EDB7FEB7328321839483FA
:1060F00083830E94418480910A060F900F900F9035
:106100000F9086FF03C085EF93E002C088EF93E015
:1061100000D000D02CE134E0ADB7BEB712963C936E
:106120002E93119714969C938E9313970E944184FB
:1061300080910A060F900F900F900F9087FF03C079
:1061400085EF93E002C088EF93E000D000D021E11A
:1061500034E0EDB7FEB732832183948383830E94BA
:10616000418480910A0690910B060F900F900F903A
:106170000F9090FF03C085EF93E002C088EF93E09B
:1061800000D000D026E034E0ADB7BEB712963C9305
:106190002E93119714969C938E9313970E9441848B
:1061A00080910A0690910B060F900F900F900F9020
:1061B00091FF03C085EF93E002C088EF93E000D029
:1061C00000D02BEF33E0EDB7FEB732832183948309
:1061D00083830E94418480910A0690910B060F9060
:1061E0000F900F900F9091FF3AC581E294E00E94CA
:1061F000618403E819E13BE0C32ED12C29E2E22EB1
:1062000024E0F22ED8018D919D918D0100D000D017
:1062100000D0EDB7FEB73196ADB7BEB71296FC927F
:10622000EE921197D382C282958384830E942F8439
:106230000894C11CD11CEDB7FEB736960FB6F89482
:10624000FEBF0FBEEDBFFBE1CF16D104D9F607C5E7
:1062500000D080E493E0ADB7BEB712969C938E93C6
:1062600011970E9441842091EC050F900F902223FA
:10627000A9F000D000D0EDB7FEB731968DE393E0E2
:10628000ADB7BEB712969C938E931197228313825B
:106290000E9441840F900F900F900F9088E10FB6ED
:1062A000F89480936000109260000FBE0C94007C04
:1062B000D6C40E94E651D3C46091F2057091F305F3
:1062C00080E090E00E949C831C0165EF73E00E94D7
:1062D000B183009749F40E94835980910A069091F6
:1062E0000B0681608D7F83C4C10168EF73E00E945B
:1062F000B183009741F40E94E55880910A0690917D
:106300000B068C7F74C404E314E0C101B8010E9441
:10631000B183009749F40E94E55880910A06909154
:106320000B068E7F826063C480910A0681FF0BC0DA
:1063300000D000D081E494E0EDB7FEB79283818372
:106340001483038383C480FF03C085EF93E002C0FE
:1063500088EF93E000D000D02DE334E0ADB7BEB7B6
:1063600012963C932E93119714969C938E931397A9
:106370006DC400D083E193E0EDB7FEB792838183D3
:106380000E9441848DB79EB740970FB6F8949EBF88
:106390000FBE8DBFEDB7FEB7319685EF92E0ADB77A
:1063A000BEB712969C938E93119780915322909131
:1063B0005422A0915522B091562282839383A483C4
:1063C000B5838091472290914822A0914922B091B3
:1063D0004A2286839783A087B18780914B22909130
:1063E0004C22A0914D22B0914E2282879387A487A0
:1063F000B58780914F2290915022A0915122B09167
:10640000522286879787A08BB18B0E94418420916E
:10641000EC05EDB7FEB772960FB6F894FEBF0FBE4F
:10642000EDBF222309F41BC400D000D0EDB7FEB7A6
:10643000319682EF92E0D6CCF89481E090E00E9411
:106440004108182F80E090E00E944108082F7894BE
:10645000F89483E090E00E944108F82E82E090E0FA
:106460000E944108E82E789400D000D000D028EE99
:1064700032E0EDB7FEB7328321832091F4193091D9
:10648000F5194091F6195091F719ADB7BEB71396AB
:106490002D933D934D935C9316970E94418400D0B9
:1064A00000D0EDB7FEB7319621EC32E0ADB7BEB704
:1064B00012963C932E931197E2821382F4821582F6
:1064C00006831782108711860E944184EDB7FEB7BC
:1064D0003A960FB6F894FEBF0FBEEDBF0E94DA1BCE
:1064E0002091660000D000D0EDB7FEB7319685EB65
:1064F00092E0ADB7BEB712969C938E93119722830C
:1065000013820E9441840F900F900F900F900E9471
:106510004A0D2091EC05222309F4A1C300D000D03C
:10652000EDB7FEB7319682EB92E05CCC80E090E074
:1065300060E070E00E94560D81E090E060E070E065
:106540000E94560D2091EC05222309F488C300D047
:1065500000D0EDB7FEB731968FEA92E043CC0E94AF
:10656000B5190E944A0D2091EC05222309F477C346
:1065700000D000D0EDB7FEB731968CEA92E032CC75
:106580006091F2057091F30580E090E00E949C8399
:1065900069E374E00E94B183009741F5F89487E4C1
:1065A00098E00E94CB450CC0C8010F960E94174985
:1065B0008BE996E0B8010E948545C8010E9491468A
:1065C000082F192F0115110579F704C087E498E009
:1065D0000E940C4687E498E00E9471460097B1F74C
:1065E00087E498E00E94C74578945AC087E498E011
:1065F0000E94CB45482F592F7A010FE314E04CC07D
:10660000EDB7FEB774970FB6F894FEBF0FBEEDBF9F
:106610003196ADB7BEB712961C930E931197D70162
:106620001A968C911A978283138212968C911297E4
:106630008483158213968C91139786831782149600
:106640008C9114978087118617968C911797828763
:10665000138619968C9119978487158615968C91B7
:1066600015978687178618968C911897808B118AB4
:1066700016968C91828B138A0E942F84EDB7FEB7F9
:1066800074960FB6F894FEBF0FBEEDBFC7010E940F
:106690009146482F592F7A01E114F10409F0B0CF47
:1066A0002091EC05222309F4DAC200D000D0EDB726
:1066B000FEB7319689EA92E095CB0E94B61DCFC213
:1066C0006091F2057091F30580E090E00E949C8358
:1066D0008C016EE774E00E94B183009731F48091E1
:1066E0000A0690910B06937F82C2C80162E074E0B3
:1066F0000E94B183009739F480910A0690910B06AD
:10670000937F986074C2C80163E874E00E94B1830B
:10671000009739F480910A0690910B06937F94605C
:1067200066C20E9448089BC26091F2057091F30511
:1067300080E090E00E949C83009751F10E94B92074
:1067400020910406309105064091060650910706F7
:10675000621773078407950739F1609304067093F5
:106760000506809306069093070684E096E06EE0A7
:1067700070E044E050E00E948A8500D081EA92E017
:10678000EDB7FEB7928381830E9441840F900F90F2
:1067900060910406709105068091060690910706A7
:1067A0000E94C61F0E944A0D00D085E992E0ADB755
:1067B000BEB712969C938E9311970E9441840F90BE
:1067C0000F906FEF7FEFCB010E94C61F0E944A0D12
:1067D0002091EC05222309F442C200D000D0EDB78D
:1067E000FEB7319682E992E0FDCA6091F2057091A0
:1067F000F30580E090E00E949C83009741F160E007
:1068000070E04AE050E00E9478817093090660933E
:10681000080600D000D0EDB7FEB7319625E732E08C
:10682000ADB7BEB712963C932E93119773836283D4
:106830000E9441840F900F900F900F9088E096E097
:1068400062E170E042E050E00E948A8514C000D00E
:1068500000D084E592E0EDB7FEB79283818380910A
:10686000080690910906948383830E9441840F90C7
:106870000F900F900F902091EC05222309F4EFC1A7
:1068800000D000D0EDB7FEB7319681E592E0AACAFC
:106890000E9454492091EC05222309F4E0C100D064
:1068A00000D0EDB7FEB731968EE492E09BCA0E940D
:1068B00056222091EC05222309F4D1C100D000D04A
:1068C000EDB7FEB731968BE492E08CCA80E090E0A1
:1068D0000E94FF1B2091EC05222309F4C0C100D0C7
:1068E00000D0EDB7FEB7319688E492E07BCA809184
:1068F000411E81FF3BC00E94FA180097B9F500D0F5
:1069000000D000D08DE392E0EDB7FEB79283818393
:1069100080913D1A90913E1AA0913F1AB091401A71
:1069200083839483A583B6830E94418480E392E0AD
:10693000ADB7BEB712969C938E9311978091B926EE
:106940009091BA26A091BB26B091BC26EDB7FEB7B8
:1069500083839483A583B6830E9441848DB79EB7B9
:1069600006960FB6F8949EBF0FBE8DBF0E944A0DCB
:106970002091EC05222309F472C100D000D0EDB7BC
:10698000FEB731968DE292E02DCA8091411E82FFC2
:106990004EC083E061E048E021E00E94791400D01D
:1069A00000D000D086E292E0EDB7FEB792838183FB
:1069B0008091301A9091311AA091321AB091331A05
:1069C00083839483A583B6830E94418400D000D042
:1069D000EDB7FEB7319685E192E0ADB7BEB712963E
:1069E0009C938E9311978091341A9091351AA091AF
:1069F000361AB091371A82839383A483B58380912A
:106A0000381A9091391AA0913A1AB0913B1A86839C
:106A10009783A087B1870E944184EDB7FEB73A966D
:106A20000FB6F894FEBF0FBEEDBF0E944A0D209135
:106A3000EC05222309F413C100D000D0EDB7FEB756
:106A4000319682E192E0CEC96091F2057091F30532
:106A500080E090E00E949C836EE874E00E94B18325
:106A60000097B1F46091F2057091F30580E090E039
:106A70000E949C83009709F4F2C00E948A828031B0
:106A800008F0EDC090915201982B90935201E7C00D
:106A90008091520100D000D023E634E0EDB7FEB77C
:106AA0003283218390E08F709070948383830E945F
:106AB00041840F900F900F900F90DDC86091F20508
:106AC0007091F30580E090E00E949C83009781F133
:106AD00060E070E04AE050E00E944B80603100F5D9
:106AE00060930D0600D000D0EDB7FEB7319685E07B
:106AF00092E0ADB7BEB712969C938E9311976283C6
:106B000013820E9441840F900F900F900F908DE0A0
:106B100096E068E170E041E050E00E948A851FC085
:106B200000D000D0EDB7FEB731968CEF91E007C0F2
:106B300000D000D0EDB7FEB7319683EF91E0ADB74E
:106B4000BEB712969C938E93119780910D06828307
:106B500013820E9441840F900F900F900F900E941B
:106B60004A0D2091EC05222309F479C000D000D011
:106B7000EDB7FEB7319680EF91E034C96091F20530
:106B80007091F30580E090E00E949C838C0165EF9A
:106B900073E00E94B183009741F40E94C75780912F
:106BA0000A0690910B06906122C0C80168EF73E05D
:106BB0000E94B183009741F5F8940E94D55788E16F
:106BC0000FB6F89480936000109260000FBE84B7F7
:106BD000877F84BF809160008861809360001092FD
:106BE0006000789480910A0690910B069F7E9093A6
:106BF0000B0680930A068AE096E064E170E042E0CA
:106C000050E00E948A852BC0C80163E974E00E94AD
:106C1000B1839C0180910A0690910B0621153105E4
:106C200021F494FF1CC0F894FFCF94FF03C085EFBC
:106C300093E002C088EF93E000D000D020E734E07A
:106C4000EDB7FEB732832183948383830E9441840E
:106C50000F900F900F900F9002C00E941F1AA981F1
:106C6000BA8111961C921E9283E00F900F90CF91E3
:106C7000DF911F910F91FF90EF90DF90CF90BF9029
:106C8000AF909F908F907F906F905F904F903F90CC
:106C90002F900895F89491E2E0E0F0E0909357008F
:106CA0008491E2E0F0E0909357002491E4E0F0E07A
:106CB00090935700E49190E0A0E0B0E0DC019927C8
:106CC000882730E040E050E0542F432F322F222716
:106CD000820F931FA41FB51F8E0F911DA11DB11D03
:106CE0008093F4199093F519A093F619B093F719BE
:106CF00078940895DF93CF93CDB7DEB761970FB641
:106D0000F894DEBF0FBECDBFCE0104966EE070E0FA
:106D100044E050E00E946C858C819D81AE81BF81F2
:106D20008F3F2FEF92072FEFA2072FEFB20749F403
:106D300084E096E06EE070E044E050E00E948A85D6
:106D400008C08093040690930506A0930606B093AE
:106D50000706CE01029662E170E042E050E00E9438
:106D60006C858A819B812FEF8F3F920779F48CE3AA
:106D700090E0909309068093080688E096E062E12F
:106D800070E042E050E00E948A8504C090930906BA
:106D900080930806CE01029664E170E042E050E084
:106DA0000E946C858A819B812FEF8F3F920779F437
:106DB0008AE090E490930B0680930A068AE096E0BE
:106DC00064E170E042E050E00E948A8504C0909344
:106DD0000B0680930A06CE01029660E070E042E066
:106DE00050E00E946C858A819B812FEF8F3F920734
:106DF00069F4109223081092220882E298E060E081
:106E000070E042E050E00E948A8504C0909323081D
:106E1000809322088DEA96E269E170E049E050E053
:106E20000E946C850E94000FCE01049666E070E01F
:106E300044E050E00E946C858C819D81AE81BF81D1
:106E40008F3F2FEF92072FEFA2072FEFB20749F4E2
:106E500084EE95E066E070E044E050E00E948A85B0
:106E600008C084EE95E066E070E044E050E00E94E7
:106E70006C85CE0104966AE070E044E050E00E9428
:106E80006C858C819D81AE81BF818F3F2FEF9207F2
:106E90002FEFA2072FEFB20749F488EE95E06AE0E2
:106EA00070E044E050E00E948A8508C088EE95E0DA
:106EB0006AE070E044E050E00E946C85CE010496E8
:106EC00062E070E044E050E00E946C858C819D811E
:106ED000AE81BF818F3F2FEF92072FEFA2072FEFD9
:106EE000B20749F480EE95E062E070E044E050E0E3
:106EF0000E948A8508C080EE95E062E070E044E080
:106F000050E00E946C85CE01019666E170E041E0A0
:106F100050E00E946C8589818F3F49F487E298E0B8
:106F200066E170E041E050E00E948A8508C087E297
:106F300098E066E170E041E050E00E946C85CE018F
:106F4000019667E170E041E050E00E946C85898124
:106F50008F3F49F48CE096E067E170E041E050E05B
:106F60000E948A8508C08CE096E067E170E041E00D
:106F700050E00E946C85CE01019668E170E041E02E
:106F800050E00E946C8589818F3F49F48DE096E046
:106F900068E170E041E050E00E948A8508C08DE021
:106FA00096E068E170E041E050E00E946C85CE011F
:106FB000089662E270E04AE050E00E946C858885A5
:106FC0008F3F49F486E699E162E270E04AE050E0E2
:106FD0000E948A8508C086E699E162E270E04AE094
:106FE00050E00E946C8561960FB6F894DEBF0FBE2C
:106FF000CDBFCF91DF9108950E94BB576C9A6B9AD9
:107000006A9A6F9A729A749A739A779A809880B3F0
:10701000897F80BB8398849887E080937E00549A10
:107020000E944A360E947A3681E00E945D0B80E021
:1070300090E00E94140F0E94545080910A0686FD31
:10704000239A0895CF93DF93EC018881998100976B
:1070500031F02CE08738920709F099C08FC00E9468
:10706000FC3780910A0680FD06C081FF02C01D9991
:1070700002C00E94E558809170008C7F8093700060
:107080008091B60080628093B6001092B20082E0D8
:107090008093B1008091B60090E087709070009767
:1070A000C9F78091700081608093700080E090E06B
:1070B0006FE678E00E949E570E94321B80E00E949B
:1070C0007C1D00D08AEE91E0ADB7BEB712969C93BE
:1070D0008E9311970E9441840F900F900E94861109
:1070E0008091411E86FF02C00E9491518091270825
:1070F00090E00E942C5C80910C0690E00E94A45AC3
:107100000E94A15A8093550880910C0690E00E943D
:10711000A45A00D000D000D0EDB7FEB7319688E970
:1071200094E0ADB7BEB712969C938E931197809161
:1071300055088283138280912708848315820E94D8
:107140002F841092540810925308EDB7FEB736966C
:107150000FB6F894FEBF0FBEEDBF8AE196E09093A4
:10716000B7268093B62683E290E090934C088093F4
:107170004B0887E89CE0998388830DC0633259F4FB
:1071800083E598E060E070E00E944924E6CF198230
:10719000188283E001C081E0DF91CF9108958436A9
:1071A000910534F100D000D02AEA34E0EDB7FEB703
:1071B00032832183948383830E942F84809153227E
:1071C00090915422A0915522B09156220196A11D72
:1071D000B11D8093532290935422A0935522B093D3
:1071E00056220F900F900F900F9021E030E002C0D8
:1071F00020E030E0C90108954F925F926F927F9234
:107200008F929F92AF92BF92CF92DF92EF92FF92B6
:107210000F931F93DF93CF93CDB7DEB7CB58D040FA
:107220000FB6F894DEBF0FBECDBF2C01633871F4EA
:1072300083E398E0C557DF4F6883CB58D0400E9466
:107240000B43C557DF4F6881CB58D040D2012D91F9
:107250003C911197BCE02A333B0711F40C94234274
:10726000ECE02B333E0750F421153105A9F0FBE08B
:1072700024313F0711F00C9475421AC04CE02B34B6
:10728000340711F40C944C425CE02235350711F0C0
:107290000C9475420C94644283E398E061E870E0DA
:1072A00047E956E00E94F04284E19BE00C941E42C4
:1072B000623111F00C947B4280910A0690910B068A
:1072C00091FDF2CF8091040690910506A0910606EB
:1072D000B0910706A0FD8C9A0E946E0C8091040666
:1072E00090910506A0910606B091070694FF02C092
:1072F0000E94FA188091040690910506A091060656
:10730000B091070695FF0AC00E94370C6093A02633
:107310007093A1268093A2269093A32680910406C1
:1073200080FF32C0EDB7FEB738970FB6F894FEBFB6
:107330000FBEEDBF3196CE014396ADB7BEB71296E4
:107340009C938E93119787E790E0938382838EEBD3
:1073500094E09583848386E699E1978386830E94EF
:107360009884E82E092FEDB7FEB738960FB6F8943B
:10737000FEBF0FBEEDBF0E94CF38009709F094CF3B
:10738000802F0E2D182F02C000E010E0809104061F
:1073900081FF5FC043E1C42ED12CCC0EDD1E00D096
:1073A00000D000D0EDB7FEB73196C601800F911F17
:1073B000ADB7BEB712969C938E93119787E790E076
:1073C0009383828386EC94E0958384830E949884DF
:1073D000080F191F3DEAE32E36E2F32EEDB7FEB794
:1073E00036960FB6F894FEBF0FBEEDBF27E7A22E6C
:1073F000B12C9AED892E92E0992ED7012D917D0125
:10740000EDB7FEB738970FB6F894FEBF0FBEEDBFCD
:107410003196C601800F911FADB7BEB712969C93EF
:107420008E931197B382A2829582848226831782DB
:107430000E949884080F191FEDB7FEB738960FB653
:10744000F894FEBF0FBEEDBFF5EBEF16F6E2FF06B8
:10745000A1F68091040682FF6EC083E1C82ED12C74
:10746000CC0EDD1E00D000D000D0EDB7FEB73196B7
:10747000C601800F911FADB7BEB712969C938E9335
:10748000119787E790E0938382838AEC94E0958359
:1074900084830E949884080F191F7E010894E11CC0
:1074A000F11C80E1F70111928A95E9F72DB73EB7FB
:1074B0002A5F3F4F0FB6F8943EBF0FBE2DBF80EB43
:1074C00068E9A70128E00E949712B9E0AB2EB12C21
:1074D000AC0EBD1EA7E78A2E912CFAED6F2EF2E0BE
:1074E0007F2ED7012D917D01EDB7FEB738970FB6EE
:1074F000F894FEBF0FBEEDBF3196C601800F911FFD
:10750000ADB7BEB712969C938E93119793828282E9
:1075100075826482268317820E949884080F191F3F
:10752000EDB7FEB738960FB6F894FEBF0FBEEDBFAD
:10753000EA14FB04B1F68091040690910506A0912F
:107540000606B09107060097A105B10581F12DB798
:107550003EB7285030400FB6F8943EBF0FBE2DBF47
:10756000EDB7FEB73196CE014396800F911FADB7B0
:10757000BEB712969C938E93119787E790E0938302
:1075800082838FEC94E09583848380912508909189
:107590002608978386830E949884080F191FEDB7E9
:1075A000FEB738960FB6F894FEBF0FBEEDBF8091C0
:1075B000040683FF50C089E290E06BE270E04AE28B
:1075C00050E027E00E946A4D8DEA96E20E94DA4F71
:1075D0002DB73EB72A5030400FB6F8943EBF0FBECD
:1075E0002DBFEDB6FEB60894E11CF11C9E012D5E88
:1075F0003F4F200F311FADB7BEB712963C932E936D
:10760000119727E730E0F7013383228326ED34E03A
:10761000358324839C01B901882777FD8095982FB5
:107620000E94B87C20E030E048EC52E40E944E7C9E
:10763000D70116966D937D938D939C9319970E9415
:107640009884080F191FEDB7FEB73A960FB6F89455
:10765000FEBF0FBEEDBF8091040684FF56C089E2D5
:1076600090E06BE270E04AE250E026E00E946A4D52
:1076700081E090E00E94BE0C809329088CEA99E199
:107680000E94DA4F2DB73EB72A5030400FB6F8941B
:107690003EBF0FBE2DBFEDB6FEB60894E11CF11C37
:1076A0009E012D5E3F4F200F311FADB7BEB7129622
:1076B0003C932E93119727E730E0F7013383228321
:1076C00020EE34E0358324839C01B901882777FDBF
:1076D0008095982F0E94B87C20E030E048EC52E47E
:1076E0000E944E7CD70116966D937D938D939C934B
:1076F00019970E949884080F191FEDB7FEB73A96A4
:107700000FB6F894FEBF0FBEEDBF8091040685FF53
:1077100036C02DB73EB72A5030400FB6F8943EBF62
:107720000FBE2DBFEDB7FEB73196CE014396800F49
:10773000911FADB7BEB712969C938E93119787E7B2
:1077400090E0938382838BEE94E095838483809191
:10775000701990917119A0917219B0917319868363
:107760009783A087B1870E949884080F191FEDB7EF
:10777000FEB73A960FB6F894FEBF0FBEEDBF8091EC
:10778000040686FF31C00E944B0C2DB73EB72A502D
:1077900030400FB6F8943EBF0FBE2DBFEDB7FEB719
:1077A00031969E012D5E3F4F200F311FADB7BEB702
:1077B00012963C932E93119727E730E03383228370
:1077C00029EF34E03583248366837783808791872C
:1077D0000E949884080F191FEDB7FEB73A960FB6AE
:1077E000F894FEBF0FBEEDBF8091040687FF3AC03C
:1077F000F8948091982690919926A0919A26B0911C
:107800009B2678942DB73EB72A5030400FB6F89497
:107810003EBF0FBE2DBF4DB75EB74F5F5F4F9E019E
:107820002D5E3F4F200F311FEDB7FEB7328321830E
:1078300027E730E0FA013383228327E035E0358300
:10784000248386839783A087B1870E949884080F3A
:10785000191F2DB73EB7265F3F4F0FB6F8943EBFB6
:107860000FBE2DBF8091040690910506A0910606DB
:10787000B091070690FF92C080910806909109068A
:10788000009709F48BC0F894C0909826D090992660
:10789000E0909A26F0909B2678948091A41990917C
:1078A000A519A091A619B091A719A7019601281BA7
:1078B000390B4A0B5B0BCA01B9010E94B67C862EBC
:1078C000A72E682EB92E609108067091090680E0F7
:1078D00090E00E94B67C9B01AC01682D7A2D862D2C
:1078E0009B2D0E944E7C5C014DB75EB74A505040C4
:1078F0000FB6F8945EBF0FBE4DBFEDB7FEB7319621
:10790000CE014396800F911FADB7BEB712969C93E0
:107910008E93119787E790E09383828380E195E0CF
:1079200095838483262F372F4A2D5B2D268337831B
:1079300040875187C557DF4F6883CB58D040C65723
:10794000DF4F7883CA58D0400E949884080F191FCF
:10795000C557DF4F6881CB58D040C657DF4F78817D
:10796000CA58D040862F972FAA2DBB2D8093A526CD
:107970009093A626A093A726B093A826C092A419F8
:10798000D092A519E092A619F092A719EDB7FEB70B
:107990003A960FB6F894FEBF0FBEEDBF8091040675
:1079A00090910506A0910606B091070691FF40C090
:1079B000F89480919C2690919D26A0919E26B0914E
:1079C0009F2678942DB73EB72A5030400FB6F894D2
:1079D0003EBF0FBE2DBF4DB75EB74F5F5F4F9E01DD
:1079E0002D5E3F4F200F311FEDB7FEB7328321834D
:1079F00027E730E0FA01338322832DE135E0358338
:107A0000248386839783A087B1870E949884080F78
:107A1000191F2DB73EB7265F3F4F0FB6F8943EBFF4
:107A20000FBE2DBFC8010E94CF38009709F03CCC93
:107A30008091040690910506A0910606B091070674
:107A400092FF92C08091080690910906009709F470
:107A50008BC0F894C0909C26D0909D26E0909E26E6
:107A6000F0909F2678948091A8199091A919A091DF
:107A7000AA19B091AB19A7019601281B390B4A0B23
:107A80005B0BCA01B9010E94B67C862EA72E682E18
:107A9000B92E609108067091090680E090E00E947E
:107AA000B67C9B01AC01682D7A2D862D9B2D0E9402
:107AB0004E7C5C014DB75EB74A5050400FB6F8940B
:107AC0005EBF0FBE4DBFEDB7FEB73196CE014396F8
:107AD000800F911FADB7BEB712969C938E931197EE
:107AE00087E790E09383828386E295E095838483A1
:107AF000262F372F4A2D5B2D2683378340875187CA
:107B0000C557DF4F6883CB58D040C657DF4F7883C7
:107B1000CA58D0400E949884080F191FC557DF4FDC
:107B20006881CB58D040C657DF4F7881CA58D040C3
:107B3000862F972FAA2DBB2D8093A9269093AA2636
:107B4000A093AB26B093AC26C092A819D092A919E5
:107B5000E092AA19F092AB19EDB7FEB73A960FB6BC
:107B6000F894FEBF0FBEEDBF80910406909105060C
:107B7000A0910606B091070693FF3EC08091432274
:107B800090914422A0914522B09146222DB73EB754
:107B90002A5030400FB6F8943EBF0FBE2DBF4DB7F0
:107BA0005EB74F5F5F4F9E012D5E3F4F200F311F2D
:107BB000EDB7FEB73283218327E730E0FA01338344
:107BC000228323E335E03583248386839783A0874C
:107BD000B1870E949884080F191F2DB73EB7265F02
:107BE0003F4F0FB6F8943EBF0FBE2DBFC8010E9495
:107BF000CF38009709F058CB809104069091050684
:107C0000A0910606B091070694FF3CC04DB75EB741
:107C10004A5050400FB6F8945EBF0FBE4DBFEDB74F
:107C2000FEB73196CE014396800F911FADB7BEB718
:107C300012969C938E93119787E790E093838283AB
:107C40008CE395E09583848380913D1A90913E1A50
:107C5000A0913F1AB091401A86839783A087B1877D
:107C60000E949884080F191FEDB7FEB73A960FB619
:107C7000F894FEBF0FBEEDBFC8010E94CF38009739
:107C800009F012CB8091040690910506A09106069A
:107C9000B091070695FF3CC02DB73EB72A50304043
:107CA0000FB6F8943EBF0FBE2DBFEDB7FEB73196AD
:107CB000CE014396800F911FADB7BEB712969C932D
:107CC0008E93119787E790E09383828387E495E012
:107CD000958384838091A0269091A126A091A226CD
:107CE000B091A32686839783A087B1870E9498844A
:107CF000080F191FEDB7FEB73A960FB6F894FEBFFE
:107D00000FBEEDBFC8010E94CF38009709F0CCCA62
:107D10008091040690910506A0910606B091070691
:107D200096FF48C081E00E94E90B2DB73EB72A506C
:107D300030400FB6F8943EBF0FBE2DBFEDB6FEB675
:107D40000894E11CF11C9E012D5E3F4F200F311F56
:107D5000ADB7BEB712963C932E93119727E730E04C
:107D6000F7013383228324E535E035832483209192
:107D7000E4053091E5054091E6055091E7050E9444
:107D8000947DD70116966D937D938D939C9319974F
:107D90000E949884080F191FEDB7FEB73A960FB6E8
:107DA000F894FEBF0FBEEDBFC8010E94CF38009708
:107DB00009F07ACA8091040690910506A091060602
:107DC000B091070697FF48C082E00E94E90B2DB7EB
:107DD0003EB72A5030400FB6F8943EBF0FBE2DBFBD
:107DE000EDB6FEB60894E11CF11C9E012D5E3F4FDE
:107DF000200F311FADB7BEB712963C932E9311974B
:107E000027E730E0F7013383228321E635E035832D
:107E100024832091E8053091E9054091EA055091CD
:107E2000EB050E94947DD70116966D937D938D93FB
:107E30009C9319970E949884080F191FEDB7FEB7FD
:107E40003A960FB6F894FEBF0FBEEDBFC8010E9470
:107E5000CF38009709F028CA809104069091050652
:107E6000A0910606B0910706A0FF39C083E00E94EA
:107E7000E90B2DB73EB72A5030400FB6F8943EBFFD
:107E80000FBE2DBFEDB7FEB731969E012D5E3F4F61
:107E9000200F311FADB7BEB712963C932E931197AA
:107EA00027E730E0338322832EE635E035832483D1
:107EB00066837783808791870E949884080F191FB3
:107EC0008C98EDB7FEB73A960FB6F894FEBF0FBE8A
:107ED000EDBFC8010E94CF38009709F0E5C9809135
:107EE000040690910506A0910606B0910706A1FF31
:107EF0003FC08091411E87FF3BC080ED61E042E1C1
:107F000021E00E9430522DB73EB72A5030400FB6C4
:107F1000F8943EBF0FBE2DBFEDB7FEB731969E0160
:107F20002D5E3F4F200F311FADB7BEB712963C9369
:107F30002E93119727E730E0338322832BE735E038
:107F40003583248366837783808791870E94988412
:107F5000080F191FEDB7FEB73A960FB6F894FEBF9B
:107F60000FBEEDBFC8010E94CF38009709F09CC931
:107F70008091040690910506A0910606B09107062F
:107F8000A2FF3FC08091411E87FF3BC080ED62E0B1
:107F900042E121E00E9430522DB73EB72A503040D6
:107FA0000FB6F8943EBF0FBE2DBFEDB7FEB73196AA
:107FB0009E012D5E3F4F200F311FADB7BEB7129609
:107FC0003C932E93119727E730E03383228329E8EF
:107FD00035E03583248366837783808791870E9489
:107FE0009884080F191FEDB7FEB73A960FB6F894AC
:107FF000FEBF0FBEEDBFC8010E94CF38009709F049
:1080000053C98091040690910506A0910606B0918F
:108010000706A3FF3FC08091411E87FF3BC080ED54
:1080200063E042E121E00E9430522DB73EB72A5072
:1080300030400FB6F8943EBF0FBE2DBFEDB7FEB770
:1080400031969E012D5E3F4F200F311FADB7BEB759
:1080500012963C932E93119727E730E033832283C7
:1080600027E935E03583248366837783808791878A
:108070000E949884080F191FEDB7FEB73A960FB605
:10808000F894FEBF0FBEEDBFC8010E94CF38009725
:1080900009F00AC98091040690910506A091060690
:1080A000B0910706A4FF3FC08091411E87FF3BC0EF
:1080B00080ED64E042E121E00E9430522DB73EB7EE
:1080C0002A5030400FB6F8943EBF0FBE2DBFEDB71B
:1080D000FEB731969E012D5E3F4F200F311FADB789
:1080E000BEB712963C932E93119727E730E0338367
:1080F000228325EA35E0358324836683778380876E
:1081000091870E949884080F191FEDB7FEB73A9621
:108110000FB6F894FEBF0FBEEDBFC8010E94CF3866
:10812000009709F0C1C88091040690910506A091BE
:108130000606B0910706A5FF0AC08091411E82FF86
:1081400006C083E061E046E020E00E94791480915F
:10815000040690910506A0910606B0910706A6FFB9
:108160000AC08091411E82FF06C083E061E046E0C4
:1081700021E00E9479148091040690910506A09157
:108180000606B0910706A5FF40C08091411E82FF00
:108190003CC02DB73EB72A5030400FB6F8943EBFD2
:1081A0000FBE2DBFEDB7FEB73196CE014396800FBF
:1081B000911FADB7BEB712969C938E93119787E728
:1081C00090E09383828383EB95E095838483809111
:1081D000341A9091351AA091361AB091371A8683C5
:1081E0009783A087B1870E949884080F191FEDB765
:1081F000FEB73A960FB6F894FEBF0FBEEDBFC801AA
:108200000E94CF38009709F04FC8809104069091E2
:108210000506A0910606B0910706A6FF41C0809111
:10822000411E82FF3DC02DB73EB72A5030400FB6E9
:10823000F8943EBF0FBE2DBFEDB7FEB73196CE010D
:108240004396800F911FADB7BEB712969C938E9345
:10825000119787E790E0938382838BEB95E095837A
:1082600084838091381A9091391AA0913A1AB0916A
:108270003B1A86839783A087B1870E949884080F52
:10828000191FEDB7FEB73A960FB6F894FEBF0FBEB2
:10829000EDBFC8010E94CF38009711F00C945439FB
:1082A000779A809122089091230892FD749A809188
:1082B000040690910506A0910606B0910706009766
:1082C000A105B105E9F1809122089091230882FD72
:1082D00008C080910A0680FD04C081FF31C01D9B4B
:1082E0002FC000D000D086EC95E0ADB7BEB7129697
:1082F0009C938E931197CE01439614969C938E93E4
:1083000013970E942F842091EC050F900F900F90EF
:108310000F902223A9F000D000D0EDB7FEB7319620
:1083200084EE91E0ADB7BEB712969C938E931197F1
:10833000228313820E9441840F900F900F900F9020
:1083400080910D068061898B809146088A8BFE01A1
:10835000E00FF11F138A68010894C11CD11C8091A1
:1083600022089091230880FF12C000D000D08DEC2D
:1083700095E0EDB7FEB7928381830D5F1F4F1483A5
:1083800003830E942F840F900F900F900F90E2E0D4
:10839000EE2EF12CEC0CFD1C8E010F5E1F4FC80160
:1083A000B7010E94684C80910A0682FF08C084EFE2
:1083B00095E0B801A70128E932E20E94ED508091D2
:1083C00022089091230882FD73980E94835983E3C9
:1083D00098E00E940E4380910A0690910B0690FF50
:1083E00043C000910806109109060E94A15AE82E88
:1083F000109209061092080689E190E00E94B95A8D
:1084000024C07398809146088F5F809346088A8BBA
:10841000B6016F5F7F4FCE0141960E94684C83E3A7
:1084200098E00E940E4380915C1090915D1065E889
:1084300040E050E00E94D4448AE39CE0D2011196CF
:108440009C938E9358C0CC24DD2420910A06309151
:108450000B0630FDD6CF8E2D90E00E94B95A1093B6
:10846000090600930806739A8091250890912608C2
:10847000009711F00E94E558809146088F5F809325
:108480004608809122089091230882FD02C00C9436
:108490005439739A0C9454398EE398E00E94B5478E
:1084A000009749F10E94835980910A0687FD2B9815
:1084B0008EE398E060E470E00E948A4782E59CE0E9
:1084C000F2019183808317C08EE398E00E94B54744
:1084D000009789F00E94E55880910A0687FD02C046
:1084E0000C9454392B9A0C945439D20111961C9245
:1084F0001E9283E001C081E0C557DF4F0FB6F894AC
:10850000DEBF0FBECDBFCF91DF911F910F91FF90C6
:10851000EF90DF90CF90BF90AF909F908F907F9023
:108520006F905F904F9008950E943843089508958A
:10853000FC01DB018C91808311968C9111978183D2
:108540000895FC01DB0190818C91981741F421E0A2
:1085500030E0918111968C911197981711F020E0DD
:1085600030E0C9010895FC0180818093BD2681819E
:108570008093BE260895DC011996ED91FC911A971F
:108580000280F381E02D309709F009950895EF926C
:10859000FF920F931F93DF93CF9300D0CDB7DEB739
:1085A0008C0188E10E94E34CBC017E010894E11C2F
:1085B000F11CC7010E949842D8011996ED91FC91D7
:1085C0001A970190F081E02DC801B70109950F902D
:1085D0000F90CF91DF911F910F91FF90EF90089531
:1085E000EF92FF920F931F93CF93DF93EC018B01D8
:1085F0007A0147EA56E00E941C43FA86E986C801E0
:108600006BEA76E00E947B43DF91CF911F910F913F
:10861000FF90EF9008950E9435430895CF93DF9324
:10862000EC0188E16DEB76E20E94D94CCE010E940C
:108630003843DF91CF910895EF92FF920F931F93EC
:10864000CF93DF93EC018B017A010E945443F886AB
:10865000EF82C8016FEA76E00E947B43DF91CF9101
:108660001F910F91FF90EF9008950E945D43089530
:108670000E945A5F0895FC01A781B0852D913C911D
:10868000F90109950895DC011796ED91FC91189771
:108690000280F381E02D309709F00995089588E56F
:1086A00090E10E94C7450895FC017383628388E5C9
:1086B00090E1BF010E9452460895BC0188E590E117
:1086C0000E9419460895CF93DF93EC0188E590E16D
:1086D0000E94CB4508C0828193818C179D0739F099
:1086E000CF010E949146E82FF92F3097A1F7CF01D3
:1086F000DF91CF9108950F931F93CF93DF938B0159
:108700000E946343EC01009731F01D830C83C80184
:108710000E94B2618E83DF91CF911F910F910895D6
:108720001F93CF93DF93EC01162F888580FF1DC028
:10873000EC81FD813097C9F0D0935D10C0935C103F
:1087400082E08887CE0106960995992787FD909546
:1087500002978230910510F0133829F4CE01BE0142
:108760000E94B94302C081E08887DF91CF911F91B9
:108770000895CF92DF92EF92FF920F931F93CF93C2
:10878000DF93EC017B01C0905C10D0905D100091F4
:108790005A1010915B10F80103C00190F081E02D98
:1087A000EC17FD0719F03097C1F746C0209709F480
:1087B00043C08885882309F118860BC0C017D107EC
:1087C00029F0C80167E8AE010E949043F8010081DA
:1087D00011810115110591F7EC81FD81309769F048
:1087E000CE15DF0551F0D0935D10C0935C10CE0123
:1087F000069663E840E050E00995E0915A10F09148
:108800005B10CE17DF0791F48881998190935B10FC
:1088100080935A100DC0808191818C179D0729F497
:10882000888199819183808303C0FC01309799F7F7
:10883000D0925D10C0925C10DF91CF911F910F918B
:10884000FF90EF90DF90CF9008951F93CF93DF9329
:1088500010925E10C0915A10D0915B1011E00EC0C2
:108860008985882341F018871986CE0162E840E0A7
:1088700050E00E9490430990D881C02D209781F745
:10888000DF91CF911F91089580910911982F9F5FDB
:1088900090930911089560915C1070915D100E9491
:1088A000B94308958AE880930911109260101092DC
:1088B0005F1010925B1010925A1010925D1010927F
:1088C0005C10089580915E10882311F00E94254469
:1088D00070915F10772309F455C02091601030E04B
:1088E000F901EE0FFF1FEE0FFF1FE20FF31FEF590D
:1088F000FF4E6081609308114181528150930711AE
:108900004093061183819481909305118093041103
:108910002F5F3F4F2F713070209360107150709314
:108920005F10009741F580915A1090915B1018C02C
:1089300080915E10882311F00E9425444091061119
:1089400050910711809102119091031160910811CB
:108950000E949043E0910211F09103118081918176
:108960009093031180930211809102119091031151
:108970000097F1F607C0613819F421E0FC01208767
:108980000E94904380915E1020915F1030E0280F8C
:10899000311DC901089580915E1020915F1030E073
:1089A000280F311DC901089570915F107032D9F000
:1089B00020916010270F2F712093011130E0F901F1
:1089C000EE0FFF1FEE0FFF1FE20FF31FEF59FF4ED9
:1089D000608352834183948383837F5F70935F10AE
:1089E00020E030E002C021E030E0C9010895CF93DB
:1089F000DF93C0915C10D0915D100E949043D093A2
:108A00005D10C0935C10DF91CF910895FC01AB0124
:108A100090915A1080915B109C01A32FB22F03C03C
:108A20000D90BC91A02DAE17BF0791F01097C1F724
:108A3000309771F090838183F0935B10E0935A102C
:108A400081E0808717821682CF0161E80E94F74497
:108A50000895FC01009741F080858150823020F418
:108A600081E0818780935E10089521E030E0FC0171
:108A70008085882311F420E030E0C9010895CF9368
:108A8000DF93EC014A815B818C819D8160E070E025
:108A90000E94AA834A815B8188819981489F9001C5
:108AA000499F300D589F300D11248E819F8160E0C9
:108AB00070E0A9010E94AA83DF91CF910895FC0183
:108AC0008281938120E030E019C0A481B581A20F9A
:108AD000B31F4C91442381F481E08C9340815181F8
:108AE000249FC001259F900D349F900D1124268155
:108AF0003781280F391F07C02F5F3F4F28173907CD
:108B000020F320E030E0C9010895FC01268137817F
:108B10004281538180E090E018C02617370781F426
:108B2000A481B581A80FB91F2C91121614F42150FD
:108B30002C930480F581E02DE80FF91F80810895C2
:108B4000A081B1812A0F3B1F01968417950728F356
:108B50008FEF0895FC01CB012681378162177307DF
:108B600090F0A081B18162817381A69FA001A79F2F
:108B7000500DB69F500D1124420F531F21E030E0DD
:108B80008417950710F020E030E0C9010895FC013A
:108B9000118210820895FC01808191810895FB016A
:108BA00020813181FC01318320830895FC012081E3
:108BB00031812115310511F407C09C01F901808133
:108BC00091810097D1F702C020E030E0C9010895FB
:108BD000CF93DF93DC012D913C9111972115310545
:108BE000A9F0F90180819181009729F411961C92D6
:108BF0001E920EC0F90120813181D9018D919C9185
:108C000011970097B9F71182108202C020E030E07E
:108C1000C901DF91CF910895DC01ED91FC9111978D
:108C2000309729F08081918111969C938E93CF018A
:108C30000895CF93DF93FC01A081B1811097D9F003
:108C4000C0E0D0E016C0A617B70771F48D919C91D3
:108C50001197209719F49183808302C099838883A8
:108C600011961C921E9207C0ED0198818981A92F4F
:108C7000B82F109741F7DF91CF9108950F931F936D
:108C8000CF93DF938C01EB010E941946F80180819C
:108C9000918199838883D183C083DF91CF911F9184
:108CA0000F910895EF92FF920F931F93CF93DF934D
:108CB000EC017B010E941946F70111821082CE015E
:108CC0000E94D645FC01009719F4E882F98202C09F
:108CD000F182E082DF91CF911F910F91FF90EF9091
:108CE0000895DC01ED91FC91119720E030E005C082
:108CF0002F5F3F4F0190F081E02D3097C9F7C901F8
:108D00000895FB01309721F4BA010E943E46089570
:108D1000DA018081918111969C938E9351834083D7
:108D20000895009721F0FC012081318102C020E0EC
:108D300030E0C901089580910A1190910B110097BC
:108D400029F410920D1110920C1108950E944756AB
:108D5000E0910A11F0910B11228133814081518100
:108D6000240F351F281B390B0CC0428153816081B1
:108D70007181460F571F481B590B4217530708F4C0
:108D80009A010480F581E02D309779F7280F391F7B
:108D900030930D1120930C1108958DEB96E00E94F5
:108DA00029450895CF92DF92EF92FF920F931F9380
:108DB000CF93DF937C01FC0180819181009729F0A2
:108DC0008A35910509F06EC00BC010920B111092FC
:108DD0000A118AE590E0F7019183808381E066C003
:108DE000673849F5CA01E0910A11F0910B1103C0EF
:108DF0000480F581E02D309741F3268137812817D3
:108E00003907B1F3E0930A11F0930B110FC01696D6
:108E10002D913C9117972817390739F414962D9105
:108E20003C91159735832483DF01FD01A481B58131
:108E3000109769F7CECF623861F6C0910A11D091D0
:108E40000B1100E010E02BC0CE010E94AA65009734
:108E5000F1F08E819F8168E8AE010E94D4440097B2
:108E6000A1F41F821E828C819D810115110521F0C4
:108E7000F8019583848304C090930B1180930A11A9
:108E80001D821C820E949B46D8CF0E94CD468E0137
:108E90009C818D81C92EE6016E01D82EE6012097B6
:108EA00099F697CFF7011182108283E0DF91CF917D
:108EB0001F910F91FF90EF90DF90CF900895CF9387
:108EC000DF93EC010E94CD468E819F81009769F06F
:108ED000E0910A11F0910B1106C0EC17FD07A9F003
:108EE0000480F581E02D3097C1F780915C1090915E
:108EF0005D109F838E8380910A1190910B119D8349
:108F00008C83D0930B11C0930A110E949B46DF9172
:108F1000CF910895CF93DF93EC010E948A65CE0133
:108F20000E945F47DF91CF910895CF93DF93EC01CB
:108F30000E949665CE010E945F47DF91CF91089510
:108F4000CF93DF93EC010E94A065CE010E945F47A2
:108F5000DF91CF910895FC0180819181860F971F49
:108F6000918380830E949B46089521E030E0FC01BC
:108F700086819781009711F020E030E0C9010895C3
:108F8000FC012281338180819181280F391FC90121
:108F90000895FC0180819181089521E030E0809165
:108FA0000A1190910B11009711F420E030E0C901F3
:108FB000089580910A1190910B11009729F020914A
:108FC0000C1130910D1102C020E030E0C90108956C
:108FD000CF93DF93EC01E0910A11F0910B118E1702
:108FE0009F0741F48C819D8190930B1180930A110E
:108FF00014C0FC01309731F0848195818C179D0756
:10900000C1F707C01D821C821F821E82DF91CF9193
:1090100008958C819D81958384830E949B46F2CF25
:10902000CF92DF92EF92FF920F931F93CF93DF9334
:109030008C017A01FC0180819181009729F08B34A9
:10904000910509F051C01EC08FE091E10E94CB450F
:10905000C82EE6017E01F92EE70109C06C817D81F1
:10906000CE0102960E948A470990D881C02D209790
:10907000A9F781E080930E118BE490E0F8019183D1
:10908000808337C06838A9F58FE091E10E94CB4515
:10909000C82EE6016E01D92EE60123C0CE0102964C
:1090A000E816F906D9F48FE091E1BE010E94194655
:1090B000E0905C10F0905D108A859B8590935D1028
:1090C00080935C10EC85FD85309719F08E859F8527
:1090D0000995F0925D10E0925C10CECF0990D88196
:1090E000C02D2097D9F6C8CFF8011182108283E0F5
:1090F00001C081E0DF91CF911F910F91FF90EF9020
:10910000DF90CF90089510920E118FE091E10E94B0
:10911000C74586ED96E060E070E00E940645089540
:109120000F931F93CF93DF93EC0100915C1010918C
:109130005D101B870A875D874C873F872E8780914C
:109140000E11882379F086ED96E090935D10809360
:109150005C10CE0102960E948A4710935D10009326
:109160005C1002C07D836C838FE091E1BE010E94A0
:1091700019468FE091E1BE010E945246DF91CF91E6
:109180001F910F9108950F931F93CF93DF93EC01DD
:1091900080910E11882391F000915C1010915D1068
:1091A00086ED96E090935D1080935C10CE01029660
:1091B0000E94954710935D1000935C108FE091E141
:1091C000BE010E9419468FE091E1BE010E94524605
:1091D000DF91CF911F910F9108950F931F93CF931C
:1091E000DF93EC0180910E11882391F000915C10C7
:1091F00010915D1086ED96E090935D1080935C1069
:10920000CE0102960E94A04710935D1000935C105F
:109210008FE091E1BE010E9419468FE091E1BE010D
:109220000E945246DF91CF911F910F910895CF93E5
:10923000DF93EC0180910E11882329F0CE01029674
:109240000E94E84704C01F821E82198618868FE09C
:1092500091E1BE010E941946DF91CF910895CF930D
:10926000DF93EC0180910E11882331F0CE0102963C
:109270000E94B5479C0114C08FE091E10E94CB454C
:10928000E82FF92F06C0EC17FD0741F00190F0819F
:10929000E02D3097C1F721E030E002C020E030E05F
:1092A000C901DF91CF9108950F931F930091BD26BF
:1092B0001091BE260E9474562DB73EB722553040FD
:1092C0000FB6F8943EBF0FBE2DBFEDB7FEB7319677
:1092D0002EE43DE0ADB7BEB712963C932E931197A6
:1092E0000283138214831582668377838087918734
:1092F0008091B0289091B128A091B228B091B32864
:1093000082879387A487B5878091B4289091B528E8
:10931000A091B628B091B72886879787A08BB18B8C
:109320008091B8289091B928A091BA28B091BB2813
:10933000828B938BA48BB58B8091BC289091BD2898
:10934000A091BE28B091BF28868B978BA08FB18F3C
:109350008091C0289091C128A091C228B091C328C3
:10936000828F938FA48FB58F8091C4289091C52848
:10937000A091C628B091C728868F978FA0A3B1A3CC
:109380008091C8289091C928A091CA28B091CB2873
:1093900082A393A3A4A3B5A38091CC289091CD28B8
:1093A000A091CE28B091CF2886A397A3A0A7B1A75C
:1093B0008091D0289091D128A091D228B091D32823
:1093C00082A793A7A4A7B5A78091D4289091D52868
:1093D000A091D628B091D72886A797A7A0ABB1AB0C
:1093E0008091D8289091D928A091DA28B091DB28D3
:1093F00082AB93ABA4ABB5AB8091DC289091DD2818
:10940000A091DE28B091DF2886AB97ABA0AFB1AFBB
:109410008091E0289091E128A091E228B091E32882
:1094200082AF93AFA4AFB5AFEDB7FEB7FF96809113
:10943000E4289091E528A091E628B091E728808360
:109440009183A283B383EDB7FEB7ED5BFF4F8091AD
:10945000E8289091E928A091EA28B091EB28808330
:109460009183A283B383EDB7FEB7E95BFF4F809191
:10947000EC289091ED28A091EE28B091EF28808300
:109480009183A283B383EDB7FEB7E55BFF4F809175
:10949000F0289091F128A091F228B091F3288083D0
:1094A0009183A283B383EDB7FEB7E15BFF4F809159
:1094B000F4289091F528A091F628B091F7288083A0
:1094C0009183A283B3830E9441840091BD261091B1
:1094D000BE262DB73EB72E5A3F4F0FB6F8943EBF6B
:1094E0000FBE2DBF0E947456ADB7BEB7D2970FB650
:1094F000F894BEBF0FBEADBFEDB7FEB731962FEDEE
:109500003CE012963C932E931197028313821483AE
:10951000158266837783808791878091F828909160
:10952000F928A091FA28B091FB2882879387A48715
:10953000B5878091FC289091FD28A091FE28B091DC
:10954000FF2886879787A08BB18B80910029909107
:109550000129A0910229B0910329828B938BA48BBE
:10956000B58B8091042990910529A0910629B0918D
:109570000729868B978BA08FB18F809108299091B6
:109580000929A0910A29B0910B29828F938FA48F6A
:10959000B58F80910C2990910D29A0910E29B09141
:1095A0000F29868F978FA0A3B1A380911029909146
:1095B0001129A0911229B091132982A393A3A4A3E6
:1095C000B5A38091142990911529A0911629B091E5
:1095D000172986A397A3A0A7B1A7809120299091CE
:1095E0002129A0912229B091232982A793A7A4A77A
:1095F000B5A78091242990912529A0912629B09181
:10960000272986A797A7A0ABB1AB0E9441842DB7AD
:109610003EB72E5C3F4F0FB6F8943EBF0FBE2DBF36
:109620001F910F91089580E3809311110895EF9297
:10963000FF92CF93DF932091111130E0C0E3D0E08F
:10964000C21BD30B2A5E3E4EB901AE010E94A1831C
:10965000CE01DF91CF91FF90EF900895AF92BF922E
:10966000CF92DF92EF92FF920F931F93CF93DF93EE
:109670007C01C0901211D09013112091111130E093
:109680008601005D1F4F021B130B01381105E0F42A
:10969000C0E3D0E0C21BD30B2A5E3E4EB901AE013F
:1096A0000E94A183CE0DDF1D209114113091151160
:1096B0008091C8119091C911280F391FCE01B901AD
:1096C000A6010E94A18302C000E010E0C801DF9162
:1096D000CF911F910F91FF90EF90DF90CF90BF90AF
:1096E000AF90089590911111980F909311110895D2
:1096F00040911211509113119C014817590798F08D
:109700008091C8119091C911820F931F9093C91134
:109710008093C811421B530B5093131140931211A5
:1097200021E030E002C020E030E0C90108959093CC
:1097300013118093121108952091C8113091C9110D
:109740002A5B3E4EC90108952091111130E02A5E36
:109750003E4EC901089521E030E0809114119091AE
:10976000151141E18634940711F420E030E0C9017D
:1097700008950E94AB4B009771F026E431E16091AF
:109780001411709115114091121150911311C901CA
:109790000E94A1830895A091C811B091C91110979A
:1097A000B9F02091121130911311205D3F4FAA5B47
:1097B000BE4EE6E4F1E180E390E003C04D914193B9
:1097C000019682179307D4F31092C9111092C81111
:1097D000089580911411909115110895809112119E
:1097E0009091131108959091111180E3891B0895B0
:1097F00080E390911111891B209112113091131166
:10980000280F311DC90108951F93CF93DF93EC01F9
:1098100010911111812F90E08C179D076CF00E9420
:10982000F84B8C0F9D1F8138910530F41C1B109351
:10983000111121E030E002C020E030E0C901DF91E9
:10984000CF911F910895CF93DF93E7ECF6E2119249
:10985000119286E2E73FF807D1F7C0E0D0E0CE01F1
:10986000880F991F8154994D65EA76E00E949842CD
:109870002196C430D10599F7DF91CF9108951092C8
:10988000C9111092C811109213111092121180E395
:109890008093111186E491E1909315118093141136
:1098A0000E94234C08950F931F93CF93DF93EC01F5
:1098B0008B010E943F4CD0931511C093141110934B
:1098C000131100931211DF91CF911F910F91089501
:1098D000CF92DF92EF92FF920F931F93DF93CF937C
:1098E00000D0CDB7DEB78C0169837A830E943F4CEC
:1098F00069817A81C62ED72E21E8C216D10418F0CC
:1099000030E8C32ED12C8091141190911511B8011B
:10991000A6010E94A183D0921311C0921211C60118
:109920000F900F90CF91DF911F910F91FF90EF90CB
:10993000DF90CF900895282F392FD901E7ECF6E278
:1099400080E301900D928150E1F7862F972FDC0183
:10995000EFEBF6E288E001900D928150E1F7089577
:10996000E7ECF6E2282F392FD90180E30D90019220
:109970008150E1F7AFEBB6E2862F972FFC0188E02C
:1099800001900D928150E1F70895E82FF0E0EE0F7D
:10999000FF1FE953F94D7183608381E090E00895E2
:1099A000E82FF0E0EE0FFF1FE953F94D8081918120
:1099B000089590E0880F991F8157994D0E94984211
:1099C00081E090E00895282F30E0220F331F2157C7
:1099D000394DC90108958115910511F00197F1F7ED
:1099E0000895E091FA26F091FB2690818091F92666
:1099F00089230895E091F726F091F82680819091CF
:109A0000F926892B8083E091FC26F091FD26808148
:109A10009091F926892B80830895E091F726F091A3
:109A2000F82690818091F926809589238083E091A2
:109A3000FC26F091FD2690818091F926809589235E
:109A400080830895FF920F931F93E091F726F09182
:109A5000F82690818091F926809589238083E09172
:109A6000FC26F091FD2680819091F926892B808338
:109A70008FEB93E00E94EB4CFFB6F894E091FC264C
:109A8000F091FD2690818091F9268095892380832D
:109A900083E890E00E94EB4CE091FA26F091FB26DF
:109AA00000811091F926FFBE78948BE393E00E9429
:109AB000EB4CE091FA26F091FB2680819091F926FB
:109AC000892319F0802F812301C081E01F910F911C
:109AD000FF9008955093FD264093FC267093F8263E
:109AE0006093F7269093FB268093FA2681E090E01E
:109AF00002C0880F991F2A95E2F78093F9260E94E9
:109B0000224D08950F931F93182F0FB7F894E091EB
:109B1000FC26F091FD2680819091F926892B808387
:109B200083E090E00E94EB4C112351F0E091FC2681
:109B3000F091FD2690818091F9268095892380837C
:109B400087E190E00E94EB4CE091FA26F091FB2631
:109B500080819091F926892309F410E089E590E04D
:109B60000E94EB4CE091FC26F091FD2690818091C3
:109B7000F9268095892380830FBF8BE390E00E94B4
:109B8000EB4C812F1F910F9108950F931F93182F66
:109B900008E0812F81700E94824D16958111106816
:109BA0000150B9F7812F1F910F9108958FEF0E94F7
:109BB000C54D0895DF92EF92FF920F931F93CF93BD
:109BC000DF93182FEB010E94224D882389F580EF47
:109BD0000E94C54DEE2400E498EFD92ED00E81E00E
:109BE0000E94824DF82E81E00E94824D882319F058
:109BF000FF2069F020C0FF2051F4011728F0888170
:109C000080FF05C0101719F0E02EFF24F3948F2D6C
:109C10000E94824D888186958883FF2011F080689C
:109C2000888301500D15D9F6002339F02196D4CF41
:109C3000EE24EA9402C08EEFE82E8E2DDF91CF91B4
:109C40001F910F91FF90EF90DF9008950F931F9356
:109C5000CF93DF93182FEB010E94224D209751F0F4
:109C600085E50E94C54D08E089910E94C54D0150CF
:109C7000D9F703C08CEC0E94C54D812F0E94C54DC1
:109C8000DF91CF911F910F9108950F931F93CF9361
:109C9000DF93FB01DA01E801408150E0718160E06F
:109CA000462B572B803171F4BA016E7F13E0660F9B
:109CB000771F1A95E1F796814CE050E0491B510956
:109CC000460F571F57FF06C091E09C935095419552
:109CD0005F4F01C01C92883289F4848190E0BC01FE
:109CE000607670706036710549F086FF02C04E7F65
:109CF00005C085FF02C04C7F01C0487FCA0154E007
:109D0000969587955A95E1F7F90180834F704883BE
:109D100080E0DF91CF911F910F9108950F931F93D2
:109D2000CF93DF938C01EB01F8018081BE010E948B
:109D3000DA4DF801808381508D3F28F48881883284
:109D400011F0803189F7DF91CF911F910F91089524
:109D50001F93CF93DF93EC010E94224D84EBBE0151
:109D60000E94264E81E00E94824D182F0E94224DB3
:109D700081E0112309F480E0DF91CF911F910895D4
:109D80001F93CF93DF93182FEB010E94224D0E9467
:109D9000F14C882349F084E4BE010E94264E113024
:109DA00029F00E94FA4C02C082E001C080E0DF91FD
:109DB000CF911F9108956F927F928F929F92AF9251
:109DC000BF92CF92DF92EF92FF920F931F93DF9398
:109DD000CF93CDB7DEB729970FB6F894DEBF0FBE8D
:109DE000CDBF7C014B013A0159010E94224D8EEBFF
:109DF000B7010E94264E8E010F5F1F4F8AE0C82ECA
:109E0000D12CCC0EDD1E0E94D64DF80181938F011E
:109E1000EC15FD05C1F78E010F5F1F4FC80169E00A
:109E200070E00E945B6A882351F4F7018081B801D9
:109E3000A401930185010E94454E80E001C083E0AA
:109E400029960FB6F894DEBF0FBECDBFCF91DF913C
:109E50001F910F91FF90EF90DF90CF90BF90AF9048
:109E60009F908F907F906F9008957F928F929F9296
:109E7000AF92BF92CF92DF92EF92FF920F931F9318
:109E8000DF93CF93CDB7DEB729970FB6F894DEBF37
:109E90000FBECDBF782E5B014A0179018EEB60E0E9
:109EA00070E00E94264E8E010F5F1F4F9AE0C92E70
:109EB000D12CCC0EDD1E0E94D64DF80181938F016E
:109EC000EC15FD05C1F78E010F5F1F4FC80169E05A
:109ED00070E00E945B6A882349F4872DB801A501D0
:109EE000940187010E94454E80E001C083E02996DD
:109EF0000FB6F894DEBF0FBECDBFCF91DF911F919B
:109F00000F91FF90EF90DF90CF90BF90AF909F9018
:109F10008F907F9008950F931F93DF93CF93CDB7CA
:109F2000DEB728970FB6F894DEBF0FBECDBF182F4F
:109F3000062FDE011196E8EEF6E088E001900D9222
:109F40008150E1F7242F332727FD309541E752E078
:109F5000249FC001259F900D349F900D112464E62D
:109F600070E00E94667FAB0164E6069FB001112499
:109F7000460F571FFE013196CE010996619170E0A0
:109F80002617370719F44F5F5F4F03C0E817F9072B
:109F9000A9F7112319F0509541955F4FCA012896F2
:109FA0000FB6F894DEBF0FBECDBFCF91DF911F91EA
:109FB0000F9108950F931F93DF93CF93CDB7DEB723
:109FC0002B970FB6F894DEBF0FBECDBF182F092F09
:109FD000885F612F792F0E94C04E882309F049C005
:109FE00066E471E48FE090E00E944750812F902F4B
:109FF000BE016F5F7F4FAE014E5F5F4F9E012D5FD1
:10A000003F4F0E94DB4E8823A1F5DE011496E0EE5F
:10A01000F6E088E001900D928150E1F74B81642FCA
:10A0200070E021E732E0629FC001639F900D729F54
:10A03000900D112464E670E00E94667F9A8184E6A8
:10A04000989FC0011124680F791FFE013496CE013C
:10A050000C962191421719F46F5F7F4F03C0E817E8
:10A06000F907B9F78981882331F0709561957F4FA1
:10A0700002C064E371E2CB012B960FB6F894DEBF09
:10A080000FBECDBFCF91DF911F910F910895DC01DD
:10A09000CB0181159105A105B10529F081509040B2
:10A0A000A040B040D9F708951092B90080E28093A3
:10A0B000B800089594EA9093BC0020EA36E841E0A5
:10A0C00050E005C02150304040405040F1F09091A8
:10A0D000BC0097FFF7CF1DC09031B9F48093BB004F
:10A0E00084E88093BC0080EA96E8A1E0B0E004C078
:10A0F0000197A109B10959F02091BC0027FFF8CFC1
:10A100000EC081E0903421F40FC081E0089581E019
:10A1100008959091B900987F9830F1F6DFCF909133
:10A12000B900987F983169F780E0089544EA34E8EF
:10A1300024E94093BC009091BC0097FFFCCF909124
:10A14000B900987F983011F0903199F78093BB0057
:10A150003093BC009091BC0097FFFCCF9091B90068
:10A16000987F903211F0983539F42093BC0090918B
:10A17000BC0094FDFCCFDDCF08950E945A50089595
:10A1800084E98093BC008091BC0084FDFCCF0895DD
:10A190008093BB0084E88093BC008091BC0087FF63
:10A1A000FCCF9091B900987F81E0983209F480E06B
:10A1B000089584EC8093BC008091BC0087FFFCCFA5
:10A1C0008091BB00089584E88093BC008091BC001E
:10A1D00087FFFCCF8091BB000895E82FF92F80E125
:10A1E000919190933F018150D9F780913C018F7DEF
:10A1F00080933C0180913C01877F80933C01862FB6
:10A20000972FFC0180E1919190933E018150D9F705
:10A2100080913C01806880933C0180913D0180FFEA
:10A22000FCCF4051504080913C01806280933C01C2
:10A2300080913C01877F80933C0114C0862F972F2B
:10A24000FC0180E1919190933E018150D9F780917A
:10A250003C01806880933C0180913D0180FFFCCFF0
:10A2600040515040141615064CF3822F932FFC01D9
:10A2700080E190913E0191938150D9F781E090E087
:10A2800008950F931F93CF93DF938C018CE70E9467
:10A2900096508CE70E94C850C0E0D0E0F801819150
:10A2A0008F010E94C8502196C031D105B9F70E9494
:10A2B000C050DF91CF911F910F910895813039F4F3
:10A2C0008CE790E060E070E040E050E006C08CE792
:10A2D00090E060E070E040EC50E00E947F12089552
:10A2E000813039F48CE790E060E070E04EE050E0BF
:10A2F00006C08CE790E060E070E048E050E00E942B
:10A300007F1208958CE790E060E070E041E050E05B
:10A310000E947F126AE67AE080E090E00E94475057
:10A3200008958CE790E060E070E048E350E00E9420
:10A330007F128CE790E060E070E049E350E00E941B
:10A340007F128CE790E060E070E044E150E00E9412
:10A350007F128CE790E060E070E048E750E00E94F8
:10A360007F128CE790E060E070E04EE550E00E94E4
:10A370007F128CE790E060E070E04DE650E00E94D4
:10A380007F126CE17AE186E090E00E9447508CE712
:10A3900090E060E070E04CE050E00E947F128CE7BB
:10A3A00090E060E070E041E050E00E947F128CE7B6
:10A3B00090E060E070E046E050E00E947F126AE6C4
:10A3C0007AE080E090E00E9447500895DF93CF93B9
:10A3D000CDB7DEB7A2970FB6F894DEBF0FBECDBFE4
:10A3E000DE011196E0EFF6E081E101900D928150DF
:10A3F000E1F7DE015296E1E0F7E081E101900D9294
:10A400008150E1F70E949151CE0101960E94415185
:10A4100082E00E945E516AE67AE080E090E00E946D
:10A420004750CE0142960E94415160E17EEA88E2A7
:10A4300090E00E94475080E00E94705160E17EEA07
:10A4400088E290E00E94475081E00E947051A296FD
:10A450000FB6F894DEBF0FBECDBFCF91DF91089548
:10A46000DF92EF92FF920F931F93DF93CF9300D071
:10A470000F92CDB7DEB7F82E042F122F213031F016
:10A48000223031F0243031F0283031F080E005C046
:10A4900081E003C082E001C083E00C3059F00E304F
:10A4A00011F4846007C0003111F4886003C00231E8
:10A4B00009F48C60613059F0623011F4806207C099
:10A4C000633011F4806403C0643009F48066682F3F
:10A4D00060688F2D90E070E0AE014F5F5F4F23E02A
:10A4E00030E00E94971269E07AE180E090E00E94FB
:10A4F000475081E0F82A8F2D0E945A500E94D9506F
:10A5000089830E94D9508A83023119F40E94D9505C
:10A510008B830E94D95087FDF1CF0E94E3500E94A7
:10A52000C05069E07AE180E090E00E9447508F2DB2
:10A530000E945A500E94D95089830E94D9508A8320
:10A54000023119F40E94D9508B830E94D95029817D
:10A55000023181F5622F70E080E090E03B814A811A
:10A5600021FF12C0CB0177276627630F711D811D64
:10A57000911D342F20E040E050E0620F731F841FD4
:10A58000951F8C6F9F6F0FC0CB0177276627630FD6
:10A59000711D811D911D342F20E040E050E0620FBD
:10A5A000731F841F951F0E94B87C20E83FEF4FEF78
:10A5B00057E41FC0722F60E08A81680F711D8827E1
:10A5C00077FD8095982F0E94B87C0C3029F420E00C
:10A5D00030EE4FEF54E40DC00E3029F420E038EF98
:10A5E0004FEF55E406C0003131F420E03EEF4FEF6D
:10A5F00056E40E944E7C2FE632E143E050E40E9494
:10A60000947DD62EE72EF82E092F612F70E0882733
:10A6100077FD8095982F0E94B87C9B01AC016D2D31
:10A620007E2D8F2D902F0E944E7C0F900F900F90BB
:10A63000CF91DF911F910F91FF90EF90DF900895E0
:10A64000E6E4F1E0808120819081308182958695D9
:10A650008695837022952F70822B832B92959F7005
:10A66000892B0895DF92EF92FF920F931F93DF9350
:10A67000CF9300D0CDB7DEB780E06CE046E00E941B
:10A68000085789E18093C4001092C50082E080934E
:10A69000C00080E00E94B2570E94375684B784B74A
:10A6A00084B784B784B7EEE7FFE222E432E4318373
:10A6B00020833A968DB79EB70A97E817F907B8F343
:10A6C00000D000D08BE99EE0ADB7BEB712969C9348
:10A6D0008E93119782E197E014969C938E93139733
:10A6E0000E9441840F900F900F900F900E9474660B
:10A6F0000E9452448DEB96E060E070E00E940645B7
:10A700000E948348E0915D07F0915E0709950E94E1
:10A71000205390E00E94B266CE0101960E946555DA
:10A72000882359F000D08BE79EE0EDB7FEB7928307
:10A7300081830E9441840F900F908E010F5F1F4F05
:10A74000C8010E94B3420E946F557C010E9474555B
:10A75000BC01C701A8010E94BF5A0E94CD540E94AB
:10A76000A45A0E9479550E942C5C00D08EE69EE08F
:10A77000ADB7BEB712969C938E9311970E944184F9
:10A7800000D0EDB7FEB731960AE61EE0ADB7BEB712
:10A7900012961C930E9311978A81828313820E94D2
:10A7A0004184EDB7FEB73196ADB7BEB712961C9394
:10A7B0000E9311978981828313820E9441840F90A6
:10A7C0000F9088E69EE0EDB7FEB7928381830E94EA
:10A7D00041840F900F900E94B866E091E007F091DD
:10A7E000E1070995E091C707F091C8070995E09145
:10A7F0008907F0918A070995E090C507F090C60790
:10A800000091DE071091DF070E94A15AD82E0E9406
:10A81000345C2DB73EB72A5030400FB6F8943EBF97
:10A820000FBE2DBFEDB7FEB731962DE43EE0ADB7BC
:10A83000BEB712963C932E931197F382E282158352
:10A840000483D6821782808711860E944184E0911A
:10A85000EA07F091EB072DB73EB7265F3F4F0FB6E3
:10A86000F8943EBF0FBE2DBF3097D1F00995BC01C3
:10A8700000D000D08AE39EE0ADB7BEB712969C939D
:10A880008E93119780E890E00E94527FEDB7FEB75B
:10A89000748363830E9441840F900F900F900F90F8
:10A8A00000D088E39EE0ADB7BEB712969C938E931E
:10A8B00011970E9441840F900F9089E098E060E02A
:10A8C00070E00E9406458BE896E00E945E6500D02D
:10A8D00080E39EE0EDB7FEB7928381830E944184BE
:10A8E0000F900F900F900F90CF91DF911F910F91CC
:10A8F000FF90EF90DF900895EF92FF920F931F93D8
:10A9000080E880936100109261000E9432530E949F
:10A9100062440E94D3578091FE269091FF260097B3
:10A9200029F001979093FF268093FE26E090002760
:10A93000F090012700910227109103270E9474567E
:10A94000E616F7060807190711F30E94745660937C
:10A950000027709301278093022790930327D7CF76
:10A9600000D000D000D0EDB7FEB731962AE23EE02D
:10A97000ADB7BEB712963C932E9311979383828303
:10A98000758364830E9441848DB79EB706960FB687
:10A99000F8949EBF0FBE8DBF08950F931F93DF9352
:10A9A000CF93CDB7DEB7A2970FB6F894DEBF0FBE38
:10A9B000CDBF8EE490E00E94848589839A83982F8E
:10A9C0009B50903108F08A839A819095891709F4F9
:10A9D00070C000D086ED9EE0ADB7BEB712969C93D6
:10A9E0008E9311970E9441848E010D5F1F4F0F902F
:10A9F0000F90D80180E090E0FC01EA54F14FE4911F
:10AA0000ED93019688309105B9F7F894CE0103963D
:10AA10006CE270E048E050E00E948A85D80180E056
:10AA200090E0FC01E254F14FE491ED9301968E30F9
:10AA30009105B9F7CE01039664E370E04EE050E073
:10AA40000E948A8580E090E0FC01E453F14FE4919C
:10AA5000D801ED938D0101968A309105A9F7CE01B9
:10AA6000039662E470E04AE050E00E948A8580E547
:10AA700090E06DEC7BEA0E94A28582E590E060E0C8
:10AA800070E00E94A28584E590E060E00E949485D9
:10AA90008CE490E060E070E00E94A2858AE1898306
:10AAA00085EE8A8369817A818EE490E00E94A28596
:10AAB00078948981A2960FB6F894DEBF0FBECDBF01
:10AAC000CF91DF911F910F910895F8946CE270E09F
:10AAD00042E050E00E946C85789480E0089580E523
:10AAE00090E00E948485089582E590E00E9484852C
:10AAF000089584E590E00E947C85089520910C27BC
:10AB000030910D2740910E2750910F2790E0A0E043
:10AB1000B0E0280F391F4A1F5B1F20930C2730938A
:10AB20000D2740930E2750930F272091082730912F
:10AB3000092740910A2750910B27280F391F4A1FD8
:10AB40005B1F209308273093092740930A275093CF
:10AB50000B272091AC282223A1F0209104273091CB
:10AB600005274091062750910727280F391F4A1FB4
:10AB70005B1F2093042730930527409306275093AB
:10AB8000072708951F920F920FB60F920BB60F92E0
:10AB900011242F933F934F935F936F937F938F93E2
:10ABA0009F93AF93BF93EF93FF938091CA119091BE
:10ABB000CB1101969093CB118093CA118091CC1147
:10ABC0008F5F8093CC118091CC118038A9F41092C2
:10ABD000CC1180910C2790910D27A0910E27B09158
:10ABE0000F270196A11DB11D80930C2790930D276F
:10ABF000A0930E27B0930F278091AC288823F1F003
:10AC00008091CD118F5F8093CD118091CD118038CF
:10AC1000A9F41092CD118091042790910527A0915D
:10AC20000627B09107270196A11DB11D8093042727
:10AC300090930527A0930627B09307270E94CD473E
:10AC4000009711F00E94CD46FF91EF91BF91AF9117
:10AC50009F918F917F916F915F914F913F912F9134
:10AC60000F900BBE0F900FBE0F901F901895F89489
:10AC70001092B60016BC83EF87BD82E084BD94E0DD
:10AC800095BD95B395BB80936E00789408952091FF
:10AC9000CA113091CB118091CA119091CB11281714
:10ACA0003907A9F7C901089507C022E330E0000081
:10ACB00021503040E1F701970097B9F708950F93BD
:10ACC0001F93CF93DF938C010E944756EC010E94A3
:10ACD00047568C1B9D0B80179107C8F3DF91CF91CE
:10ACE0001F910F910895089520910C2730910D2701
:10ACF00040910E2750910F2780910C2790910D279E
:10AD0000A0910E27B0910F27281739074A075B0734
:10AD100059F7B901CA0108951F920F920FB60F9209
:10AD20001124109236070F900FBE0F901F901895A8
:10AD30001F920F920FB60F920BB60F9211242F9302
:10AD40003F934F935F936F937F938F939F93AF93B3
:10AD5000BF93EF93FF93E0912C07F0912D07808133
:10AD6000E0913707F0913807309709F00995FF9186
:10AD7000EF91BF91AF919F918F917F916F915F9173
:10AD80004F913F912F910F900BBE0F900FBE0F90E0
:10AD90001F9018951F920F920FB60F9211241092C8
:10ADA00043070F900FBE0F901F9018951F920F92A0
:10ADB0000FB60F920BB60F9211242F933F934F9320
:10ADC0005F936F937F938F939F93AF93BF93EF9313
:10ADD000FF93E0913907F0913A078081E0914407B1
:10ADE000F0914507309709F00995FF91EF91BF91D8
:10ADF000AF919F918F917F916F915F914F913F9113
:10AE00002F910F900BBE0F900FBE0F901F901895B3
:10AE100090E02DE030E0829FF001839FF00D929F43
:10AE2000F00D1124E45DF84FA281B3811C92A4813E
:10AE3000B5816C93A681B78188ED8C93A085B1858F
:10AE40004C93128614861386089590E02DE030E02E
:10AE5000829FF001839FF00D929FF00D1124E45D1D
:10AE6000F84F81E08287A081B1816C933A9680810E
:10AE70008823E9F708951F93182F8A3031F48091C1
:10AE8000CE116DE00E94255702C08D3029F08091CF
:10AE9000CE11612F0E94255780E090E01F91089508
:10AEA000EF92FF921F93CF93DF93182FE62EE701C7
:10AEB0007E01F72EE7010CC08A3021F4812F6DE06E
:10AEC0000E94255769916D3019F0812F0E942557F6
:10AED0008881882389F7DF91CF911F91FF90EF90B0
:10AEE00008950F931F93DF93CF93CDB7DEB7FE0185
:10AEF0003A960FEC11E1C80160E470E0488559858D
:10AF00009F010E94D6848F81B8010E945057CF9133
:10AF1000DF911F910F9108951F93CF93DF93182F07
:10AF2000EB0104C0812F0E9425572196FE016491F8
:10AF30006623C1F7DF91CF911F91089590E02DE036
:10AF400030E0829FF001839FF00D929FF00D11245D
:10AF5000E45DF84F748763870895682F80E00E944E
:10AF6000255708958093CE118EE197E09093792F25
:10AF70008093782F089584B7877F84BF88E10FB6C8
:10AF8000F89480936000109260000FBE08952FE047
:10AF900088E190E00FB6F894A895809360000FBE0A
:10AFA000209360000895A895089588E10FB6F8945D
:10AFB00080936000109260000FBE0895F89428E01E
:10AFC00088E190E00FB6F894A895809360000FBEDA
:10AFD00020936000FFCF80911F2790E0FC01EE0FCF
:10AFE000FF1F9695982F882797958795E80FF91F4B
:10AFF000E05EF84D10820895809117278091172701
:10B0000090E008958091390181FD0CC081E491E0C8
:10B010006FE140E00E94D55D813039F021E030E001
:10B02000813129F020E030E002C021E030E0C901A8
:10B0300008958091390181FD12C081E491E06FE1B2
:10B0400040E00E94D55D982F8151823050F09F31B1
:10B0500041F0913041F081E0923031F402C081E062
:10B06000089580E0089580E008950E94195888238B
:10B07000E1F3089581E491E06FE140E00E94D55D45
:10B080000895E9E3F1E0808180818D7F80838DE008
:10B0900090E00197F1F782E491E06FE140E023E076
:10B0A0000E94DF5D83E090E00197F1F708950E9430
:10B0B00035581092AC280E94415880913901826025
:10B0C0008093390180912F298823E9F180919400A0
:10B0D0009091950020914029309141298217930742
:10B0E000A0F480910C2990910D29A0910E29B09186
:10B0F0000F298C57914EAF4FBF4F80930C299093DF
:10B100000D29A0930E29B0930F298091940090915E
:10B110009500821B930BA0E0B0E020910C293091A8
:10B120000D2940910E2950910F29820F931FA41FC2
:10B13000B51F80930C2990930D29A0930E29B093ED
:10B140000F2910922F29809131298823E9F18091CC
:10B1500094009091950020914429309145298217BF
:10B160009307A0F48091142990911529A091162994
:10B17000B09117298C57914EAF4FBF4F8093142930
:10B1800090931529A0931629B093172980919400C4
:10B1900090919500821B930BA0E0B0E020911429C0
:10B1A000309115294091162950911729820F931F2C
:10B1B000A41FB51F8093142990931529A0931629D5
:10B1C000B09317291092312908958091AC288823D3
:10B1D00081F080910F12882321F40E94195888234E
:10B1E00031F481E08093921221E030E004C00E94AB
:10B1F000575820E030E0C90108950F931F93182F8E
:10B20000883049F0863039F0893029F0863119F0DC
:10B21000893109F041C08091390181FD40C00E940F
:10B2200035580E943A58082F181709F43BC01830B7
:10B2300019F40E94415829C0193141F48631A9F40A
:10B2400082E491E06FE140E029E009C0163169F441
:10B25000893159F482E491E06FE140E026E00E94F8
:10B26000DF5DE3E0F0E03197F1F782E491E06FE138
:10B2700040E0212F0E94DF5D083019F4E9E6F1E09B
:10B2800002C0E3E0F0E03197F1F70E943A588117ED
:10B2900049F023E430E008C022E430E005C024E4B3
:10B2A00030E002C020E430E0C9011F910F91089501
:10B2B0008091940090919500909345298093442922
:10B2C00021E0209331298091390181FF15C020931D
:10B2D000AB288091940090919500909341298093A0
:10B2E000402920932F29809139018D7F8093390146
:10B2F0008091AB288823E1F786E10E94FD5881E028
:10B300008093AC2808958091AC28882351F48091D3
:10B310000F12882321F081E08093911202C00E94D5
:10B32000585981E090E008951F93DF93CF930F92D7
:10B33000CDB7DEB78FB7898380910F12882331F59F
:10B34000F8948091AC28882351F08091390181FDD7
:10B350001BC00E9419588823B9F080E003C00E94E6
:10B36000835981E0909147019E3010F010E001C0B8
:10B370001FEF882311F00E94E55816FF05C0898150
:10B380008FBF21E030E004C089818FBF20E030E032
:10B39000C9010F90CF91DF911F9108958091911273
:10B3A000882321F00E945859109291128091921294
:10B3B000882321F00E9457581092921210920F1277
:10B3C0000895EF92FF92CF93DF93B82FA92FF62F16
:10B3D000E72F81E080930F122091F0283091F1281F
:10B3E0004091F2285091F3282F5F3F4F4F4F5F4F0E
:10B3F0002093F0283093F1284093F2285093F328BB
:10B40000862F8E5F87FF0CC08091A9289091AA2873
:10B4100001969093AA288093A928CFEFDFEF0BC065
:10B4200020E132E1C9016B2F7A2F4F2F5E2F0E944E
:10B43000A183C0E0D0E00E94CE59CE01DF91CF9130
:10B44000FF90EF9008959091390191FD0AC0282F47
:10B45000803108F02FE085E491E06FE040E00E9449
:10B46000DF5D08958093941208950E943A588250A7
:10B47000813130F4E82FF0E0EF58F84F80810895E3
:10B4800081E0089508958FEF80934E018CE691E05E
:10B4900060EF44E022E00E94DF5D8CE290E06EE02D
:10B4A00041E025E00E94DF5D80E880936F0180919C
:10B4B000460180936D0184E491E060E245E021E083
:10B4C0000E94DF5D0895CF93DF93CDEFD3E0CE01EF
:10B4D0000197F1F70E94CB5D109220271092A227CE
:10B4E0001092242810921F2710921E27E9E3F1E002
:10B4F00080818E7F808380818D7F80838DE090E04E
:10B500000197F1F780818160808382E491E06FE1AF
:10B5100040E023E00E94DF5D2197F1F780915D011B
:10B5200080915E010E94435A83E597E060E070E0FD
:10B530000E9406450E94585981E090E0DF91CF912A
:10B540000895809193120895DF93CF930F92CDB712
:10B55000DEB789830E94355829812093931288E4AD
:10B5600091E06FE140E00E94DF5D0F90CF91DF91AD
:10B5700008950E94A45A86E00E94FD580895809381
:10B5800062019093630160936001709361014115C2
:10B59000510531F1FA01819180936B01DA01119625
:10B5A0008C9180936A01DF011196818180936901FA
:10B5B000FD01319611968C9180936801DF011196FF
:10B5C000818180936701FD01319611968C911197CD
:10B5D00080936601818180936501828180936401FB
:10B5E000089583E597E00E94294581E0809317271D
:10B5F000809118279091192701969093192780938D
:10B60000182781E090E00895EF92FF92CF93DF93A7
:10B6100050911F27252F30E0F901EE0FFF1F3695BF
:10B62000322F222737952795E20FF31FE05EF84D62
:10B630004081442309F4CEC02091390121FDCAC0C4
:10B640002091AC28222309F4C5C047FF16C00E94F0
:10B65000EB578091E0289091E128A091E228B091E9
:10B66000E3280196A11DB11D8093E0289093E12865
:10B67000A093E228B093E328ADC04330B0F40E9419
:10B68000EB578091DC289091DD28A091DE28B091C5
:10B69000DF280196A11DB11D8093DC289093DD2841
:10B6A000A093DE28B093DF2895C0C42FD0E0229766
:10B6B0006C177D07B0F40E94EB578091D8289091C9
:10B6C000D928A091DA28B091DB280196A11DB11DDF
:10B6D0008093D8289093D928A093DA28B093DB28B8
:10B6E00079C0652F70E09B01220F331F7695762F6E
:10B6F000662777956795260F371F2F5D384DB9015F
:10B7000050E00E94A18320911F27822F90E0FC012E
:10B71000EE0FFF1F9695982F882797958795E80F2E
:10B72000F91FE056F84D808180931027822F90E01A
:10B73000FC01EE0FFF1F9695982F88279795879508
:10B74000E80FF91FE05EF84D10822F5F20931F274E
:10B75000233010F010921F2780911F2790E0FC01EA
:10B76000EE0FFF1F9695982F882797958795E80FDE
:10B77000F91FE05EF84D8081882311F00E94F15A94
:10B78000609147016093112780911627882311F05B
:10B79000681710F46093162784E070E00E94C54C8F
:10B7A0006091102783E070E00E94C54C8091F428DE
:10B7B0009091F528A091F628B091F7280196A11D47
:10B7C000B11D8093F4289093F528A093F628B093A8
:10B7D000F72802C0C0E0D0E0CE01DF91CF91FF900A
:10B7E000EF900895CF93DF93EC01888199810097C2
:10B7F00029F024E08B3F920739F505C08BEF94E0E8
:10B800009983888325C0623819F5109217270E9402
:10B810003F4C0E949C4B60E870E00E94045B18164D
:10B82000190644F40E94974BE091E407F091E50774
:10B830000995E4CF80911427909115270196909354
:10B84000152780931427DACF1982188283E001C06C
:10B8500081E0DF91CF91089591E090930F120E94C3
:10B86000235A0E94CE5908958091390181FD07C065
:10B8700085E491E06FE040E00E94D55D089580E1AD
:10B880000895CF92DF92EF92FF920F931F93CF9381
:10B89000DF93182F21E020930F120091AC288091A4
:10B8A000390181FF16C0809194009091950090938A
:10B8B00041298093402920932F292093AB28809100
:10B8C00039018D7F809339018091AB288823E1F77E
:10B8D00000E00E9435588091AC28882309F441C0CB
:10B8E000809131298823E9F12091940030919500CD
:10B8F000809144299091452928173907A0F4209177
:10B9000014293091152940911629509117292C5747
:10B91000314E4F4F5F4F2093142930931529409398
:10B920001629509317292091940030919500281BD7
:10B93000390B40E050E0C0901429D0901529E090D8
:10B940001629F09017292C0D3D1D4E1D5F1D2093CB
:10B9500014293093152940931629509317291092D2
:10B96000312989E10E94FD5886E00E94D04C009761
:10B9700051F00E94345CC82F86E00E94D04C815068
:10B980000E94235A02C0C0E0D0E0809194009091C0
:10B990009500909343298093422981E08093302938
:10B9A000F894809139018260809339018091390146
:10B9B0008D7F80933901612F6E5F80E192E10E945B
:10B9C000105E78948091A6289091A7280196909374
:10B9D000A7288093A6280E94355882E491E060EE63
:10B9E00045E00E94D55D182F86E00E94D04C00975C
:10B9F00019F08C2F0E94235A002319F00E945859E5
:10BA000002C00E945758809130298823E9F1809123
:10BA100094009091950040914229509143298417B8
:10BA20009507A0F48091102990911129A0911229D5
:10BA3000B09113298C57914EAF4FBF4F809310296F
:10BA400090931129A0931229B09313292091940067
:10BA500030919500241B350B40E050E08091102977
:10BA600090911129A0911229B0911329280F391F03
:10BA70004A1F5B1F209310293093112940931229EC
:10BA800050931329109230298091AC28882361F0BB
:10BA9000809194009091950090934529809344293A
:10BAA00081E08093312907C082E491E06FE140E0BA
:10BAB00023E00E94DF5D0E94CE591130E1F0133087
:10BAC000A9F48091E8289091E928A091EA28B09102
:10BAD000EB280196A11DB11D8093E8289093E928D9
:10BAE000A093EA28B093EB2812E00AC0153029F0A1
:10BAF000173031F404C010E003C013E001C011E0BE
:10BB0000812F90E0DF91CF911F910F91FF90EF90E7
:10BB1000DF90CF900895CF93DF93EB010E94E1591E
:10BB20009C01009731F4CE010E94415C9C0100977A
:10BB300049F08091A9289091AA2801969093AA286B
:10BB40008093A928C901DF91CF9108950F931F9386
:10BB50008091AC28882321F40E94835911E001C010
:10BB600010E00E943A58863111F0813119F40091A9
:10BB7000470109C086E491E06FE140E00E94D55D95
:10BB8000082F000F080F112311F00E94E558802F95
:10BB90001F910F9108951092961210929512EFE650
:10BBA000F0E08081806280830895FC01808186239B
:10BBB00090E002C0959587954A95E2F70895F8942C
:10BBC000FC019081862F8095892330E002C0220FEE
:10BBD000331F4A95E2F72623282B20837894089573
:10BBE000DC01119620917B01FC012083215030E083
:10BBF000A9014F575E4FE0E8F1E061916D93E417C2
:10BC0000F507D9F7FC01E058FF4F2F573E4FD901F8
:10BC10002C9120838F579F4F21E0FC0120830895B2
:10BC2000FC016093800101966350860F911DA1E88D
:10BC3000B1E021912D93E817F907D9F708951F92E4
:10BC40000F920FB60F920BB60F9211242F933F93C2
:10BC50004F935F936F937F938F939F93AF93BF9314
:10BC6000EF93FF93809147018093112720911E2726
:10BC700030E0C901880F991F3695322F222737955A
:10BC80002795820F931F805E984D0E94F05D8091F2
:10BC90001E278F5F80931E27833010F010921E277F
:10BCA0000E94F15AFF91EF91BF91AF919F918F91B7
:10BCB0007F916F915F914F913F912F910F900BBEAC
:10BCC0000F900FBE0F901F9018951F920F920FB6F6
:10BCD0000F9211240F900FBE0F901F9018951F9276
:10BCE0000F920FB60F9211240F900FBE0F901F905E
:10BCF00018951F920F920FB60F9211240F900FBE3E
:10BD00000F901F9018951F920F920FB60F9211244B
:10BD10001092AB280F900FBE0F901F9018951F9296
:10BD20000F920FB60F9211241092AB280F900FBEF6
:10BD30000F901F9018951F920F920FB60F9211241B
:10BD40008F9381E0809317278F910F900FBE0F90F4
:10BD50001F9018951F920F920FB60F9211241092F8
:10BD6000AB280F900FBE0F901F9018951F920F9247
:10BD70000FB60F9211248F939F93809195129091FB
:10BD80009612019690939612809395129F918F919F
:10BD90000F900FBE0F901F9018950F931F93CF9386
:10BDA000DF938091B4289091B528A091B628B091E6
:10BDB000B7280196A11DB11D8093B4289093B52892
:10BDC000A093B628B093B7280E947E61EC0187E962
:10BDD00092E10E94CB450BC0D8011296ED91FC91E7
:10BDE0001397309709F00995C8010E949146082FD2
:10BDF000192F0115110581F7209719F0CE010E9426
:10BE00003B43DF91CF911F910F9108950E94B86637
:10BE10000E943F4C0E94885F85EC97E09093AF288A
:10BE20008093AE280E947B6182E090E060E074E045
:10BE300040E05EE12FEF31E00E943C610895CF9237
:10BE4000DF92EF92FF920F931F93CF93DF936C01DA
:10BE5000EB018A0187E992E10E94CB450CC0D70132
:10BE60001496ED91FC911597309711F0CE0109953C
:10BE7000C7010E949146E82EF92EE114F10479F7EA
:10BE8000C601BE01A8010E944343DF91CF911F91DB
:10BE90000F91FF90EF90DF90CF900895BC0187E95C
:10BEA00092E10E9452460895BC0187E992E10E9406
:10BEB00019460895CF93DF93EC018091B0289091BB
:10BEC000B128A091B228B091B3280196A11DB11D4F
:10BED0008093B0289093B128A093B228B093B32850
:10BEE000CE010E949561009769F00E94B94BE091E4
:10BEF000C907F091CA078FE19FE5BE01099521E0CE
:10BF000030E002C020E030E0C901DF91CF91089518
:10BF100089E992E10E94C74508950F93CF93DF937B
:10BF2000EC017B836A8318865F834E8389E992E103
:10BF3000BE010E945246E0919B12F0919C123097F4
:10BF400049F04C815D818A819B81688520E030E0E9
:10BF500001E00995DF91CF910F910895BC0189E926
:10BF600092E10E94194608950F93DC0118961C92E5
:10BF70001897E0919B12F0919C12309759F012960D
:10BF80008D919C91139760E040E050E020E030E01C
:10BF900000E009950F9108950F93DC01AB01149611
:10BFA0002D913C91159781E018968C9318971596D2
:10BFB0007C936E931497E0919B12F0919C123097B2
:10BFC00039F012968D919C91139761E000E00995EC
:10BFD0000F9108950F93DC01E0919B12F0919C1258
:10BFE000309769F014962D913C91159712968D918A
:10BFF0009C91139718966C91A90101E009950F91F6
:10C000000895E0919D12F0919E12309709F00995E4
:10C01000089590939E1280939D12089590939C1280
:10C0200080939B12089589E992E10E94CB4508957F
:10C03000EF92FF920F931F93CF93DF938C01EB014D
:10C040007A0189E992E10E94CB4515C0DC01129684
:10C050002D913C9113972C173D0759F41696ED91AD
:10C06000FC911797309761F0B801AE0197010995DF
:10C0700007C00E949146282F392FC901009731F738
:10C08000DF91CF911F910F91FF90EF900895089548
:10C09000AF92BF92CF92DF92EF92FF920F931F93D6
:10C0A000DF93CF9300D0CDB7DEB75B010E949C4BEE
:10C0B000FC01008111811A8309830C30110518F4E9
:10C0C000EE24FF242EC000D000D08DE897E0EDB71D
:10C0D000FEB792838183148303830E942F840F9081
:10C0E0000F900F900F9020C00E949C4BF701EE0F15
:10C0F000FF1FEE0FFF1FE80FF91FC280D3800E94C1
:10C100009C4B0894E11CF11CF701EE0FFF1FEE0F92
:10C11000FF1FE80FF91F40815181C501B6010E9440
:10C120001860E016F10600F30F900F90CF91DF91A9
:10C130001F910F91FF90EF90DF90CF90BF90AF9045
:10C140000895CF93DF93CAEBD2E16091D012709142
:10C15000D112CE0143ED50E620E030E00E9490483D
:10C160000E94B5666091D0127091D1120E94527FE8
:10C17000BC01CE01409748EE50E620E030E00E943E
:10C180009048DF91CF9108950F93013051F4809141
:10C19000CA129091CB129093D1128093D0120E9428
:10C1A000A1600F9108958091D0129091D1122091A9
:10C1B000CE123091CF12880F991F2817390708F433
:10C1C000C9019093D1128093D0120E94A16008956A
:10C1D000EF92FF92CF93DF930E943F4C0E949C4BC3
:10C1E000E82EE7017E01F92EE701198218820E94EC
:10C1F000136026C028813981F901EE0FFF1FEE0F71
:10C20000FF1FEC0FFD1FDC0112964D915C911397FF
:10C21000538342832F5F3F4FF901EE0FFF1FEE0F55
:10C22000FF1FEC0FFD1F14964D915C9115975183E4
:10C230004083398328830E949146282F392FC901D2
:10C24000009721F0FC0120852223A1F688819981A5
:10C25000880F991F880F991F02960E94974B88811B
:10C260009981009721F08FE992E10E940E43DF91BE
:10C27000CF91FF90EF900895EF92FF920F931F934D
:10C28000CF93DF93FC018B017A01E9018FE992E101
:10C29000BF014AEA57E00E94F0421093CB1200938C
:10C2A000CA12F092CD12E092CC12D093CF12C0936A
:10C2B000CE1284EC90E60E940E60DF91CF911F9128
:10C2C0000F91FF90EF900895CF93DF93CAEBD2E1E7
:10C2D000CE010E941749CE0140970E941749CE0116
:10C2E0004B970E940B43DF91CF9108958091D0121C
:10C2F0009091D11208950E944F430895EF92FF92BA
:10C30000CF93DF93E091AE07F091AF070995EC0171
:10C31000009729F06A817B8181E00E94C54CCE01A3
:10C32000DF91CF91FF90EF9008950F931F93CF93DC
:10C33000DF938C01E091B007F091B1070995EC0112
:10C34000F8016281738181E00E94C54C21E030E0F8
:10C35000209711F420E030E0C901DF91CF911F91C7
:10C360000F910895E091B207F091B30709950895F0
:10C37000FC0120E030E004C08181280F311D32969D
:10C3800080818823C9F7C9010895FC01818190E06B
:10C39000308120E0822B932B02C0880F991F6A9571
:10C3A000E2F7892F9927FA01EC54F84F208130E009
:10C3B0008223932328E030E0241B350B02C096959E
:10C3C00087952A95E2F708956F927F928F929F92B8
:10C3D000AF92BF92CF92DF92EF92FF920F931F9393
:10C3E000CF93DF936C017B015A018901283031051D
:10C3F00044F4CB01BA01A9010E94C561F601808312
:10C4000041C0390133E0759467943A95E1F74115DD
:10C41000510521F04C01C0E0D0E016C0DB01FC0169
:10C42000C0E0D0E08D9181932196C615D705D4F355
:10C43000A801477050704115510521F1C7018C0FBB
:10C440009D1F60E070E019C0C7018C0F9D1FB501F2
:10C4500048E050E00E94C561F40181934F012196AC
:10C46000C615D7058CF3A8014770507041155105CA
:10C4700049F0C7018C0F9D1FB5010E94C561CC0D0D
:10C48000DD1D8883DF91CF911F910F91FF90EF9079
:10C49000DF90CF90BF90AF909F908F907F906F90E4
:10C4A00008954F925F926F927F928F929F92AF9278
:10C4B000BF92CF92DF92EF92FF920F931F93DF9381
:10C4C000CF9300D000D0CDB7DEB70E949C4BE82EB2
:10C4D000092F82E090E00E94784B009709F464C035
:10C4E000EE2DF02F918180E02081820F911D0E941E
:10C4F00063437C01009709F459C00E949C4B3C01A6
:10C50000F7014681242F30E02770307081E090E001
:10C510002115310511F480E090E046954695469549
:10C52000840F911D0E94784B0097F1F1F70104816F
:10C530001581CC24DD2453E0452E512C4C0E5D1E7C
:10C540004E010894811C911C2AC0F801A180BB24D3
:10C55000B60143E0759567954A95E1F7660D771D3D
:10C56000A60147705070883150F0C40195010E94B7
:10C57000E461F8018081B4010E94D94C0CC01C8296
:10C580001B82C20195010E94E4616B817C81F801EC
:10C5900080810E94C54CCA0CDB1C0E5F1F4FF80146
:10C5A0008081882391F602C0EE24FF24C7010F90FA
:10C5B0000F900F900F90CF91DF911F910F91FF90EF
:10C5C000EF90DF90CF90BF90AF909F908F907F9033
:10C5D0006F905F904F900895FC0150E080E190E0F3
:10C5E000861B970B821B930B02C0440F551F8A9525
:10C5F000E2F78081852B80838181842B818308955C
:10C600006F927F928F929F92AF92BF92CF92DF9262
:10C61000EF92FF920F931F93CF93DF938C015B01F7
:10C620006A0179012830310524F4C801FA014081FA
:10C6300056C0390163E0759467946A95E1F7A114D7
:10C64000B10421F04A01C0E0D0E021C0DA01F801D4
:10C6500080E090E02D912193019686159705D4F303
:10C6600097012770307021153105D9F1F601E80FD7
:10C67000F91F408150E068E070E0621B730B02C05C
:10C68000559547956A95E2F7800F911F26C0F401F2
:10C6900041914F01C8018C0F9D1FB50128E030E08A
:10C6A0000E94EC622196C615D7058CF3970127707E
:10C6B000307021153105A9F0F601EC0FFD1F408106
:10C6C00050E0C5010896821B930B02C05595479513
:10C6D0008A95E2F7C8018C0F9D1F60E070E00E9410
:10C6E000EC62DF91CF911F910F91FF90EF90DF905F
:10C6F000CF90BF90AF909F908F907F906F90089554
:10C700004F925F926F927F928F929F92AF92BF9261
:10C71000CF92DF92EF92FF920F931F93DF93CF930D
:10C7200000D0CDB7DEB78C01DC0116964C91169780
:10C73000842F90E08770907021E030E0009711F432
:10C7400020E030E04695469546957901E40EF11CCF
:10C75000C70102960E94044C009709F453C00E943E
:10C76000A44BFC01D80112968C91129780831396EA
:10C770008C9181830E94A44BF2E06F2E712C680E85
:10C78000791EC30160E070E0A7010E94AA83F8014E
:10C79000C480D58000E010E02E010894411C511C9B
:10C7A0002AC0D60111968C90119799247801E3E064
:10C7B000F594E794EA95E1F7E60CF71C77E0A72EED
:10C7C000B12CA022B122883130F00E94E34CAC01A0
:10C7D000C701B50107C00E94D04C9A838983C70165
:10C7E000B501A20194010E940063080D191DE2E049
:10C7F000F0E0CE0EDF1ED6018C91882391F621E069
:10C8000030E002C020E030E0C9010F900F90CF91DE
:10C81000DF911F910F91FF90EF90DF90CF90BF902D
:10C82000AF909F908F907F906F905F904F90089502
:10C83000E091E207F091E30709950895E0918B07F5
:10C84000F0918C0709950895E091E607F091E707CC
:10C8500009950895E091E807F091E9070995089591
:10C8600080E090E008950895E0916D07F0916E07E3
:10C8700009950895009731F0E0916D07F0916E07EA
:10C8800009950895E0916F07F09170070995089553
:10C8900080E090E008950F931F93DF93CF93CDB77F
:10C8A000DEB7E0970FB6F894DEBF0FBECDBF0E9493
:10C8B000EE4B8C010E949C4B602FAE014F5F5F4F8F
:10C8C0000E947E6C882309F445C088A99801281B22
:10C8D0003109C9010E94784B0097E1F12E81222392
:10C8E00071F18A859B853BEA8D3C930721F03FEFF0
:10C8F0008F3F930779F5223041F088E090E007C040
:10C90000019722912F3F41F00BC082E090E0FE01A1
:10C91000E80FF91F3C96F4CF181619068CF30FC0D8
:10C9200089E1BE01645F7F4F0E94D94C89E10E947A
:10C93000E34C6DEB76E20E94A142009759F088E14A
:10C94000BE016A5E7F4F0E94D94CE091CB07F09107
:10C95000CC070995E0960FB6F894DEBF0FBECDBFA9
:10C96000CF91DF911F910F910895AF92BF92CF9217
:10C97000DF92EF92FF920F931F93DF93CF93CDB788
:10C98000DEB7E0970FB6F894DEBF0FBECDBF6C01E7
:10C990008B01FE01319680E3DF011D928A95E9F754
:10C9A00081E089838CE00E94D04C8C831D821F82A1
:10C9B0008091D41289878F5F8093D41283E0E82E10
:10C9C000E8868DEC9BEA9B878A8789E10E94E34C8D
:10C9D00065EA76E00E94A142009731F082E08E8302
:10C9E0008FEF8C878D8709C089E10E94E34CBC01E1
:10C9F000CE010C960E949842EE828DEC9BEA9D8BB4
:10CA00008C8BCE0146966DEB76E20E9498420E9496
:10CA10009C4B9FA78EA70E94EE4B88AB7E0108948B
:10CA2000E11CF11CC7010E94756BA82E90E00E94CA
:10CA3000044C009741F10E94A44BBC01C7014A2D50
:10CA40000E94936BA0906307B09064070E94A44B70
:10CA50007C010E94F84BBC01C701F5010995C11486
:10CA6000D10489F0009721F08130910561F404C070
:10CA7000C80160E070E003C0C80164E070E041E01C
:10CA800050E0F6010995E0960FB6F894DEBF0FBEB0
:10CA9000CDBFCF91DF911F910F91FF90EF90DF906D
:10CAA000CF90BF90AF9008950E94B5668093D41246
:10CAB000E0916D07F0916E0709950895EF92FF924E
:10CAC000CF93DF93E82EE7017E01F92EE70104C042
:10CAD00060E070E00E940645899199910097C1F746
:10CAE000DF91CF91FF90EF900895EF92FF92CF9357
:10CAF000DF93E82EE7017E01F92EE70102C00E94D4
:10CB00004B44899199910097D1F7DF91CF91FF9094
:10CB1000EF900895CF93DF93EC017B836A830E94AB
:10CB2000475699838883DF91CF910895FC018081D6
:10CB3000918122813381820F931F91838083089595
:10CB4000CF93DF93EC010E94475699838883DF914E
:10CB5000CF910895CF93DF93EC010E94475628812F
:10CB60003981821B930B019621E030E04A815B8181
:10CB70004817590710F020E030E0C901DF91CF914C
:10CB80000895EF92FF92CF93DF93FC01C281D3818E
:10CB900080819181C80FD91F0E944756C81BD90BAD
:10CBA000CE01DF91CF91FF90EF900895CF93DF9367
:10CBB000E6E3F9E2C8EFD8E2AAE2B9E211921192F3
:10CBC00019921992199219921D9289E2EE34F8077E
:10CBD000A9F7DF91CF9108950F931F93CF93DF9320
:10CBE000FC01DC01A65DB64D8C91882339F10091E2
:10CBF000940010919500EF01CC0FDD1FCC0FDD1FCD
:10CC0000C850D74DDF01AA0FBB1FAA5CB64D8D914E
:10CC10009C9111979801281B390B40E050E06881E6
:10CC200079818A819B81260F371F481F591F2883CE
:10CC300039834A835B8311961C930E93EE0FFF1F7B
:10CC4000EE0FFF1FE850F74D608171818281938163
:10CC5000DF91CF911F910F91089560E070E0CB01BB
:10CC60000895FC01EE0FFF1FEE0FFF1FE850F74D78
:10CC700040835183628373830895EF92FF920F93F1
:10CC80001F93CF93DF932AE239E2C8EFD8E2E6E3BD
:10CC9000F9E2D9018D919D018823C9F0409194005A
:10CCA00050919500808191817A01E81AF90A00E09B
:10CCB00010E088819981AA81BB818E0D9F1DA01FE4
:10CCC000B11F88839983AA83BB83518340832496B1
:10CCD0003296B9E226333B07E1F6DF91CF911F91FF
:10CCE0000F91FF90EF9008950E94F26A08950F93BC
:10CCF0001F93FC01CB014091D5125091D612338382
:10CD000022831583048371836083F093D612E093AA
:10CD1000D5124115510511F40E940C6B80E090E092
:10CD20001F910F9108958091D5129091D61200977E
:10CD3000C1F01092D6121092D512DC0114966D91AA
:10CD40007C9115971296ED91FC9113970995E091BE
:10CD5000D512F091D612309721F0808191810E94F6
:10CD60000C6B08950E94408008950E943B800895B6
:10CD70008CEE97E00E943F4584EF97E00E943F458C
:10CD80000895EF92FF92CF93DF930E94AB4B0097F1
:10CD9000C9F084EF97E00E945F45E82EE7017E012D
:10CDA000F92EE701209731F10E94EE4B9983888399
:10CDB0000E94E94B9B838A83C70104960E94174B0C
:10CDC0008CAB18C08CEE97E00E945F45EC017E01B1
:10CDD000F92EE701209771F0C70102960E942E4BB1
:10CDE00099838883B7016E547F4FC7018E579F4F39
:10CDF0000E949B4CCE01DF91CF91FF90EF90089560
:10CE0000BC016E547F4F8E579F4F0E949B4C0895DC
:10CE1000CF93DF93EC018CEE97E0BE010E94AA4510
:10CE2000009719F08CEE97E009C084EF97E0BE01FF
:10CE30000E94AA45009729F084EF97E0BE010E9466
:10CE40008545DF91CF910895EF92FF92CF93DF93C5
:10CE5000EC018CEE97E0BE010E94AA45009779F0A4
:10CE600068817981CE0102960E94684CBE016E54A1
:10CE70007F4FCE018E579F4F0E94B04C1BC084EF56
:10CE800097E0BE010E94AA450097A1F00E943F4C86
:10CE9000688179818A819B810E94684C8CA990E08D
:10CEA0000E94044C0E94A44B4CA92496BE0150E061
:10CEB0000E94A183DF91CF91FF90EF900895EF92B0
:10CEC000FF92CF93DF93EC018CEE97E0BE010E94BE
:10CED000AA45009711F022960DC084EF97E0BE019D
:10CEE0000E94AA45009721F00A80DB81C02D02C074
:10CEF000C0E0D0E0CE01DF91CF91FF90EF90089598
:10CF0000FC0180819181089570E06F5B7F4F660F17
:10CF1000771F680F791FCB010895E62FF0E0EF5BD4
:10CF2000FF4FEE0FFF1FE80FF91F808191810895D9
:10CF300008958DE299E10E94B547009721F08DE2B6
:10CF400099E10E94A0470895E0913A19F0913B19A8
:10CF5000309711F00995089580E00895EF92FF92BF
:10CF60000F931F93CF93DF93EC018A0188819981FE
:10CF7000009731F023E08C30920709F006C12BC0F6
:10CF800080E00BC0E82FF0E0EE0FFF1FEE0FFF1F59
:10CF9000E55EF64E118210828F5F843098F38093A5
:10CFA000351980915C1090915D1090932C198093AD
:10CFB0002B190E94444480934E298DE299E160E44C
:10CFC00070E00E948A470E940D6E8CE093E0998386
:10CFD000888381E0DDC0623009F4B9C0633030F489
:10CFE000662309F489C0613081F79CC0673819F065
:10CFF000683859F741C0109236194BE1E42E49E1E7
:10D00000F42E18C0F701828193818017910749F4AB
:10D01000808191810E94546FF701118210821382E6
:10D02000128284E090E0E80EF91E809136198F5F3D
:10D030008093361980913619843020F3EEE5FEE2B4
:10D04000848D958D8017910719F4158E148E118E8D
:10D05000B0969EE2EE3DF90799F7E4EFFEE2818596
:10D0600092858017910711F4158214823D962FE264
:10D07000E637F207A1F7A9CF89E14D32580709F049
:10D08000A4CFCA010E94B547009709F49ECF109221
:10D0900036192DC0F0E035E0EE0FFF1F3A95E1F7AD
:10D0A000E25AF14D818D8823E9F08DE299E10E94E9
:10D0B000A0478091361990E025E0880F991F2A95A6
:10D0C000E1F7825A914D90935D2E80935C2E82E021
:10D0D0000E94886F80914F2990915029009711F0FC
:10D0E0000E94A467809136198F5F80933619E09172
:10D0F0003619E43078F269CF4115510509F465CF4E
:10D1000050935D2E40935C2E83E00E94886F809147
:10D110004F2990915029009711F00E94A4670E9416
:10D12000996753CF4115510509F44FCF5093592EAC
:10D130004093582E85E00E94886F80914F299091EE
:10D140005029009709F441CF0E94A4673ECF8091F7
:10D150004F2990915029009709F437CF8091602989
:10D16000863031F48091782981FF02C00E9499674E
:10D1700081E00E94886F80914F29909150290097FB
:10D1800009F423CF0E94D76920CF1982188283E047
:10D19000DF91CF911F910F91FF90EF9008959093A1
:10D1A0003B1980933A19089520915C1030915D10DD
:10D1B00060E0EBE1F9E113C0408151814817590764
:10D1C00061F4428153814217530739F4609339194E
:10D1D000118210820E94546F089534966F5F6430FC
:10D1E00058F360933919089540E0EBE1F9E116C076
:10D1F000542F5F5F208131812115310569F44093FF
:10D2000038199183808320915C1030915D103383B5
:10D2100022830E946E6F08953496452F443040F368
:10D22000409338190895FC0180915C1090915D1035
:10D23000958F848F778F668F0895FC0180915C10A5
:10D2400090915D1092878187748763870895CF934B
:10D25000DF93EA010E94D06EFC01009741F08091BB
:10D260005C1090915D1092878187D487C387CF012E
:10D27000DF91CF9108950F931F93DF93CF9300D049
:10D2800000D0CDB7DEB78C01AB018FEF89838A83E5
:10D290008B838C83CE010196B8010E942769FC0123
:10D2A000009711F015830483CF010F900F900F901A
:10D2B0000F90CF91DF911F910F91089589E098E031
:10D2C00062E040E050E00E94F74410925029109232
:10D2D0004F290895AC0189E098E061E00E94D444B0
:10D2E0000895AC0189E098E060E00E94D44408957C
:10D2F0000F931F93CF93DF93EA010E94466E8C0138
:10D30000009761F080915C1090915D10F801958F0D
:10D31000848FD78FC68FC8010E947169C801DF91C1
:10D32000CF911F910F910895CF93DF93A0915C2E21
:10D33000B0915D2E109719F0ED016C9605C0C0916B
:10D34000582ED091592E29968091572E86FF22C0B3
:10D350001092371940E0EBE1F9E116C020813181EC
:10D3600014968D919C9115972817390759F482814D
:10D370009381009739F040933719998388831B82F2
:10D380001A8206C034964F5F443040F340933719F9
:10D390000E94996788819981009731F04A815B8169
:10D3A00060914E290E94F744DF91CF9108950F9329
:10D3B0001F93CF93DF9380916029863009F074C06A
:10D3C00080914F299091502925E08030920709F0F3
:10D3D0006BC0C4E9D2E0D0935029C0934F2902E03A
:10D3E0000093592914E910935A2910927C2910921C
:10D3F0007B290E94056E8095909590937C2980935F
:10D400007B2910926229109261290E94F46D809507
:10D41000909590936229809361290E94A467D0938C
:10D420005029C0934F290093592910935A2990915C
:10D430005A2E80915B2EE92FF82FDF01A459BD4FA2
:10D440008CE692E00D9001920197E1F78FE699E268
:10D450006CE672E00E94986D8091532980936F2949
:10D460008091542980937029809155298093712946
:10D47000809156298093722910927C2910927B29E1
:10D480000E94056E8095909590937C2980937B29CE
:10D4900010926229109261290E94F46D80959095F6
:10D4A00090936229809361290E94A467DF91CF91B4
:10D4B0001F910F910895282F392FF90120E030E0B6
:10D4C00080E0A8E112C0419198E0542F5827B52F71
:10D4D000B17050FD8A278695B13009F4806891506B
:10D4E00011F04695F2CF2F5F3F4F2617370759F7B8
:10D4F00008951F920F920FB60F920BB60F92112440
:10D500002F933F934F935F936F937F938F939F934B
:10D51000AF93BF93EF93FF93809194009091950008
:10D5200090933B2980933A2981E080932C29809124
:10D530007100807D809371000E94936680912C29F8
:10D540008823E9F1809194009091950020913A29E7
:10D5500030913B2982179307A0F480910029909184
:10D560000129A0910229B09103298C57914EAF4F08
:10D57000BF4F8093002990930129A0930229B09373
:10D5800003298091940090919500821B930BA0E059
:10D59000B0E0209100293091012940910229509159
:10D5A0000329820F931FA41FB51F80930029909316
:10D5B0000129A0930229B093032910922C29FF91ED
:10D5C000EF91BF91AF919F918F917F916F915F91FB
:10D5D0004F913F912F910F900BBE0F900FBE0F9068
:10D5E0001F9018959FB7F894E1E7F0E08081807D67
:10D5F000808388B38F6288BB10929000E1E9F0E0ED
:10D6000010821092920010929500109294008081E6
:10D61000856080839FBF08952FB7F89490939900F9
:10D620008093980088B38F6288BBE1E7F0E0808147
:10D63000826080832FBF0895EF92FF92CF93DF9394
:10D64000FC01DB0185E0EB0119928A95E9F7858100
:10D6500090E083709070009711F082E08C93878146
:10D6600090E083709070009721F082E012968C9386
:10D670001297858190E083709070009799F0878170
:10D6800090E083709070009769F0238934898185D8
:10D6900092852817390731F481E0848312961C9211
:10D6A000129701C01482858183708250823030F4D9
:10D6B000C82FD0E0CD5ED74F888101C080E01196A1
:10D6C0008C931197E781E370E250E23028F4F0E0A8
:10D6D000ED5EF74F808101C080E013968C93139725
:10D6E000DF91CF91FF90EF900895DF93CF9300D01B
:10D6F00000D00F92CDB7DEB7BE016F5F7F4F0E94A3
:10D700001C6B89819A81890F8D5F9B81890F9C8118
:10D71000890F9D81890F0F900F900F900F900F90A0
:10D72000CF91DF910895AF92BF92CF92DF92EF92A7
:10D73000FF920F931F93DF93CF9300D000D000D0C0
:10D74000CDB7DEB78C017B01BE016F5F7F4F4E838B
:10D750000E941C6BC9809A81A92EBB24DB808C811E
:10D76000682F70E095012C0D311D2D5F3F4F2D0D61
:10D77000311D260F371F5D81250F311D4E8150E071
:10D78000421753070CF4A8C0D80111964C91119779
:10D7900050E041705070E3E0440F551FEA95E1F707
:10D7A00012962C91129730E02170307054E0220FC5
:10D7B000331F5A95E1F7242B3C913770232B139696
:10D7C0003C911397E32FF0E0E170F07045E0EE0F2D
:10D7D000FF1F4A95E1F72E2B14963C911497E32FE7
:10D7E000F0E0E170F07036E0EE0FFF1F3A95E1F7E0
:10D7F0002E2BF701208315964C91159750E043701E
:10D800005070440F551F440F551F16962C911697B4
:10D8100030E02370307054E0220F331F5A95E1F747
:10D82000242B17963C9117973295330F330F307C8A
:10D83000322B318318962C9118972283FC2DF230CD
:10D8400069F419962C91D70113962C931397F8012C
:10D85000228514962C93149745E001C043E0E92FEC
:10D86000F0E03B96E00FF11F542F0AC09701250FFF
:10D87000311DC290D901CC925F5F0894A108B10814
:10D88000A114B10499F7940FBD2DB23089F4F701BA
:10D89000E90FF11DD80153962C91539720839F5F78
:10D8A000F701E90FF11D54962C91549720839F5F47
:10D8B000E82FF0E07596E00FF11F292F08C0D7017F
:10D8C000A20FB11D32913C932F5F615070406115E2
:10D8D0007105A9F7890F01C080E026960FB6F8946C
:10D8E000DEBF0FBECDBFCF91DF911F910F91FF9093
:10D8F000EF90DF90CF90BF90AF900895BF92CF92FE
:10D90000DF92EF92FF920F931F93CF93DF937C01EF
:10D91000D62EEA01633008F4ADC0FC018081B82E38
:10D92000B294B694B694B3E0BB22F1E0BF22F70103
:10D930009181292F269526952370C92EC294C694CD
:10D94000C694A3E0CA22382F37703883382F369513
:10D950003695369531703983382F329531703A8348
:10D960008295869581708B83BC822D83892F8295C9
:10D9700083708E83CF828281888787010D5F1F4FDE
:10D98000222361F1F801918180E0F7013381830F57
:10D99000911D9A87898787010B5F1F4F223081F481
:10D9A000CA010B9665EA76E00E949842F8018181EF
:10D9B0008B87F70185818C878701095F1F4F16C010
:10D9C0002330A1F4F7013D96DA011B9682918D93E5
:10D9D000E017F107D9F7085F1F4F08C0CA010B967F
:10D9E00065EA76E00E9498421A861986CC2089F171
:10D9F000BB2059F4F801918180E02081820F911DB4
:10DA00009C8B8B8B0E5F1F4F04C089859A859C8BE6
:10DA10008B8BFC2DF23071F4CE01459665EA76E0F1
:10DA20000E949842F80181818D8B80818E8B0E5FE0
:10DA30001F4F17C0FC2DF330A1F4085F1F4FD80112
:10DA4000FE01759680E09E9191938F5F8830D9F7A3
:10DA500008C0CE01459665EA76E00E9498421C8A8D
:10DA60001B8A802F8E199D2D981B9FA71EA70DA77F
:10DA7000D81608F480E0DF91CF911F910F91FF90AD
:10DA8000EF90DF90CF90BF9008959C01415050409F
:10DA9000460F571FDB0110C0FC91E0E011968C91FE
:10DAA0001197BF01680F711D260F371F2617370703
:10DAB00010F42F5F3F4F1296A417B50768F3A41711
:10DAC000B50749F49C9180E0280F391F28173907C2
:10DAD00010F42F5F3F4FC9010895CF93DF939091CA
:10DAE0005A29C92FD0E064973091592920E0C20FFC
:10DAF000D31F9E01280F311DC90163E679E248E07A
:10DB000050E00E94456D6BE679E2AE010E94456DE2
:10DB1000009719F0382F292F02C02FEF3FEFC901CE
:10DB2000DF91CF91089590934B1980934A190895EE
:10DB3000FC014381460F40935629872F9927228164
:10DB4000280F20935529A181A093542950815093E7
:10DB5000532930E02817390748F48A2F8F5F8093C4
:10DB60005429882319F45F5F50935329842F90E040
:10DB700070708617970798F4809155298F5F80936E
:10DB80005529882361F4809154298F5F809354290B
:10DB9000882329F4809153298F5F80935329089516
:10DBA000BC0180915C2E90915D2E08960E94986D2C
:10DBB000E0915C2EF0915D2E8091532980878091B9
:10DBC000542981878091552982878091562983879E
:10DBD00008959C01AB0180E090E0B9010E94456D81
:10DBE000382F292FC901089580E090E067E579E298
:10DBF00044E150E00E94456D009719F0382F292F1D
:10DC000002C02FEF3FEFC901089586E00E946D6DBD
:10DC1000089581E10E946D6D089580E009C0E82FAC
:10DC2000F0E0EE0FFF1FE252F14D118210828F5F84
:10DC30008430A8F380E00BC0E82FF0E095E0EE0F11
:10DC4000FF1F9A95E1F7E25AF14D118E8F5F8430F4
:10DC500098F380E094E090934D1980934C1940E044
:10DC60008DE090E00EC0242F30E0289FF001299F26
:10DC7000F00D389FF00D1124EC50F14D15821482F7
:10DC80004F5F4A3080F340934819089520914C1912
:10DC900030914D192F5F3F4F4DE72030340710F082
:10DCA00020E030E1522F432FA0E013C0EA2FF0E034
:10DCB000B5E0EE0FFF1FBA95E1F7E25AF14DB18DD5
:10DCC000BB2331F00480F581E02DE417F50711F353
:10DCD000AF5FA43059F730934D1920934C1910922F
:10DCE000481920E0E0E0F0E01EC0A22FB0E035E0EF
:10DCF000AA0FBB1F3A95E1F7A25AB14D59963C9134
:10DD00005997332321F420934819FD0110C037306F
:10DD100049F4309731F05A964C915A97328D341716
:10DD200008F4FD012F5F243000F320934819309749
:10DD3000A9F122E0218F20914219248720914319D3
:10DD4000258720914419268720914519278728ED9A
:10DD500034E0338B228B358B248B21E030E0318B08
:10DD6000208B138E21E0228F23E0208F168A20E162
:10DD7000278B20914C1930914D19322723273227B8
:10DD80003583248377836683DC012D913D914D910A
:10DD90005C9113972083318342835383CF0108958D
:10DDA0000F931F93CF93DF9320914C1930914D190E
:10DDB0004DE050E02F5F3F4FADE720303A0710F0C5
:10DDC00020E030E1B22FA32F10E012C0C12FD0E02D
:10DDD000C49FF001C59FF00DD49FF00D1124EC50AD
:10DDE000F14D0480F581E02DEA17FB0719F31F5F61
:10DDF0001A3061F730934D1920934C1910E02DE043
:10DE000030E01AC0012F0F5FC12FD0E0C29FF00198
:10DE1000C39FF00DD29FF00D1124EC50F14DDF01A6
:10DE20001496448155814115510529F410934819E0
:10DE3000309749F433C0102F1A3020F3109348194B
:10DE4000E0E0F0E02BC020914C1930914D193227C1
:10DE50002327322711963C932E937783668300976E
:10DE600029F4108211821282138209C0DC012D91E3
:10DE70003D914D915C9120833183428353838DE0AA
:10DE800090E0C89FD001C99FB00DD89FB00D11245C
:10DE9000AC50B14D80E418968C931897CF01DF9168
:10DEA000CF911F910F91089540E013C0E42FF0E04F
:10DEB000542F5F5FEE0FFF1FE252F14D2081318141
:10DEC0002817390729F440934819118210820895C0
:10DED000452F443058F340934819089540E013C04B
:10DEE000E42FF0E0542F5F5FEE0FFF1FE252F14D81
:10DEF000208131812115310529F4409348199183FE
:10DF000080830895452F443058F34093481908956D
:10DF1000EF92FF920F931F93CF93DF93C0915C2EEC
:10DF2000D0915D2E843009F4F7C10FE719E2109308
:10DF30005B2E00935A2E109352290093512983305F
:10DF400071F4898D90E08F7090708330910509F0A5
:10DF500074C088899989009709F02FC78DC08230D5
:10DF600009F08EC0809145198F5F809345198823F1
:10DF700099F4809144198F5F80934419882361F448
:10DF8000809143198F5F80934319882329F48091EE
:10DF900042198F5F809342191092502910924F2995
:10DFA0001092F32E1092F22E898D873011F0853069
:10DFB00041F48A8D8F5F8A8F843109F0FEC6198EF5
:10DFC000FCC6882309F4F9C6288939892115310549
:10DFD00009F44EC09A8D292F21502A8F992309F0D8
:10DFE000ECC69B8D983031F0282F2150223048F418
:10DFF000953039F4198E80E88093572E0E949469E9
:10E0000095C5953048F423E030E0092E02C0220F78
:10E01000331F0A94E2F701C020E32A8F9F5F9B8F92
:10E0200090E08F70907083309105E1F0843091051D
:10E030004CF48130910509F461C38230910509F0F7
:10E04000BCC60DC08630910509F40CC58830910519
:10E0500009F408C58430910509F0AFC603C51092D4
:10E0600078294FC384E08093572E0E94946990C50D
:10E070008F70833009F0A1C688E08093572E4BC57E
:10E08000853019F5E091582EF091592E84819581B3
:10E09000009709F492C610925D2E10925C2E0C50DF
:10E0A000104010935B2E00935A2E10935229009328
:10E0B00051291092F32E1092F22E109250291092A4
:10E0C0004F2988E08093572E25C108521040809137
:10E0D0005729853409F071C69091592980E0209123
:10E0E0005A297C01E20EF11C80914F299091502910
:10E0F0008E159F0508F461C6F0925029E0924F29D1
:10E1000080915D2990E08F739070009709F055C65B
:10E1100080915E29882309F050C68091EE2E90915F
:10E12000EF2EC0911908D0911A088C179D0759F449
:10E130004091F02E5091F12E20911B0830911C0837
:10E1400042175307A1F020916729309168292817B9
:10E15000390709F032C62091692930916A298091E6
:10E16000F02E9091F12E2817390709F026C60E944B
:10E17000F46D2FEF8F3F920709F01FC68091602941
:10E18000863009F431C18131E9F1813009F015C6D9
:10E1900080916B29883009F010C610926B2980910C
:10E1A0006D2990916E294FEF873F940710F00996E3
:10E1B00001C0089690936E2980936D298091632900
:10E1C00090916429A0916529B0916629809367296F
:10E1D00090936829A0936929B0936A298091EE2EC3
:10E1E0009091EF2EA091F02EB091F12E80936329A3
:10E1F00090936429A0936529B093662980E4F8017F
:10E200008087B8C5C7014C979093502980934F29B8
:10E2100083E799E290935B2E80935A2E8091712927
:10E2200090917229009739F00E94096EFFEF8F3F9D
:10E230009F0709F0C2C520916D2930916E292115E3
:10E24000310509F4BAC584EF9EE29093592E80936C
:10E25000582E60911B0870911C0840911508509130
:10E260001608009117081091180839C0848195810B
:10E27000009781F12817390769F586819781009702
:10E2800039F0A0916B29B0916C29A817B90711F545
:10E29000808191818C179D0729F4A281B381A617F3
:10E2A000B70739F18417950729F4A281B381A01724
:10E2B000B107F9F0A0916329B0916429A817B907B3
:10E2C00049F4A0916529B091662982819381A817AC
:10E2D000B90779F03D96F093592EE093582EE091CE
:10E2E000582EF091592E8FE2E637F80708F4BECF8A
:10E2F00064C510925D2E10925C2E82E08093572EA2
:10E3000083E799E290935229809351291092F32E3A
:10E310001092F22E0E9494698091F22E9091F32E29
:10E32000009709F44AC59C01245E3F4F3093502961
:10E3300020934F293093592920935A29E091582E40
:10E34000F091592E208520935F2921E120936029A7
:10E3500008969827892798279093702980936F298A
:10E3600010927229109271298481958190936C2961
:10E3700080936B298681978190936E2980936D2974
:10E380008091EE2E9091EF2EA091F02EB091F12E73
:10E390008093632990936429A0936529B09366299B
:10E3A00080819181A281B3818093672990936829AC
:10E3B000A0936929B0936A298FE799E290935B2E25
:10E3C00080935A2E0E94096E8095909590937229A1
:10E3D00080937129009709F0CDC48FEF9FEF909340
:10E3E000722980937129C6C40E94056EEFEF8F3F9A
:10E3F0009E0709F0E2C480916D2990916E290097E3
:10E4000009F4DBC420916B2930916C292115310569
:10E4100009F4D3C4CEE5DEE2498D4423E9F06C81F2
:10E420007D8186179707C1F46E817F812617370794
:10E4300099F4E0916329F091642968817981E61764
:10E44000F70751F4E0916529F09166296A817B8193
:10E45000E617F70709F46DC1A096FEE2CE3DDF078F
:10E46000D9F6209178292F732230B9F49093471967
:10E470008093461940E00DC0E42FF0E0EE0FFF1F3F
:10E48000E252F14D208131814F5F8217930709F4E9
:10E490006EC0443088F3409348198091782982FDFA
:10E4A0008CC484E1F80181A388E290E09093502924
:10E4B00080934F2980E580A38091722990917629DD
:10E4C000938F3091712990917529928F368F209179
:10E4D000702990917429918F258F90916F29909335
:10E4E000481940917329408F948F8F5F878F8823BD
:10E4F00061F4832F8F5F868F882339F4822F8F5F9B
:10E50000858F882311F49F5F948F80916B29909160
:10E510006C29909347198093461920916D29309169
:10E520006E29F801358B248B978B868B809163291C
:10E5300090916429A0916529B091662980936729FB
:10E5400090936829A0936929B0936A298091EE2E4F
:10E550009091EF2EA091F02EB091F12E809363292F
:10E5600090936429A0936529B0936629E8C310921B
:10E57000481980E0C0E0D0E022C0E82FF0E075E06C
:10E58000EE0FFF1F7A95E1F7E25AF14D918D992335
:10E5900021F480934819EF0116C0973079F4209741
:10E5A00021F0228D9A8D921748F4C82FD0E065E0B3
:10E5B000CC0FDD1F6A95E1F7C25AD14D8F5F8430D1
:10E5C000E0F280934819209709F4F7C3D0935D2EA9
:10E5D000C0935C2E83E08A8F888F1E8A84E08F8BA5
:10E5E0001B8E80916D2990916E299D838C838091E3
:10E5F0006B2990916C299F838E83809163299091E0
:10E600006429A0916529B091662988839983AA839A
:10E61000BB8381E0898F809142198C878091431957
:10E620008D87809144198E87809145198F8781E06D
:10E6300090E0998B888B809172298B8780917129CA
:10E640008A8780917029898780916F29888781E0E6
:10E6500090E00E94D06D80917729282F30E0207FB4
:10E660003070213531050CF449C082958F7090E0EF
:10E670000597880F991F880F991F5091491940E0FD
:10E6800034C0F901E95AF64D50A5552329F44093B9
:10E6900048191092491932C0513011F44F5F25C00A
:10E6A0005230E1F461A56430C9F4409348195093A5
:10E6B000491932A520E083A590E0822B932B9093FB
:10E6C000471980934619F4E0893D9F0710F088EDC3
:10E6D00094E09B8B8A8B9D8B8C8B10C0295A364D76
:10E6E000F90121A5222331F0420F242F30E0281711
:10E6F00039073CF2409348195093491980E18093BF
:10E7000078298091782982608093782982E08093AB
:10E710007F2984E0809380298093812988ED8093EC
:10E7200082298CE290E09093502980934F2980E6D3
:10E73000B3C2D0935D2EC0935C2E1092572E809161
:10E74000782990E082FF03C0198E80E24EC22091AA
:10E75000772922952F70220F220F20934819B70195
:10E76000621B71099B012451304030935029209342
:10E770004F2950E04F7050704230510539F4AC01D0
:10E780004F7350704231510551F42AC04130510548
:10E7900031F4AC014F7350704230510509F121152D
:10E7A000310531F49C012370307021153105C1F021
:10E7B00030916F292885321709F064C23091702991
:10E7C0002985321709F05EC2309171292A853217E6
:10E7D00009F058C2309172292B85321709F052C2C4
:10E7E00084FF4AC0688979896115710509F444C0BC
:10E7F000CE010C960E94986D309173298091532917
:10E800003817D1F520917429809154292817A1F542
:10E810009091752980915529981771F580917629E5
:10E8200040915629841741F53C872D879E878F8715
:10E830008B8D8823D1F42E89888D9A8D891B922FF8
:10E84000969596959695891B280F2E8B87FD819519
:10E850009F89392F36953695931B980F9F8B822F62
:10E86000869586958695890F888F81E08093572EAF
:10E87000888D8A8F198A188A298D30E0C9018F7096
:10E8800090708430910509F4B5C18530910564F428
:10E8900082309105C9F1833091050CF0B9C0813007
:10E8A000910509F08AC211C08630910509F4E2C1D0
:10E8B000863091050CF4BEC18730910509F4E2C1A0
:10E8C0008830910509F079C28AC18091572E80FF66
:10E8D00014C083E0898F80E48093572E198A188AA8
:10E8E00080914F2990915029009709F410C122E49A
:10E8F0002093572E0E94D06D0AC1809178298F7382
:10E90000823009F05AC2FACE8091572E80FF75C02E
:10E91000809178298F73823109F06FC080917729B7
:10E92000282F30E0207F3070213531050CF449C0AC
:10E9300082958F7090E00597880F991F880F991F17
:10E940005091491940E034C0F901E95AF64D50A5FB
:10E95000552329F4409348191092491932C0513077
:10E9600011F44F5F25C05230E1F461A56430C9F461
:10E97000409348195093491932A520E083A590E0AF
:10E98000822B932B909347198093461974E0893D0D
:10E99000970710F088ED94E09B8B8A8B9D8B8C8B76
:10E9A00010C0295A364DF90121A5222331F0420F1A
:10E9B000242F30E0281739073CF240934819509330
:10E9C000491983E0898F80916F2988878091702908
:10E9D0008987809171298A87809172298B8781E04C
:10E9E00090E00E94D06D82E48093572E198A188A95
:10E9F0001092502910924F298AC080E28093572E9E
:10EA00000E949469E0915C2EF0915D2E118E45CDAF
:10EA10008091782980FF2AC024FD28C0888999899F
:10EA2000009709F0CAC180914F2990915029019611
:10EA30000E94D06D2091572E822F80618093572E97
:10EA400080914F2990915029009719F022612093CD
:10EA5000572E0E94946981E090E0998B888B88E022
:10EA6000898F1B8E81E1809378290FC185FF1CC09F
:10EA700050917D2940E080917E2990E0842B952B58
:10EA800040915A2E50915B2E480F591F50935B2E88
:10EA900040935A2E40914F2950915029481B590BB1
:10EAA0005093502940934F2980914F29909150299C
:10EAB000009749F024FD07C02091572E2260209333
:10EAC000572E0E94D06D9091792980E020917A296B
:10EAD000820F911D90934719809346192C893D8987
:10EAE0002817390710F0009721F430934719209325
:10EAF000461980914619909147199B8B8A8B80917A
:10EB0000572E90E083709070009709F456C11092D0
:10EB1000F32E1092F22E0E9494698091572E85FF59
:10EB200007C01092F32E1092F22E198E84E19BCF23
:10EB300084FF0AC01092F32E1092F22E81E090E032
:10EB4000998B888B84E08CCF2091F22E3091F32E1C
:10EB500021153105E1F080FF02C0198A188A8889E1
:10EB60009989009781F48A899B898217930720F4F9
:10EB70009093F32E8093F22E8091F22E9091F32EAB
:10EB8000998B888B04C09093F32E8093F22E1B8E6A
:10EB9000809151299091522990935B2E80935A2E07
:10EBA0008091F22E9091F32E009759F088899989DF
:10EBB000009739F088969093502980934F2988E1E7
:10EBC0000BC08091572E81FFF8C088E290E09093AF
:10EBD000502980934F2980E1809378295CC08091EF
:10EBE000572E80FFEAC0198E80E18093572E0E9435
:10EBF0009469E3C080914F2990915029009711F0BA
:10EC00000E94D06D909178298091572E90FF0BC073
:10EC100080FF06C087E0898F1A8E198A188A19C06A
:10EC200086E0898F16C080FF1EC085E0898F198A13
:10EC3000188AC3C080914F2990915029009711F0F4
:10EC40000E94D06D8091782980FF0DC087E0898F68
:10EC50001A8E81E090E00E94D06D80E18093572E63
:10EC60000E9494690FC080914F299091502900977C
:10EC700049F4A3C08091572E80FF9FC087E0898F01
:10EC80001A8E9BC080E1F80181A388E290E0909306
:10EC9000502980934F2980E5809377298885809338
:10ECA00073298985809374298A85809375298B853A
:10ECB000809376298C8580936F298D858093702928
:10ECC0008E85809371298F858093722986E0809349
:10ECD00060298C819D8190936C2980936B298E8112
:10ECE0009F8190936E2980936D298091EE2E909153
:10ECF000EF2EA091F02EB091F12E80936329909386
:10ED00006429A0936529B093662988819981AA8195
:10ED1000BB818093672990936829A0936929B09358
:10ED20006A29898D84FF05C010927A291092792969
:10ED300006C084E08093792988ED80937A2980E465
:10ED400080935F2980914F29909150299093592960
:10ED500080935A2910927E2910927D2910927C2945
:10ED600010927B290E94056E8095909590937C2946
:10ED700080937B2985E4809357291092582910921B
:10ED80005E2910925D2980914A1990914B19019644
:10ED900090934B1980934A1990935B2980935C2937
:10EDA00010926229109261290E94F46D80959095CD
:10EDB000909362298093612904C010925029109287
:10EDC0004F291092572EDF91CF911F910F91FF90F5
:10EDD000EF900895382F292FC9010895382F292F32
:10EDE00040E050E076276727762780E090E0CB016F
:10EDF00077276627262B372B482B592BB901CA01B9
:10EE00000895AC01E0915129F0915229222733272E
:10EE10002E1B3F0B295A314D621773070CF49B01CF
:10EE20001216130664F42093F22E3093F32E4E172D
:10EE30005F0729F0CF01BA01A9010E94A1830895BB
:10EE40000F93DF93CF93CDB7DEB760970FB6F894EB
:10EE5000DEBF0FBECDBF002309F459C029833A831A
:10EE60004B835C836D837E838F839887E0E2E01B16
:10EE700029813A814B815C811E16BCF019861A8665
:10EE80001B861C868E2F992787FD909590958195DE
:10EE90009F4F04C0220F331F441F551F8A95D2F77E
:10EEA0002D873E874F87588B2AC0CA01B901002E93
:10EEB00004C0660F771F881F991F0A94D2F76987CD
:10EEC0007A878B879C87DA01C90104C0B695A7951C
:10EED00097958795EA95D2F72D813E814F81588588
:10EEE00004C0220F331F441F551F0A95D2F7822BEF
:10EEF000932BA42BB52B8D879E87AF87B88B298545
:10EF00003A854B855C856D857E858F859889609671
:10EF10000FB6F894DEBF0FBECDBFCF91DF910F913A
:10EF20000895A0E1B0E0E7E9F7E70C94BE7F2983FC
:10EF30003A834B835C836D837E838F839887A98616
:10EF4000BA86CB86DC86ED86FE860F87188B2D81F0
:10EF50003E814F8158858D859E85AF85B88928175C
:10EF600039074A075B07C8F082179307A407B5075C
:10EF700090F029813A814B815C8189859A85AB85A6
:10EF8000BC85281739074A075B0738F082179307B3
:10EF9000A407B50720F482E003C080E001C081E04F
:10EFA0006096EAE00C94DA7F2F923F924F925F9244
:10EFB0006F927F928F929F92AF92BF92CF92DF9289
:10EFC000EF92FF920F931F93DF93CF93CDB7DEB7EE
:10EFD00063970FB6F894DEBF0FBECDBF6C017F877D
:10EFE0006E87FC0117821682838181FD04C06FC386
:10EFF0004C855D8504C01E010894211C311CF6015E
:10F000009381EE85FF8593FD859193FF8191FF8725
:10F01000EE87882309F457C3853241F493FD859127
:10F0200093FF8191FF87EE87853259F490E0B60116
:10F030004A8B5B8B0E9403844A895B895D874C877E
:10F04000D7CF10E0FF2400E00032B0F48B3269F03B
:10F050008C3228F4803251F0833271F40BC08D323F
:10F0600039F0803349F401602CC00260046029C08B
:10F07000086027C0006125C007FD2EC0282F20533F
:10F080002A3098F406FF08C0812F880F182F110F1F
:10F09000110F180F120F15C08F2D880FF82EFF0CAF
:10F0A000FF0CF80EF20E00620CC08E3221F406FD49
:10F0B0000AC3006406C08C3611F4006802C08836AA
:10F0C00059F4EE85FF8593FD859193FF8191FF872C
:10F0D000EE87882309F0B8CF982F9554933018F411
:10F0E0000061805E06C0982F9556933008F09BC152
:10F0F0000F7E06FF16E06FE3E62EE022853619F458
:10F10000F0E4EF2A07C0863619F420E8E22A02C0AC
:10F1100011111150E7FE06C01C3340F4912E939458
:10F1200027E00BC0183030F4212F06C027E03CE365
:10F13000932E03C027E017E09924CA0104969D8707
:10F140008C87FA016081718182819381A101092DEF
:10F150000E94A8825C016980262D30E0398B288BC3
:10F1600060FE03C0388933FF06C0E1FC06C0E2FE42
:10F1700006C000E205C00DE203C00BE201C000E0E2
:10F18000888999898C7090700097C1F1002311F0E3
:10F1900084E001C083E08F1558F4F81AE3FC09C03D
:10F1A00080E290E0B6010E940384FA94C9F701C09E
:10F1B000FF24002329F0802F90E0B6010E940384F1
:10F1C000888983FD03C007E01FE00EC003E01FE055
:10F1D0000BC0A114B10409F0805290E0B6010E9466
:10F1E00003840F5F1F4F05C0AE2CBB2490E1A92202
:10F1F000BB24F8018491882361F762C2E7FE0EC048
:10F200009A0CF889F4FF04C08A81813309F49A9436
:10F21000191454F5292D293050F52DC0E6FC2BC0CA
:10F22000812F90E08A159B054CF03CEFA3163FEF31
:10F23000B30624F080E8E82A01C01150112349F0F8
:10F24000E2E0F0E0EC0FFD1FE10FF11D8081803363
:10F25000A1F3E7FE10C0912E9394812F90E0A816A1
:10F26000B90644F41A1907C09924939404C098E08D
:10F27000992E01C010E0E7FE07C01A141B043CF4ED
:10F2800095012F5F3F4F05C025E030E002C021E02F
:10F2900030E0002311F02F5F3F4F112329F0812F21
:10F2A00090E00196280F391F8F2D90E0281739071D
:10F2B00014F4F21A01C0FF244E2C5524C2018970A7
:10F2C0009070009749F406C080E290E0B6010E9479
:10F2D0000384FA94FF20C1F7002329F0802F90E0E7
:10F2E000B6010E94038443FC09C006C080E390E09D
:10F2F000B6010E940384FA94FF20C1F7E7FE46C0DE
:10F300003501B7FE02C06624772425010894411C0C
:10F31000511C46185708420C531CF501E919F10914
:10F320004F01812F90E000271127081B190BFFEFD9
:10F330006F16FFEF7F0629F48EE290E0B6010E947F
:10F340000384A614B70434F0861497041CF4F20165
:10F35000808101C080E30894610871080894411C11
:10F36000511C601671062CF090E0B6010E940384D7
:10F37000DECF6A147B0441F49A81963320F49533EE
:10F3800019F4F889F4FF81E390E049C08A81813360
:10F3900011F02FEE622290E0B6010E940384112347
:10F3A00089F08EE290E0B6010E94038402E0F10150
:10F3B000E00FF11D0F5F808190E0B6010E94038491
:10F3C0001150A9F744FE03C085E490E002C085E631
:10F3D00090E0B6010E940384B7FC05C0A114B104FB
:10F3E00041F464FE06C0B094A194B108B3948DE2D8
:10F3F00001C08BE290E0B6010E94038480E305C067
:10F400008F5FE6EFFFEFAE0EBF1EFAE0AF16B1045E
:10F41000BCF790E0B6010E940384C501C096B60116
:10F420000E9403844DC1833631F0833789F08335E0
:10F4300009F059C022C09A012E5F3F4F3D872C87AB
:10F44000FA0180818983310181E0A82EB12C13C09B
:10F450009A012E5F3F4F3D872C87FA0160807180B3
:10F4600006FF03C0612F70E002C06FEF7FEFC301A2
:10F470000E94C9835C010F7714C09A012E5F3F4F31
:10F480003D872C87FA016080718006FF03C0612FE1
:10F4900070E002C06FEF7FEFC3010E9491835C01B7
:10F4A000006803FD1CC006C080E290E0B6010E9427
:10F4B0000384FA948F2D90E0A816B906A8F30FC024
:10F4C000F30107FD859107FF81913F0190E0B601AF
:10F4D0000E940384F110FA940894A108B108A114C1
:10F4E000B10471F7EDC0843611F0893661F507FF7C
:10F4F0000BC09A012C5F3F4F3D872C87FA0160813A
:10F500007181828193810CC09A012E5F3F4F3D87AC
:10F510002C87FA0160817181882777FD8095982F6B
:10F520000F7697FF08C090958095709561957F4FF5
:10F530008F4F9F4F0068A1012AE030E00E940E85A6
:10F54000982E921841C0853721F40F7E2AE030E0D2
:10F5500020C0097F8F36A9F0803720F4883509F064
:10F56000B2C00BC0803721F0883709F0ACC001C0B1
:10F57000006104FF09C0046007C004FF08C0066002
:10F5800006C028E030E005C020E130E002C020E104
:10F5900032E007FF0AC0CA0104969D878C87FA01F2
:10F5A000608171818281938109C0CA0102969D8721
:10F5B0008C87FA016081718180E090E0A1010E9456
:10F5C0000E85982E92180F7706FF09C00E7F9116B0
:10F5D00030F404FF06C002FD04C00F7E02C0E92C17
:10F5E00001C0E12E802F90E004FF0CC0FE01E90D68
:10F5F000F11D2081203311F4097E09C0E39402FF3C
:10F6000006C004C086789070009709F0E394A02E9D
:10F61000BB2403FD14C000FF0FC0EF1428F4192D04
:10F620001F0D1E19EF2C08C0192D06C080E290E0B6
:10F63000B6010E940384E394EF14C0F304C0EF14F6
:10F6400010F4FE1801C0FF24A4FE0FC080E390E078
:10F65000B6010E940384A2FE1FC0A1FE03C088E57C
:10F6600090E010C088E790E00DC0C50186789070EA
:10F67000009791F0A1FC02C080E201C08BE207FD7F
:10F680008DE290E0B6010E94038406C080E390E022
:10F69000B6010E94038411509116C0F39A94F101AF
:10F6A000E90DF11D808190E0B6010E94038499204C
:10F6B000A9F706C080E290E0B6010E940384FA94A4
:10F6C000FF20C1F795CCF6012681378102C02FEFCC
:10F6D0003FEFC90163960FB6F894DEBF0FBECDBFF2
:10F6E000CF91DF911F910F91FF90EF90DF90CF901E
:10F6F000BF90AF909F908F907F906F905F904F9052
:10F700003F902F9008955058BB27AA270ED0CBC109
:10F71000BCD130F0C1D120F031F49F3F11F41EF480
:10F720008CC10EF4E095E7FB82C1E92FCDD180F3C7
:10F73000BA17620773078407950718F071F49EF5EE
:10F74000E5C10EF4E0950B2EBA2FA02D0B01B901E7
:10F7500090010C01CA01A0011124FF27591B99F047
:10F76000593F50F4503E68F11A16F040A22F232F53
:10F77000342F4427585FF3CF469537952795A795A3
:10F78000F0405395C9F77EF41F16BA0B620B730B4A
:10F79000840BBAF09150A1F0FF0FBB1F661F771FBB
:10F7A000881FC2F70EC0BA0F621F731F841F48F470
:10F7B000879577956795B795F7959E3F08F0B3CFF6
:10F7C0009395880F08F09927EE0F979587950895E0
:10F7D0005CD158F080E891E009F49EEF5DD128F00B
:10F7E00040E851E059F45EEF09C027C18FC1E92F0D
:10F7F000E0786AD168F3092E052AC1F32617370786
:10F800004807590738F00E2E07F8E02569F0E02583
:10F81000E0640AC0EF6307F8009407FADB01B9015E
:10F820009D01DC01CA01AD01EF9347D03CD10AD064
:10F830005F91552331F02BED3FE049E450FD49EC59
:10F8400063CF0895DF93DD27B92FBF7740E85FE3EB
:10F850001616170648075B0710F4D92F5ED19F9341
:10F860008F937F936F930FD2E0E2F1E0E9D01BD149
:10F870002F913F914F915F9163D1DD2349F09058D3
:10F88000A2EA2AED3FE049EC5FE3D0785D274DDF47
:10F89000DF9109C1A8D008F481E008950CD003C11C
:10F8A000FBD040F0F2D030F021F45F3F19F0BFC040
:10F8B00051112DC1C2C008D198F39923C9F3552322
:10F8C000B1F3951B550BBB27AA2762177307840753
:10F8D00038F09F5F5F4F220F331F441FAA1FA9F309
:10F8E00033D00E2E3AF0E0E830D091505040E695FB
:10F8F000001CCAF729D0FE2F27D0660F771F881F5C
:10F90000BB1F261737074807AB07B0E809F0BB0B4A
:10F91000802DBF01FF2793585F4F2AF09E3F51056E
:10F9200068F085C0F4C05F3FECF3983EDCF3869549
:10F9300077956795B795F7959F5FC9F7880F911DE4
:10F940009695879597F90895E1E0660F771F881FD0
:10F95000BB1F621773078407BA0720F0621B730B83
:10F96000840BBA0BEE1F88F7E0950895E89409C060
:10F9700097FB3EF490958095709561957F4F8F4FE2
:10F980009F4F9923A9F0F92F96E9BB279395F695F8
:10F99000879577956795B795F111F8CFFAF4BB0F76
:10F9A00011F460FF1BC06F5F7F4F8F4F9F4F16C0DA
:10F9B000882311F096E911C0772321F09EE8872F64
:10F9C000762F05C0662371F096E8862F70E060E020
:10F9D0002AF09A95660F771F881FDAF7880F969599
:10F9E000879597F90895990F0008550FAA0BE0E83D
:10F9F000FEEF16161706E807F907C0F012161306F1
:10FA0000E407F50798F0621B730B840B950B39F430
:10FA10000A2661F0232B242B252B21F408950A2696
:10FA200009F4A140A6958FEF811D811D089597F9D6
:10FA30009F6780E870E060E008959FEF80EC089594
:10FA4000DF93CF931F930F93FF92EF92DF927B018F
:10FA50008C01689405C0DA2EEF0172D0FE01E894A3
:10FA6000A5912591359145915591AEF3EF015DDE5C
:10FA7000FE019701A801DA9479F7DF90EF90FF90EB
:10FA80000F911F91CF91DF91089500240A941616CB
:10FA9000170618060906089500240A94121613067C
:10FAA000140605060895092E0394000C11F488230A
:10FAB00052F0BB0F40F4BF2B11F460FF04C06F5F26
:10FAC0007F4F8F4F9F4F089557FD9058440F551FFC
:10FAD00059F05F3F71F04795880F97FB991F61F0D0
:10FAE0009F3F79F087950895121613061406551F47
:10FAF000F2CF4695F1DF08C0161617061806991FB3
:10FB0000F1CF86957105610508940895E894BB27A7
:10FB100066277727CB0197F908959B01AC0160E038
:10FB200070E080E89FE3BACE0BD0BDCFAEDF28F007
:10FB3000B3DF18F0952309F07ACF7FCF1124E7CFF8
:10FB4000C3DFA0F3959FD1F3950F50E0551F629F3F
:10FB5000F001729FBB27F00DB11D639FAA27F00D26
:10FB6000B11DAA1F649F6627B00DA11D661F829F4D
:10FB70002227B00DA11D621F739FB00DA11D621F32
:10FB8000839FA00D611D221F749F3327A00D611D4F
:10FB9000231F849F600D211D822F762F6A2F112431
:10FBA0009F5750408AF0E1F088234AF0EE0FFF1F84
:10FBB000BB1F661F771F881F91505040A9F79E3FBB
:10FBC000510570F034CFA3CF5F3FECF3983EDCF3E8
:10FBD000869577956795B795F795E7959F5FC1F7F8
:10FBE000FE2B880F911D9695879597F90895FA0138
:10FBF000EE0FFF1F30962105310599F16115710552
:10FC000061F48038BFE39B0749F16894903881051F
:10FC100061F08038BFEF9B0741F0992342F5FF3F29
:10FC2000E1053105210511F1E8940894E795D90122
:10FC3000AA2329F4AB2FBE2FF85FD0F310C0FF5FCB
:10FC400070F4A695E0F7F73950F019F0FF3A38F460
:10FC50009F779F930CD00F9007FC905808953EF02B
:10FC6000ECCE60E070E080E89FE308954FE79F7777
:10FC70005F934F933F932F9375D02F913F914F9167
:10FC80005F9152DF08C09B01AC014ECF19F40EF01A
:10FC9000CECE3CCFD2CE20DFC8F39638C0F707F8DF
:10FCA0000F92E8942BE33AEA48EB5FE74BDF0F92C1
:10FCB0000F920F924DB75EB70F9294D0EDE4F1E042
:10FCC000BFDE4F915F91EF91FF91E595EE1FFF1F12
:10FCD00049F0FE57E0684427EE0F441FFA95E1F71C
:10FCE0004195550B06D00F9007FE17CF08959FCE74
:10FCF000ACC0F2DEE8F39923D9F3940F511DBBF3A6
:10FD00009150504094F059F0882332F0660F771FDD
:10FD1000881F91505040C1F79E3F510544F7880F0E
:10FD2000911D9695879597F908955F3FACF0983EA1
:10FD30009CF0BB27869577956795B79508F4B160D9
:10FD40009395C1F7BB0F58F711F460FFE8CF6F5FD1
:10FD50007F4F8F4F9F4FE3CFDACE0EF076C06DCE40
:10FD6000689465CEB9DEC8F39923D1F3C6F3DF9367
:10FD7000CF931F930F93FF92C92FDD2788232AF07B
:10FD80002197660F771F881FDAF720E030E040E800
:10FD90005FEB9FE3883920F0803E30F021968F772B
:10FDA000B3DCE5E7F1E003C0AFDCE2EAF1E048DE16
:10FDB0008B01BE01EC01FB2E6F5771097595771F02
:10FDC000880B990BD5DD28E132E741E35FE3B8DE2C
:10FDD000AF2D9801AE01FF900F911F91CF91DF9150
:10FDE000A4DC61CEFA01DC01AA0FBB1F9B01AC01B0
:10FDF000BF5728F422273327442750781FC0B75114
:10FE000088F4AB2F0024469537952795011CA395C0
:10FE1000D2F3002069F0220F331F441FB395DAF3A9
:10FE20000DD071CC61307105A0E88A07B94630F475
:10FE30009B01AC016627772788279078309621F0C0
:10FE4000208331834283538308959F3F31F0915043
:10FE500020F4879577956795B795880F911D9695AE
:10FE6000879597F90895629FD001739FF001829F53
:10FE7000E00DF11D649FE00DF11D929FF00D839F39
:10FE8000F00D749FF00D659FF00D9927729FB00DD6
:10FE9000E11DF91F639FB00DE11DF91FBD01CF01E9
:10FEA00011240895AA1BBB1B51E107C0AA1FBB1F49
:10FEB000A617B70710F0A61BB70B881F991F5A95F6
:10FEC000A9F780959095BC01CD01089597FB092E67
:10FED00007260AD077FD04D0E5DF06D000201AF40B
:10FEE000709561957F4F0895F6F7909581959F4F96
:10FEF0000895A1E21A2EAA1BBB1BFD010DC0AA1F6B
:10FF0000BB1FEE1FFF1FA217B307E407F50720F082
:10FF1000A21BB30BE40BF50B661F771F881F991FFD
:10FF20001A9469F760957095809590959B01AC0146
:10FF3000BD01CF01089597FB092E05260ED057FD70
:10FF400004D0D7DF0AD0001C38F450954095309586
:10FF500021953F4F4F4F5F4F0895F6F7909580954D
:10FF6000709561957F4F8F4F9F4F08952F923F92CD
:10FF70004F925F926F927F928F929F92AF92BF92B9
:10FF8000CF92DF92EF92FF920F931F93CF93DF9365
:10FF9000CDB7DEB7CA1BDB0B0FB6F894DEBF0FBEC2
:10FFA000CDBF09942A88398848885F846E847D840F
:10FFB0008C849B84AA84B984C884DF80EE80FD8011
:10FFC0000C811B81AA81B981CE0FD11D0FB6F89487
:10FFD000DEBF0FBECDBFED010895AF92BF92CF92AD
:10FFE000DF92EF92FF920F931F93CF93DF93EC0179
:10FFF000688179818A819B816115710581059105EF
:020000021000EC
:1000000021F464E279ED8BE597E02DE133EF41E0F7
:1000100050E00E949B7F79018A0127EA31E440E0A9
:1000200050E00E94337F5B016C01C801B7012CEEE8
:1000300034EF4FEF5FEF0E94337F6A0D7B1D8C1D05
:100040009D1D97FF04C061507040804090486883B8
:1000500079838A839B837F77CB01DF91CF911F9137
:100060000F91FF90EF90DF90CF90BF90AF900895E9
:100070000E94ED7F08958DE198E00E94ED7F089544
:10008000A0E0B0E080931D0890931E08A0931F0885
:10009000B093200808952F923F924F925F927F92E3
:1000A0008F929F92AF92BF92CF92DF92EF92FF9288
:1000B0000F931F93CF93DF934B01EA0161157105F5
:1000C00019F0FB0180839183209739F09E01225023
:1000D00030402332310508F0F4C0A82EB92EF501C6
:1000E00011915F017F01812F90E00E948083009732
:1000F000B1F71D3229F4F50111917F0101E006C02D
:100100001B3219F4F50111917F0100E0209719F0DD
:10011000C031D105B9F4103381F4F70180818837FB
:1001200011F0883551F4F701118182E090E0E80E7A
:10013000F91E0260C0E1D0E005C0209719F4103329
:10014000C1F422C0C830D105F9F0C930D10524F47A
:10015000C230D10509F507C0CA30D10551F0C03110
:10016000D105D1F427C0A12CB12CC12CF0E4DF2E95
:1001700026C0CAE0D0E0ECECAE2EECECBE2EECECEF
:10018000CE2EECE0DE2E1BC0C8E0D0E0A12CB12CBE
:10019000C12C70E1D72E13C09E01442737FD409536
:1001A000542F60E070E080E090E80E94797F590170
:1001B0006A0105C0A12CB12CC12C68E0D62E40E00C
:1001C00060E070E0CB011E01442437FC4094542CC5
:1001D00050ED752E710EE72DEA3070F0212F21546D
:1001E0002A3118F439EC732E06C0212F21562A31FA
:1001F00030F529EA722E710E272D30E02C173D07BD
:10020000F4F447FD18C0A616B706C806D90680F054
:10021000A20191010E94337F670D711D811D911D07
:100220006130F0E07F07F0E08F07F0E89F0710F003
:100230004FEF01C041E0F70111917F01C9CF811457
:10024000910491F0442339F00894E108F108F40195
:10025000F182E08209C001FF1BC0970122503040AB
:10026000F4013183208314C047FF12C000FF05C092
:1002700060E070E080E090E804C06FEF7FEF8FEF08
:100280009FE722E230E030937D2F20937C2F16C031
:1002900000FF08C090958095709561957F4F8F4FB6
:1002A0009F4F0CC097FF0AC082E290E090937D2F91
:1002B00080937C2F6FEF7FEF8FEF9FE79B01AC0167
:1002C00003C020E030E0A901B901CA01DF91CF915C
:1002D0001F910F91FF90EF90DF90CF90BF90AF9064
:1002E0009F908F907F905F904F903F902F900895B8
:1002F0002F923F924F925F926F927F929F92AF9216
:10030000BF92CF92DF92EF92FF920F931F93CF9302
:10031000DF933B01EA016115710519F0FB01808350
:100320009183209739F09E012250304023323105CD
:1003300008F0D5C0C82ED92EF60111916F017F01AA
:10034000812F90E00E9480830097B1F71D3231F435
:10035000F60111917F019924939406C01B3219F480
:10036000F60111917F019924209719F0C031D10530
:10037000D1F4103389F4F7018081883711F0883582
:1003800059F4F701118182E090E0E80EF91E92E045
:10039000992AC0E1D0E007C0209729F41033B1F0CA
:1003A000CAE0D0E02BC0CA30D10541F1C031D1053F
:1003B00021F0C830D105A9F409C02FEFA22E2FEFEC
:1003C000B22E2FEFC22E2FE0D22E20C0C8E0D0E0F8
:1003D0009FEFA92E9FEFB92E9FEFC92E9FE1D92E37
:1003E00015C09E01442737FD4095542F6FEF7FEFD6
:1003F000CB010E94797F59016A0108C089E9A82EC2
:1004000089E9B82E89E9C82E89E1D82E60E020E07C
:1004100030E0A9011E01442437FC4094542C012FE4
:1004200000530A3060F0812F81548A3110F4075054
:1004300006C0812F81568A3150F5012F0755802F34
:1004400090E08C179D071CF56F3FE9F0A216B306EC
:10045000C406D506A8F0CA01B901A20191010E9403
:10046000337F9B01AC01802F90E0A0E0B0E0280F2B
:10047000391F4A1F5B1F281739074A075B0710F40B
:100480006FEF01C061E0F70111917F01C8CF6114E6
:10049000710481F0662339F00894E108F108F30152
:1004A000F182E08207C091FE05C0C7010297F30107
:1004B0009183808390FE07C050954095309521959B
:1004C0003F4F4F4F5F4F67FF0DC082E290E0909328
:1004D0007D2F80937C2F2FEF3FEFA90103C020E0F9
:1004E00030E0A901B901CA01DF91CF911F910F91AD
:1004F000FF90EF90DF90CF90BF90AF909F907F9054
:100500006F905F904F903F902F90089566277727C8
:100510000C94A785FC0188279927E8942191203223
:10052000E9F3293010F02E30C8F32B3241F02D3290
:1005300039F4689404C00E94FB83820F911D2191BD
:1005400020532A30C0F31EF4909581959F4F089553
:10055000283008F027E03327DA01990F311D87FD95
:10056000916000966105710539F432602E5F3D930C
:1005700030E32A95E1F708959F3F30F08038710508
:10058000610509F03C5F3C5F3D93913008F0806865
:10059000911DDF93CF931F930F93FF92EF92192F2B
:1005A000987F9695E92F96959695E90FFF27EB5939
:1005B000F04F99273327EE24FF24A701E701059088
:1005C0000894079428F4360FE71EF81E491F511DA2
:1005D000660F771F881F991F0694A1F7059007944F
:1005E00028F4E70EF81E491F561FC11D770F881FFC
:1005F000991F661F0694A1F70590079428F4F80E3A
:10060000491F561FC71FD11D880F991F661F771FCF
:100610000694A1F70590079420F4490F561FC71FB1
:10062000D81F990F661F771F881F0694A9F784911A
:100630001095177041F0D695C79557954795F79443
:10064000E7941A95C1F7EBE0FFE0689415901591D7
:1006500035916591959105907FE27395E118F10AC6
:10066000430B560BC90BD009C0F7E10CF11E431F19
:10067000561FC91FD01D7EF4703311F48A95E6CF42
:10068000E894015030F0080F0AF40027021708F42C
:10069000202F2395022F7A3328F079E37D932A9532
:1006A000E9F710C07D932A9589F60694979567958A
:1006B000379517951794E118F10A430B560BC90BA0
:1006C000D00998F023957E9173957A3308F070E302
:1006D0007C932013B8F77E9170617D9330F0839501
:1006E00071E37D9370E32A95E1F71124EF90FF9079
:1006F0000F911F91CF91DF91992787FD90950895D4
:100700009111B3C3803219F089508550D0F7089504
:10071000FB01DC018D91059080190110D9F3990B33
:100720000895FC010590615070400110D8F7809544
:1007300090958E0F9F1F08954EE459E10E94D48337
:100740000895FB01DC0102C001900D924150504020
:10075000D8F70895DC0101C06D9341505040E0F797
:100760000895FB01DC018D91019080190110D9F3EE
:10077000990B0895FB01DC014150504048F0019075
:100780000D920020C9F701C01D9241505040E0F782
:100790000895FC016150704001900110D8F78095D8
:1007A00090958E0F9F1F0895FA01A191B081009737
:1007B00019F41097E1F0CD01DC01CD010D9000207E
:1007C00011F4C00113C0FB012191222319F020155F
:1007D000D9F7F3CFFB012191201519F41E92119640
:1007E00006C02223C1F70D900020A1F7D001FA0125
:1007F000A193B08308957AE0979F902D879F802DD5
:10080000910D112408950F931F93CF93DF938C01C3
:10081000EB018B8181FF1BC082FF0DC02E813F81C8
:100820008C819D812817390764F4E881F98101934F
:10083000F983E88306C0E885F985802F099500973C
:1008400031F48E819F8101969F838E8302C00FEFCA
:100850001FEFC801DF91CF911F910F910895DF9392
:10086000CF93CDB7DEB7FE0135966191719180913E
:10087000782F9091792FAF010E94D477CF91DF919B
:100880000895DF93CF93CDB7DEB7FE013596619122
:1008900071918091782F9091792FDC0113962C9192
:1008A0001397286013962C93AF010E94D477E091A0
:1008B000782FF091792F2381277F2383CF91DF91A8
:1008C0000895EF92FF920F931F93CF93DF938C01C4
:1008D000E091782FF091792F838181FF1FC0C0E0D4
:1008E000D0E00AC0DB011896ED91FC9119970995AB
:1008F000009711F0CFEFDFEFF80181918F01609148
:10090000782F7091792F882369F7DB011896ED9184
:10091000FC9119978AE00995009711F0CFEFDFEF6E
:10092000CE01DF91CF911F910F91FF90EF9008952D
:100930000F931F93DF93CF93CDB7DEB72E970FB6EC
:10094000F894DEBF0FBECDBF0D891E898F89988DAB
:1009500026E02C831A83098397FF02C080E090E889
:1009600001979E838D839E01255E3F4FCE010196A8
:10097000698D7A8DA9010E94D4774D815E8157FDE2
:100980000AC02F813885421753070CF49A01020FD1
:10099000131FF80110822E960FB6F894DEBF0FBE1B
:1009A000CDBFCF91DF911F910F9108950F931F93AA
:1009B000DF93CF93CDB7DEB72E970FB6F894DEBF97
:1009C0000FBECDBF8C01CB01BA0146E04C831A8328
:1009D000098397FF02C080E090E801979E838D8392
:1009E000CE010196A9010E94D4774D815E8157FD09
:1009F0000AC02F813885421753070CF49A01020F61
:100A0000131FF80110822E960FB6F894DEBF0FBEAA
:100A1000CDBFCF91DF911F910F910895FA01AA27C1
:100A2000283051F1203181F1E8946F936E7F6E5F31
:100A30007F4F8F4F9F4FAF4FB1E03ED0B4E03CD0DF
:100A4000670F781F891F9A1FA11D680F791F8A1FC2
:100A5000911DA11D6A0F711D811D911DA11D20D029
:100A600009F468943F912AE0269F11243019305DE3
:100A70003193DEF6CF010895462F4770405D4193D4
:100A8000B3E00FD0C9F7F6CF462F4F70405D4A3321
:100A900018F0495D31FD4052419302D0A9F7EACFE9
:100AA000B4E0A6959795879577956795BA95C9F718
:100AB00000976105710508959B01AC010A2E06940B
:100AC0005795479537952795BA95C9F7620F731FC4
:100AD000841F951FA01D0895DC01CB01FC01F9992D
:100AE000FECF06C0F2BDE1BDF89A319600B40D927A
:100AF00041505040B8F70895F999FECF92BD81BD9D
:100B0000F89A992780B50895A8E1B0E042E050E056
:100B10000C946E85DC01CB0103C02D910E9495855C
:100B200041505040D0F70895262FF999FECF1FBAB3
:100B300092BD81BD20BD0FB6F894FA9AF99A0FBE06
:100B4000019608950E949485272F0C9495856F92A5
:100B50007F928F929F92AF92BF92CF92DF92EF924D
:100B6000FF920F931F93DF93CF930F92CDB7DEB712
:100B70005B016115710521F0DB018C9311969C934B
:100B8000482F592F6A01F601E1906F018F018E2DD8
:100B900090E00E9480830097B1F7FE2DFD3229F48A
:100BA000D601ED908D0121E007C0BE2DBB3219F4B6
:100BB000F601E1908F0120E068010894C108D10896
:100BC000C60165E070E143E050E029830E94388768
:100BD0002981009711F572E0E72EF12CE00EF11E4D
:100BE000C70168E070E145E050E00E943887298144
:100BF000009729F467E0E62EF12CE00EF11EA11417
:100C0000B10421F0D5011196FC92EE9220FF0FC1A4
:100C100030E020E090E88FEF12C1C6016DE070E196
:100C200043E050E029830E9438872981009731F002
:100C300060E070E0CB01662477240AC0A114B104FF
:100C400009F4F9C00E5F1F4FF50111830083F3C053
:100C50003E2D30533A30A0F52260E22FF0E0AF0194
:100C60004870507022FF07C04115510571F5089476
:100C7000611C711C2AC04115510519F008946108C6
:100C800071086B017C0152E0CC0CDD1CEE1CFF1CDA
:100C90005A95D1F76C0D7D1D8E1D9F1D660F771F18
:100CA000881F991F630F711D811D911D6839F9E916
:100CB0007F07F9E98F07F9E19F0738F0246005C045
:100CC0003E3F39F423FD3FC02860D801ED908D01EF
:100CD000BFCF353311F03531B1F5F80131913D32E7
:100CE00011F4206102C03B3241F4D80111963C91CD
:100CF0001197319642E050E002C041E050E030539D
:100D00003A3020F08F01041B150B1DC040E050E06D
:100D1000BCE040385B075CF4DA01AA0FBB1FAA0FE6
:100D2000BB1F4A0F5B1F440F551F430F511D3191CD
:100D300030538F013A3060F324FF03C05095419542
:100D40005F4F640E751EC22EDD2421FF08C0A11462
:100D5000B10429F001501040F501118300830E9475
:100D6000B67C7B018C01F3E0CF22DD2433E0C31697
:100D7000D10421F417FB109517F91095C801B7019C
:100D800020E030E0A9010E944A7C882309F44AC08F
:100D900077FE09C044E2C42E40E1D42E70946194E1
:100DA0007108739404C03CE3C32E30E1D32E26E0D7
:100DB000822E912C90E2A92EB12C0FC0F601259124
:100DC000359145915491C801B7010E94947DE62E5A
:100DD000F72E082F192F6A187B086A147B0474F702
:100DE000B594A7940894810891088114910429F07E
:100DF0008CEF9FEFC80ED91EF0CFB701C801282F86
:100E0000220F292F221F2F3F39F020E030E0A901C7
:100E10000E944A7C882331F482E290E090937D2FF7
:100E200080937C2F3E2D2F2D902F812F08C030E0F6
:100E300020E090E803C030E020E090EC8FE7F9017B
:100E4000AC016F2F722F852F942F0F90CF91DF91D0
:100E50001F910F91FF90EF90DF90CF90BF90AF90D8
:100E60009F908F907F906F9008959927882708957D
:100E7000FB01DC014150504088F08D9181341CF021
:100E80008B350CF4805E659161341CF06B350CF48D
:100E9000605E861B611171F3990B0895881BFCCF6E
:040EA000F894FFCFF4
:100EA40054696D656F757420414444523D252D6429
:100EB4002E252D64205345513D252D642052535336
:100EC400493D252D75204C51493D252D750A002697
:100ED4003A202573205B414444523D252D642E2540
:100EE4002D64205345513D252D642054544C3D25FB
:100EF4002D7520525353493D252D75204C51493DA4
:100F0400252D75204452503D252D642E2530326404
:100F14005D0A00523D252D75204C3D252D7520532D
:100F24003D252D6420002C002845787450777229C3
:100F34000000415432344D4143004849483631336E
:100F44003000424D50303835004144584C3334352C
:100F540000484D4335383833004C33473432303051
:100F640044004D435033343258004E4844433032E9
:100F740031360065756936343D00253032780025F8
:100F84003032780A00736E3D00413A2025642025F2
:100F940064202564200A00433A2025642025642027
:100FA400256420613D25352E31660A007374617411
:100FB40075733D3078253032780A20006669726D89
:100FC400776172653D53322D352E322D32303134F6
:100FD4002D30332D313500656570726F6D006F7083
:100FE40065720072785F6C6564720074785F6C651A
:100FF400647900706B74006F77006C6564006576CB
:10100400656E740070305F6C6564720070315F6C83
:101014006564790061657300705F70777200707247
:10102400657300616363656C00636F6D70617373F6
:101034000072656C61795F6C656479007478740022
:10104400653634006964007400743100745F6D6344
:101054007500765F6D63750070300070305F7400EA
:1010640070310070315F7400757074696D65007261
:101074006800765F696E006131006132006133009F
:10108400616431006164320061643300616434007E
:1010940070007061006F6E006F6666007265736544
:1010A40074006E6F6E650073746174730074787489
:1010B4003D25730A00310032003300340035003618
:1010C40000636820706B74730025327520252D3100
:1010D40030750A006175746F00666C75736800443E
:1010E40055503D252D6420414444523D252D642E08
:1010F400252D64205345513D252D642054544C3DE9
:10110400252D752F252D7520525353493D252D75B9
:101114002F252D75204C51493D252D750A006465F8
:10112400657000666F7263655F69646C65007472F4
:10113400696D00746573740043683D252D64205403
:10114400785077723D252D640A004572726F7220C3
:101154005458204C656E6774683D25640A005458E1
:10116400543D2573200049443D004536343D00205C
:1011740050533D25640020543D252D362E32660003
:101184002054313D252D362E32660020545F4D43C8
:10119400553D252D352E31660020565F4D43553D76
:1011A400252D342E3266002050303D252D6C5800FC
:1011B4002050305F543D252D372E336600205031AA
:1011C4003D252D6C58002050315F543D252D372E80
:1011D4003366002055503D252D6C58002052483D63
:1011E400252D342E31660020565F494E3D252D3580
:1011F4002E32660020565F41313D252D352E326654
:101204000020565F41323D252D352E326600205692
:101214005F41333D252D352E30660020565F414415
:10122400313D252D382E36660020565F4144323D2F
:10123400252D382E36660020565F4144333D252D3A
:10124400382E36660020565F4144343D252D382E15
:1012540036660020503D252D6C64002050413D250C
:101264002D372E326600263A2025730A0054582062
:10127400706B74206C656E203D2025640A000100AB
:10128400D734EF3C22FFCC3B22FFCC3B1A20090D84
:101294002C00ED056162636465666768696A6B6C5E
:1012A4006D6E6F704D2001003C000A401A0F636D93
:1012B400642070726F636573730000000E06223839
:1012C40000000000737464696E2070726F6365734C
:1012D40073000000240648100000000062726F6171
:1012E40064636173742070726F63657373000000CC
:1012F4003C06FC3800000000536C65657020707279
:101304006F6365737300000058063A110000000013
:10131400506572696F6469632070726F636573737B
:1013240000000070067518000000001A0632064E10
:1013340006810666060000D50800001F004000581C
:1013440008980810000000C742BB421810000000B3
:10135400004576656E742074696D6572000000B195
:1013640006D246000000004374696D6572207072F5
:101374006F63657373000000C70610480000000027
:10138400020306070A0B0E0F020306070A0B0E0FD1
:101394002843292032303132204865726A756C66E0
:1013A4000055747665636B6C696E6720202020207D
:1013B4002000436F6E74696B6920322E3500000083
:1013C4000002000000003B5700000000C600C500FA
:1013D400C400C100C200000000CE00CD00CC00C992
:1013E40000CA00000000524632333020647269762D
:1013F40065720000004607F25B00000000635AE1DA
:1014040059415C8B5D045B94590258FC578359E540
:101414005800010101010101010101010101010162
:10142400010052696D65008207065FCD5E616461EB
:1014340074612E6E756D20776179206F75742074D8
:10144400686572653A2025640A0048604760516205
:101454008063B8610080C0E0F0F8FCFEFF6E756C3C
:101464006C6D616300BD07336418641E6424642AD0
:10147400643064736963736C6F776D616300D30761
:101484005465B5644B6434643A644864BA00080033
:10149400D712DF1235000200AF18B1185443502F91
:1014A400495020737461636B000000FC07AE670051
:1014B4000000000208FFFFFFFF0000000001000021
:0214C400000026
:00000001FF
